:1000000000800020BD010000410800000D08000034
:100010000D0800000D0800000D0800000D0800008C
:100020000D0800000D0800000D0800004108000048
:10003000410800000D080000C53B0000113E000013
:10004000410800004108000041080000410800008C
:10005000410800004108000041080000410800007C
:10006000410800004108000041080000410800006C
:10007000410800004108000041080000410800005C
:10008000410800004108000041080000410800004C
:10009000410800004108000041080000410800003C
:1000A000410800004108000041080000410800002C
:1000B000410800004108000041080000410800001C
:1000C000410800004108000041080000410800000C
:1000D00041080000410800004108000041080000FC
:1000E00041080000410800004108000041080000EC
:1000F00041080000591900004108000039210000A2
:1001000041080000DD260000410800004108000011
:1001100041080000410800004108000041080000BB
:1001200041080000410800004108000041080000AB
:10013000410800004108000041080000410800009B
:10014000410800004108000041080000410800008B
:10015000053F00001D3F0000353F00004D3F0000FF
:1001600041080000912A00004108000041080000F9
:10017000410800004108000041080000410800005B
:10018000410800004108000041080000410800004B
:10019000410800004108000041080000410800003B
:1001A000410800004108000041080000410800002B
:1001B0004108000041080000B93A0000584B4CF2D9
:1001C000205210B5DA814DF62812DA8100BF00BF47
:1001D00000F039FB534B4FF010621A63524A9A6396
:1001E000524ADA63524A136913F4807302BF5361AF
:1001F0004FF4A85313614F4B9A78100748BF9A7871
:100200004D4844BF42F008029A704C4B2A221A70A3
:100210004B4BDA1C121AC11E22F00302994288BF0E
:100220000022484905F0F2FF474B4848DA1C121AF1
:10023000C11E22F00302994288BF0022002106F06D
:1002400021F9434943484FF4DE7205F0DFFF424B8A
:10025000424A802103F8011B9342FBD14FF0E02377
:100260003C4AC3F8082D3E4B8A221A70A3F58053EE
:1002700024225A70A0221A709A799107FCD59A7993
:10028000D206FCD4374B9A7902F00C02082AFAD134
:1002900003221A7140225A719A799406FCD5314989
:1002A0008B795806FCD51F4B2F4A5A6402229A6458
:1002B00020220A708A7902F00C020C2AFAD12B4A09
:1002C0005A604FF0E0234BF67F325A6100229A6168
:1002D00007221A61264AC3F8202D62B600F08FFF6C
:1002E000134B5B69DA0705D5224800F0CDFC224BA1
:1002F000224ADA61224B1B785B0609D51E4C1F4B44
:10030000E2699A4204D11B4800F0BEFC0023E3617D
:1003100005F096FE00F09EFA04F0B6FCFEE700BF82
:100320000020054000800440823F04000100002BB3
:1003300000D0034000D007402087FF1F00E00740A7
:10034000B48FFF1FE82301001894FF1F1890FF1FB0
:10035000000000000082FF1F00E400E05FE400E016
:10036000005006400040064000001311C010050078
:10037000000020200000000000E00340A5C3945AC4
:1003800000F00740FFFFFFFFFFFFFFFFFFFFFFFF42
:10039000FFFFFFFFFFFFFFFFFFFFFFFFFFFFFFFF6D
:1003A000FFFFFFFFFFFFFFFFFFFFFFFFFFFFFFFF5D
:1003B000FFFFFFFFFFFFFFFFFFFFFFFFFFFFFFFF4D
:1003C000FFFFFFFFFFFFFFFFFFFFFFFFFFFFFFFF3D
:1003D000FFFFFFFFFFFFFFFFFFFFFFFFFFFFFFFF2D
:1003E000FFFFFFFFFFFFFFFFFFFFFFFFFFFFFFFF1D
:1003F000FFFFFFFFFFFFFFFFFFFFFFFFFFFFFFFF0D
:10040000FFFFFFFFFFFFFFFFFFFFFFFFDEF9FFFF23
:1004100018009FE518309FE5000053E11EFF2F01F3
:1004200010309FE5000053E31EFF2F0113FF2FE163
:10043000B48FFF1FB48FFF1F0000000024009FE552
:1004400024109FE5003041E0A31FA0E1431181E0AB
:10045000C110B0E11EFF2F0110309FE5000053E3F3
:100460001EFF2F0113FF2FE1B48FFF1FB48FFF1F5B
:100470000000000010402DE92C409FE50030D4E53D
:10048000000053E30600001AE0FFFFEB1C309FE57D
:10049000000053E318009F150000A0110130A0E3F5
:1004A0000030C4E51040BDE81EFF2FE11890FF1F8B
:1004B00000000000E023010020309FE5000053E32E
:1004C0000500000A10402DE914109FE514009FE577
:1004D0000000A0E11040BDE8D7FFFFEAD6FFFFEA29
:1004E000000000001C90FF1FE0230100F0B52B4A24
:1004F0002B4B516A0906FCD4586A10F08000F8D1E1
:1005000072B6284C2178002946D0956BD16BD2F871
:1005100040E0D2F844C0976CD66C294471446144E1
:1005200039443144C1F34E0141F40041D162956D2B
:10053000D16DD2F860E0D2F864C0976ED66E2944CF
:100540007144614439443144C1F34E0141F40041E6
:100550001163996BDA6BD3F840C05F6C9E6CDD6CF5
:100560000A4462443A4432442A44C2F34E0242F4FA
:100570000042DA62996DDA6DD3F860C05F6E9E6EEC
:10058000DD6E0A4462443A4432442A44C2F34E02C5
:1005900042F400421A63207062B6F0BD00B003401E
:1005A00000B00B403490FF1F1E4B602210B51A7034
:1005B0001D4CE1225A7021781C4A082903F58E232C
:1005C00018D1012090601321D16098601848D9603B
:1005D00043781649174A03B101230B62136261780D
:1005E000124A144B012910D880215162596201230B
:1005F000037010BD0A2901D13920E3E70C290CBF93
:1006000035203D2012219060DEE7042901D88421A5
:10061000EBE7082901D88521E7E7102994BF862157
:100620008721E2E7004007401C88FF1F00B003401D
:100630003490FF1F00B00B400D4B5A7858B1AAB947
:10064000012159701B7823B10A4B5A6203F500232C
:100650005A62FFF7A9BF4AB158701B78002BF8D037
:10066000044B586203F500235862F2E7704700BF5D
:100670003490FF1F00B003400C2810B417D9102885
:1006800028BF102010230F4A0F49181A90700878BD
:100690009842DCB214D013780C702BB10B4A0023B3
:1006A000536202F50022536210BCFFF77DBF0A2897
:1006B00004D808288CBF0A230823E4E70C23E2E7C8
:1006C00010BC70473490FF1F1C88FF1F00B0034010
:1006D00010B5144B1B7804460BB1FFF707FF012C34
:1006E000114A04D800235362104A537010BD042CE1
:1006F0000F4903D8042353624B62F5E7082C04D852
:10070000052353624B620823EEE7102C95BF0623A6
:1007100007235362536295BF4B624B621023202321
:10072000E2E700BF3490FF1F00B003401C88FF1FAA
:1007300000B00B402828F8B543D8234B1D5CFF2D93
:100740003FD0224C23780BB1FFF7D0FE290616D5F7
:1007500072B61F4E05F0400705F03F05F36837B34A
:1007600023F01003F36001233560237162B672B683
:1007700033681B061ED50023306923710CE072B666
:10078000144E01273560E77062B672B633681A06F8
:1007900006D500233069E37062B6A3781841F8BD2E
:1007A000E378002BEED062B604F086FAEDE743F072
:1007B0001003D7E72379002BD0D062B604F07CFA7F
:1007C000D5E70020EBE700BFF41C01003490FF1FC9
:1007D00000B00B4000B00340094AD36A43F4805391
:1007E000D362084B5A78084B3AB1802280F30C0050
:1007F00000B283F8212018807047C022F6E700BFBE
:10080000008004403490FF1F00C00C4008B50B4C22
:10081000636B580301D502F03BF9636B590501D5B1
:1008200001F09AF8636B1A0501D501F085FC636B42
:10083000DB04EDD501F052FFEAE700BF0080044081
:1008400008B5FFF7E3FF024B10221A80704700BF84
:100850000020054070470A4908B5034608685BB1A7
:100860006A460344A2F58052934206D305F0D8FBB2
:100870000C2303604FF0FF3008BD0B60FCE700BFA6
:100880002088FF1F002070474FF0FF3070474FF463
:1008900000534B6000207047012070474FF0FF303D
:1008A0007047FEE7FEE70078B0FA80F04009704735
:1008B000012303707047EFF31380A0B9EFF31083A7
:1008C0009BB9EFF305825AB10F2A01D9074B9B5C04
:1008D000EFF3118212B1934228BF134618467047B6
:1008E0004FF48073F4E74FF0FF307047F0E300E01F
:1008F000FEE7FFFF70B5044608460021B4FBF2F5A1
:1009000002FB1546F3B2092E94BF30333733DBB206
:10091000A242435402D801312C46EFE7431800228B
:100920005A70441E8D1AAA4200DB70BD14F8015F94
:100930001E782670013203F80159F3E7031E10B543
:100940000C4603DBBDE81040FFF7D4BF2D2001F8B3
:10095000010B5842FFF7CEFF204610BD2DE9F04FA6
:1009600081EAE17885B08946A8EBE1780146054641
:1009700017461C4605F0E8F898B30021284605F014
:10098000B3F8002814BF0426032646450ADAB9F155
:10099000000FA8EB060606DA20463246202105F0B5
:1009A00071FD3444002628464FF07E5363F31E0049
:1009B000002105F099F810B12D2304F8013B4123E3
:1009C0004E2263702270E31CA2701846324620212A
:1009D00005F058FD034600229A55304405B0BDE8A5
:1009E000F08F25F000467849304605F0ADF868BB39
:1009F0003046754905F084F8064638BB0021284684
:100A000005F072F8002840F0D880B8F1030F1BDD24
:100A10000326B9F1000FA8EB060606DA3246204697
:100A2000202105F02FFD344400260021284605F042
:100A30005BF810B12D2304F8013B492323704E23AA
:100A400063704622E31CBFE70646EEE702AB01AA4D
:100A50003946284605F0F8F9019B57EA030280461B
:100A60004ED10278594B5A48342A94BF9846804652
:100A700001230193404606F051F9019B834206464B
:100A8000B8BF461C002B43D10136DDF808B0BBF1DE
:100A9000000F00D00136A9EB0605002D04EB060A75
:100AA00060DD2A462021204605F0ECFCAA446319AB
:100AB000BBF1000F02D02D2203F8012BDDF804C09A
:100AC000BCF1000F50D137B11A46302102F8021B99
:100AD0002E21597013462E219A451D465FD8B9F133
:100AE000000F09DA4E44764226EAE6762846324678
:100AF000202105F0C7FC354400232B7020466DE70C
:100B00005B429F42BEBF7B42DFF8C0800193B1E7EA
:100B1000BBDA002FB9D03B44984207F10206B4D9A2
:100B2000DFF8B0A0B84606E02846514604F006FEBD
:100B300008F1FF380546B8F1000FF5DC002FACBF17
:100B4000F91B394602AB03AA284605F07DF9019B43
:100B5000039A791CD21A8A4208BF0133804608BF23
:100B6000019392E72346A3E7B5DA002FB3D01946E5
:100B7000302501F8025B2E225A70CCF10202134498
:100B800000200A469A4206D1A1EB0C030028A2D00D
:100B9000002201929FE702F8015B0120F2E718F8BA
:100BA000012B05F8012BAA4599D0019A013A01922F
:100BB0000AB99D1C59702B468EE7B8F1040F7FF7D8
:100BC00039AF042625E700BFFFFF7F7F1D1D010011
:100BD0001F1D010000002041704700F14040A0F5BA
:100BE00092237C2B12D9A0F594237C2B10D9A0F54D
:100BF00096237C2B0ED9A0F598237C2B0CD9A0F53D
:100C00009A207C28054888BF002070470448704718
:100C1000044870470448704704487047FC88FF1F29
:100C20004488FF1F7C88FF1FCC88FF1F2488FF1F7C
:100C3000024B103043F82010704700BF0082FF1FA6
:100C400008B50C4B03EBC0035A681046FFF7C5FF0D
:100C500070B172B6136823F0877323F4803343F0C6
:100C600080731360C2F38402034B40F8223062B6F3
:100C700008BD00BF241D0100D90B0000014B1868FE
:100C8000704700BF00D00340034B00225A615A60F6
:100C9000102218605A61704700D00340002816DB0C
:100CA00003024FF48071B3F5004F0A4601F1FF31A2
:100CB00004D30129A3EB000207D10A461B0A013A1B
:100CC00043EA02230D4AD36070471346EBE76FF007
:100CD000FF0343434FF48071B3F5014F0A4601F11E
:100CE000FF3104D3012900EB030204D10A461B0A99
:100CF000C3F58073E3E71346EEE700BF00D003407F
:100D00001028034628BF1023044A012B38BF0123B3
:100D100092F8E00082F8E030704700BF2488FF1F9F
:100D20002DE9F8430E4605462949304604F0DCFE1D
:100D3000284B002847F6122812BF022701279846A1
:100D400000244FF05E5928FA04F004F085FC49466F
:100D500004F0F4FC0146304604F0DEFE10B9013424
:100D6000072CF0D128FA04F004F076FC314604F0A8
:100D7000B1FD4FF07C5104F08FFB04F001FF4FF602
:100D8000FF73984228BF1846EB1E012B08D8124B60
:100D9000002244EAC7041A605A6098601C6014E09C
:100DA000172D05D9202D01D0192D0ED10B4BEFE7B2
:100DB0000B4BEB40DB4313F0010306D1094A44EA35
:100DC000C7041360536090601460BDE8F88300BFEF
:100DD000001BB740006CDC020090034000800B4019
:100DE0006006F00000800340212810B509D80D4BA3
:100DF00053F8302092F880423CB1012311B182F8BF
:100E0000803010BD82F80031FBE703EBC00043687F
:100E10001A6819B142F003021A60F2E722F00202E6
:100E2000FAE700BF241D010021289FBF034B53F8A0
:100E30003030012283F88021704700BF241D01005B
:100E400021289FBF044B53F8303093F80002C0B202
:100E500088BF0020704700BF241D0100212817D83B
:100E6000144A02EBC00301295B6852F8300001D03C
:100E700004290ED1012280F880224FF4A2721A6058
:100E80001A6804290CBF42F0200222F020021A60E6
:100E90007047002280F8802211B94FF48072F6E783
:100EA000022902D140F20312F1E7032908BF4FF4EF
:100EB0008172ECE7241D0100212870B50E4632D85E
:100EC000042A30D8184B1A4403EBC00392F810419F
:100ED0005D68296811F4E0614FEA044401D1FFF72D
:100EE000BDFF124B124AC3F89C21124AC3F8A0213D
:100EF000114AC3F8A421114AC3F8A8212846104A70
:100F0000C3F8AC21FFF769FE68B172B62B6823F411
:100F100070232B601C43C5F3840344F0807440F8B5
:100F200023602C6062B670BD241D01000082FF1F8B
:100F3000E987FF1FB987FF1F8587FF1F5587FF1FA1
:100F40002187FF1F38B5514B282893F8E03004461D
:100F50000CD10B2B95BFC3F10C030C3B01FA03F032
:100F600041FA03F0BDE83840FFF736BC01250029FF
:100F700005FA03F204DC0021FFF736FF012104E04B
:100F8000914207D32946FFF72FFF2046BDE838409E
:100F9000FFF764BFC21ED0B2012818D83C48806851
:100FA00000FB011020FA03F31D2A69D8DFE802F0E4
:100FB0004C5345336868252C6868686868686868B9
:100FC00068373E171E68616868686868685A202C30
:100FD00001D0192C01D12F48E1E72F48DFE72E4A35
:100FE00013612E4B40F244425A6038BD2A4A936145
:100FF0002A4B40F244429A60F7E7274A1362274B94
:1010000040F24442DA60F0E7234A9362234B40F215
:1010100044421A61E9E7204A1363214BF7E71E4A6D
:1010200093631F4B40F244425A61DEE71A4A13644D
:101030001B4B40F244429A61D7E7174A9364184B1E
:1010400040F24442DA61D0E7114A1361154B4FF484
:1010500051721A63C9E70E4A9361124B4FF45172F1
:101060005A63C2E70B4A13610F4B4FF451729A64F3
:10107000BBE7084A93610C4B4FF45172DA64B4E752
:101080007F29D4BF00210121204675E72488FF1F56
:101090000090034000800B400080034000B00440FB
:1010A00000C004400090044000A004402DE9F0413D
:1010B00007460D4690460826012408EA04013846F2
:1010C000FFF792FE01212846FFF78EFE00212846F9
:1010D000FFF78AFE6400013EE4B2EED1BDE8F08184
:1010E0002DE9F04107460C4690460825802608EA7F
:1010F00006013846FFF778FE01212046FFF774FE0F
:1011000000212046FFF770FE013D4FEA5606EED162
:10111000BDE8F08110B414461A4614B910BCFFF7AC
:10112000C5BF10BCFFF7DCBF2DE9F04180460D467E
:1011300008270026012428460121FFF755FE4046D6
:10114000FFF77EFE00B1264300212846FFF74CFE44
:101150006400013FE4B2EED13046BDE8F0812DE9F4
:10116000F04180460C4608260025802720460121B4
:10117000FFF73AFE4046FFF763FE00B13D43002112
:101180002046FFF731FE013E4FEA5707EED12846D1
:10119000BDE8F0810AB9FFF7C7BFFFF7E0BF72B63D
:1011A0004FF0E0210A4A8B691268D1F8041D62B63B
:1011B000490102D5322B88BF0132C3F53B433020B1
:1011C0007F33B3FBF0F34FF47A7000FB02307047CB
:1011D0003C90FF1F38B50446FFF7E1FF05466CB1B0
:1011E000FFF7DDFF401BB0F57A7F02D203F064FD0C
:1011F000F6E7013C02D005F57A75F1E738BD4FF00E
:10120000E0234FF4000210B5C3F808214FF08072BC
:10121000C3F808214FF00072C3F808214FF0806234
:10122000C3F808214FF00062C3F80821154A2823AB
:1012300009214BF6FF70002454609060D360536125
:10124000D3615362D3625363D3635364116002F575
:10125000805254609060D3605361116002F5FE22A9
:1012600054609060D36053611160FFF79DF91920BD
:10127000FFF7B0FF02F0CCF8BDE8104040F21310C9
:10128000FFF7A8BF0080034070B50546C1EBC1045D
:101290002B7853B92B7863B1FFF781FF06462B7883
:1012A00053B9FFF77CFF801B02E0013CF0D1002026
:1012B00070BD013CEED1FAE7013CF0D1F7E770B523
:1012C0000546C1EBC1042B7853B12B7863B9FFF706
:1012D00066FF06462B7853B1FFF761FF801B02E0E3
:1012E000013CF0D1002070BD013CEED1FAE7013C99
:1012F000F0D1F7E721280B46114609D8054A52F8E4
:10130000300000F500700BB1FFF7BEBFFFF7D7BF8D
:1013100000207047241D0100254A536B43F480636D
:101320005363244B00221A705A709A70DA701A7143
:101330005B7943B3152B2BD01F4B1B78012B2CD083
:10134000052B2FD020281D4B38BF2020C0F344325E
:101350001A70C0F347125A7000F01F0004220221D5
:1013600098729A70D9745A7588221A743C22DA706D
:10137000134B402283F82D204FF0E0234FF400520E
:10138000C3F8042170470F4B40F213321A64D3E7BD
:101390000D4B40F213329A61CEE70A4B4FF4517273
:1013A0005A64CFE7084B4FF45172DA61CAE700BFC5
:1013B000008004404090FF1F0889FF1F00A00640E6
:1013C00000E400E000A0044000C0044010B5204A42
:1013D000937800F0030103F0EC030B43440748BF8C
:1013E00043F01003937000F00F03042B08BF9379B0
:1013F000184C04BF43F040039371154A5379C1065A
:1014000003F0EF0348BF43F0100353719379820652
:1014100003F0EF030E4A48BF43F0100310F40070CE
:1014200093710D4B0ED0917841F0A00191700B4A51
:101430009C6011780A4A02EBC10240F247315268BF
:10144000116010BD9A68A24208BF9860F9E700BF1A
:1014500000A00640D400D4424090FF1F0889FF1F1F
:10146000241D01001F4B5B6B5B0510B522D51E4C84
:10147000237903F0FF02F3B94FF0E0234FF400515A
:10148000C3F88411194BDA706379BBB1152B1AD0EC
:10149000174B1B7803F07F03012B19D0052B1CD0B1
:1014A000124B1A79DB79002323706370E3680BB168
:1014B00001221A7010BD03F0FFFBD9E70D4B40F27B
:1014C00003121A64E4E70C4B40F203129A61DFE75F
:1014D000084B40F203125A64E2E7074B40F2031252
:1014E000DA61DDE7008004404090FF1F00A0064065
:1014F0000889FF1F00A0044000C0044070B50A4DD9
:1015000004462B7903F0FF06002BFAD10121204677
:10151000FFF7A4FC31462046FFF766FC034B53F867
:101520003430AB6070BD00BF4090FF1F241D010030
:1015300010B509B140F08000154A1378834214D0E9
:10154000144C646B64050FD503F07F03012B0DD0A1
:10155000052B0FD0002900F07F0114BF6023442326
:1015600001290BD005290ED0107010BD0A4B0024A4
:101570005C64EFE7094B0024DC61EBE7064943F4C8
:1015800040734B64F0E7054943F44073CB61EBE7EC
:101590000889FF1F0080044000A0044000C00440F0
:1015A000104A537983420AD00F49496B490505D542
:1015B00033B1152B07D050B115280DD0507170479D
:1015C0000A490B64F7E70A4B00219961F3E7074BDF
:1015D00040F213311964F1E7054B40F21331996180
:1015E000ECE700BF4090FF1F0080044000A00440D3
:1015F00000C0044038B50D4B5B6B13F480634FF0B3
:10160000000410D021280A4D0AD80A4B012153F8B2
:101610003030EB60FFF722FCEB6801201C7038BD16
:10162000EC602046FBE71846F9E700BF0080044065
:101630004090FF1F241D0100104B0246586B10F410
:1016400080600CD0122A03F5083309D10C4A40F20D
:101650000231D1605A7B42F001025A730120704777
:10166000142A04D1074A40F202315161F2E75A7B51
:1016700002F0FE025A730020704700BF0080044051
:1016800000A0044000C00440274B5B6B5A052DE9C5
:10169000F041064622D5254DAB680BB101221A70E8
:1016A000DFF88C80AC78D8F80430224F01349C42AB
:1016B00028BF0024EB78A34212D03F2C8ABF2A6DAA
:1016C0002B19A4F14003F6B28CBFD6541E7401232B
:1016D0002B71184BE4B2BC22AC70DA70BDE8F0811B
:1016E000FFF7E9F8402819DC3B791B06E2D5EB78D7
:1016F000D8F80410DAB201338B4209D23F2B09D853
:10170000EA18127CD2B2D2B2DBB2FA71EB70D1E736
:101710000023F5E7296D3F3A8A5CF3E7FF28C9DD2E
:1017200003F0CAFAC6E700BF008004404090FF1FE4
:101730000889FF1F00A0064000F00F00092894BF91
:1017400030303730FFF7A0BF2DE9F8432D4B5B6BEE
:101750005A0507460ED52C4DAB680BB101221A7005
:10176000DFF8A890DFF8A8807E18B74204D3284B92
:10177000BC22DA70BDE8F883AC78D9F804300134C3
:10178000A34298BF0024EB78A34208D03F2C17F85F
:10179000011B2FD92A6DA4F14003D1542CE0BC23A6
:1017A00088F80330FFF787F840281EDC98F80430EB
:1017B0001B0610D5EB78D9F80420D9B201339A4230
:1017C0000DD93F2B0DD8EA18127CD2B2D2B2DBB2BF
:1017D00088F80720EB70EB789C42E3D0D6E7002333
:1017E000F1E72A6D3F39525CEFE7FF28F3DD03F0A4
:1017F00063FAF0E72B1919740123E4B22B71AC7072
:10180000B3E700BF008004404090FF1F0889FF1F1E
:1018100000A0064010B5034C237903B910BD03F0B6
:101820004BFAF9E74090FF1F084B9978DB78994213
:10183000DAB222BF064B5B6803F1FF33C8B22CBF9C
:101840009B1802F1FF33181A704700BF4090FF1F2A
:101850000889FF1F064A117852789142D0B23CBFE6
:10186000044A9268CBB238BF9B18181A704700BF61
:101870004090FF1F0889FF1F70B5164A11785378F2
:101880009942CCB2D8B221D0134DA968431C9942D9
:1018900015D93F2B15D8D01890F85400DEB25670E9
:1018A000D268C0B252B19C423CBF0919CB1AE96858
:1018B00028BFE31A8B4201D80023137070BD0023A8
:1018C000E9E7D2F894603F38305CE7E74FF0FF304B
:1018D000F4E700BF4090FF1F0889FF1F0D4B1878E9
:1018E00059788842CAB212D00B488068511C88428D
:1018F00006D93F2906D80B4493F85400C0B270476C
:101900000021F8E7D3F894303F3A985CF6E74FF0BF
:10191000FF3070474090FF1F0889FF1F0B4B5B6B28
:101920005B0512D50A4BDA7802F0CB02DA7040225E
:101930005A74DA7842F03402DA70064B5A78D2B22E
:101940001A70DB680BB100221A70704700800440E7
:1019500000A006404090FF1FF0B5424F3B7913F0C6
:10196000300F09D072B6BB7D03F0FF04002B3BD1D2
:10197000FB7940237B7462B63A48C3781E06DDB219
:1019800023D503791C0620D5374C384AA678E3784E
:101990005768D4F850C0F6B2DBB2B3420DD0591C30
:1019A0008F4254D80379002163181A7CD2B2D2B284
:1019B000C271027D072A0B46EFD9DBB2E370294BD7
:1019C0001A79100644BF7C22DA7069060BD5254BC4
:1019D0001A79520607D5244A00211171926802B182
:1019E00011703C22DA70F0BD62B61F48DFF87CC08F
:1019F00003784278D0F894E0D6B2DCF80820DBB265
:101A0000FD79591C8A42EDB228D98E4205D03F2972
:101A100019D8431883F854500B46013C14F0FF04C6
:101A2000EED1D9B20170C1680029A5D0B3423CBF44
:101A3000921B9B18DCF8102028BF9B1B934224BFED
:101A400001230B7098E73F3B0EF80350E4E73F2972
:101A50000279A9D93F3B1CF80320A7E7002EDCD070
:101A60000021D6E700A006404090FF1F0889FF1F15
:101A700038B5441E14F8015F05B938BD0A2D02D1EE
:101A80000D20FFF701FE2846FFF7FEFDF2E710B537
:101A900004460009FFF750FE2046BDE810404BE623
:101AA00010B50446000AFFF7F2FF2046BDE81040DB
:101AB000FFF7EDBF10B50446000EFFF7E8FF200C5E
:101AC000FFF7E5FF200AFFF7E2FF2046BDE81040E0
:101AD000FFF7DDBF074BC3F8940048B101F14002A6
:101AE000054B9A6001F11A022831DA6019617047DA
:101AF0004022F5E74090FF1F0889FF1F044B18653F
:101B000018B14031034B596070474021FAE700BFDC
:101B10004090FF1F0889FF1F254A536B43F4006361
:101B20005363244B00221A705A709A70DA701A713B
:101B3000214B1A78092A27D01A2A2AD05B780A2B37
:101B40002CD01F2B2FD020281C4B38BF2020C0F3B7
:101B500044321A70C0F347125A7000F01F0004227A
:101B6000022198729A70D9745A7588221A743C228C
:101B7000DA70134B402283F82F204FF0E0234FF40C
:101B80000042C3F8042170470E4A40F21331D1607D
:101B9000D4E70D4A40F213315160CFE7094B4FF4BF
:101BA00051721A61CFE7084B4FF451721A60CAE7BD
:101BB00000800440D890FF1F1C89FF1F00B0064022
:101BC00000E400E000B0044000D0044010B5204A1A
:101BD000937800F0030103F0EC030B43440748BF84
:101BE00043F01003937000F00F03042B08BF9379A8
:101BF000184C04BF43F040039371154A5379C10652
:101C000003F0EF0348BF43F010035371937982064A
:101C100003F0EF030E4A48BF43F0100310F40070C6
:101C200093710D4B0ED0917841F0A00191700B4A49
:101C30009C6051780A4A02EBC10240F24731526877
:101C4000116010BD9A68A24208BF9860F9E700BF12
:101C500000B00640D400D642D890FF1F1C89FF1F59
:101C6000241D0100204B5B6B1B0510B523D51F4CB9
:101C7000237903F0FF02FBB94FF0E0234FF400415A
:101C8000C3F884111A4BDA701A4B1A78092A16D045
:101C90001A2A19D05B7803F07F030A2B19D01F2B67
:101CA0001CD0134B1A79DB79002323706370E3682F
:101CB0000BB101221A7010BD02F0FEFFD8E70E4AE8
:101CC00040F20311D160E5E70C4A40F20311516084
:101CD000E0E7094B40F203121A61E2E7074B40F2DA
:101CE00003121A60DDE700BF00800440D890FF1F98
:101CF00000B006401C89FF1F00B0044000D0044023
:101D000070B50A4D04462B7903F0FF06002BFAD17B
:101D100001212046FFF7A2F831462046FFF764F87C
:101D2000034B53F83430AB6070BD00BFD890FF1F39
:101D3000241D010010B509B140F08000154A537808
:101D4000834214D0144C646B24050FD503F07F0339
:101D50000A2B0DD01F2B0FD0002900F07F0114BFDC
:101D6000602344230A290BD01F290ED0507010BDC8
:101D70000A4B00241C61EFE7094B00241C60EBE7D1
:101D8000064943F440730B61F0E7054943F440739F
:101D90000B60EBE71C89FF1F0080044000B004408B
:101DA00000D00440114A137883420CD01049496B8B
:101DB000090507D5092B07D01A2B09D009280BD004
:101DC0001A280ED0107070470A4B0021D960F5E731
:101DD000094B00215960F1E7064B40F21331D960FD
:101DE000F0E7054B40F213315960EBE71C89FF1F08
:101DF0000080044000B0044000D0044038B50D4BD2
:101E00005B6B13F400634FF0000410D021280A4DDF
:101E10000AD80A4B012153F83030EB60FFF71EF867
:101E2000EB6801201C7038BDEC602046FBE71846CB
:101E3000F9E700BF00800440D890FF1F241D010077
:101E40000C4B0246586B10F4006012D0172A03F5B1
:101E50000C3309D1084A40F2023191605A7B42F0BA
:101E600001025A73012070475A7B02F0FE025A7336
:101E7000002070470080044000B00440274B5B6B9B
:101E80001A052DE9F041064622D5254DAB680BB168
:101E900001221A70DFF88C80AC78D8F80430224F19
:101EA0000134A34298BF0024EB78A34212D0272C20
:101EB0008ABFAA6B2B19A4F12803F6B28CBFD654A3
:101EC0001E7401232B71184BE4B2BC22AC70DA7083
:101ED000BDE8F081FEF7EFFC402819DC3B791B06DA
:101EE000E2D5EB78D8F80410DAB20133994209D977
:101EF000272B09D8EA18127CD2B2D2B2DBB2FA711F
:101F0000EB70D1E70023F5E7A96B273A8A5CF3E78A
:101F1000FF28C9DD02F0D0FEC6E700BF0080044004
:101F2000D890FF1F1C89FF1F00B006402DE9F84321
:101F30002D4B5B6B1A0507460ED52C4DAB680BB1CC
:101F400001221A70DFF8A890DFF8A8807E18B74247
:101F500004D3284BBC22DA70BDE8F883AC78D9F8FA
:101F600004300134A34298BF0024EB78A34208D088
:101F7000272C17F8011B2FD9AA6BA4F12803D154E1
:101F80002CE0BC2388F80330FEF795FC40281EDCCB
:101F900098F804301B0610D5EB78D9F80420D9B294
:101FA00001339A420DD9272B0DD8EA18127CD2B2F0
:101FB000D2B2DBB288F80720EB70EB789C42E3D01A
:101FC000D6E70023F1E7AA6B2739525CEFE7FF2839
:101FD000F3DD02F071FEF0E72B1919740123E4B26E
:101FE0002B71AC70B3E700BF00800440D890FF1F96
:101FF0001C89FF1F00B0064010B5034C237903B9BC
:1020000010BD02F059FEF9E7D890FF1F084B9978F0
:10201000DB789942DAB222BF064B5B6803F1FF33EB
:10202000C8B22CBF9B1802F1FF33181A704700BFCB
:10203000D890FF1F1C89FF1F064A117852789142E1
:10204000D0B23CBF044A9268CBB238BF9B18181A72
:10205000704700BFD890FF1F1C89FF1F70B5154A3D
:10206000117853789942CCB2D8B220D0124DA968D9
:10207000431C994215D93F2B15D8D01890F83C0035
:10208000DEB25670D268C0B252B19C423CBF091950
:10209000CB1AE96828BFE31A8B4201D800231370DA
:1020A00070BD0023E9E7D66F3F38305CE8E74FF0BA
:1020B000FF30F5E7D890FF1F1C89FF1F0D4B1878E4
:1020C00059788842CAB211D00B488068511C8842A6
:1020D00006D93F2906D80B4493F83C00C0B270479C
:1020E0000021F8E7DB6F3F3A985CF7E74FF0FF30ED
:1020F000704700BFD890FF1F1C89FF1F0B4B5B6B05
:102100001B0512D50A4BDA7802F0CB02DA704022B6
:102110005A74DA7842F03402DA70064B5A78D2B246
:102120001A70DB680BB100221A70704700800440FF
:1021300000B00640D890FF1FF0B5424F3B7913F036
:10214000300F09D072B6BB7D03F0FF04002B3BD1EA
:10215000FB7940237B7462B63A48C3781E06DDB231
:1021600023D503791C0620D5374C384AA678E37866
:102170005768D4F838C0F6B2DBB2B3420DD0591C60
:102180008F4254D80379002163181A7CD2B2D2B29C
:10219000C271027D072A0B46EFD9DBB2E370294BEF
:1021A0001A79100644BF7C22DA7069060BD5254BDC
:1021B0001A79520607D5244A00211171926802B19A
:1021C00011703C22DA70F0BD62B61F48DFF87CC0A7
:1021D00003784278D0F87CE0D6B2DCF80820DBB295
:1021E000FD79591C8A42EDB228D98E4205D03F298B
:1021F00019D8431883F83C500B46013C14F0FF04F7
:10220000EED1D9B20170C1680029A5D0B3423CBF5C
:10221000921B9B18DCF8102028BF9B1B934224BF05
:1022200001230B7098E73F3B0EF80350E4E72729A2
:102230000279A9D9273B1CF80320A7E7002EDCD0A0
:102240000021D6E700B00640D890FF1F1C89FF1F71
:10225000074BD86748B101F14002064B9A6001F183
:102260001A022831DA60196170474022F5E700BF91
:10227000D890FF1F1C89FF1F044B986318B12831A9
:10228000034B596070472821FAE700BFD890FF1F21
:102290001C89FF1F174A536B43F480535363164A3C
:1022A0000023137053709370D3701371134A40F26C
:1022B0001331916020284FF45171D16038BF202034
:1022C00002F50032C0F344311170C0F3471100F041
:1022D0001F0051709072937013742C23D370084BAD
:1022E000402283F831204FF0E0234FF40032C3F84E
:1022F00004217047008004405891FF1F00C0044033
:1023000000E400E010B5204A937800F0030103F0E8
:10231000EC030B43440748BF43F01003937000F0F5
:102320000F03042B08BF9379184C04BF43F04003FC
:102330009371154A5379C10603F0EF0348BF43F088
:10234000100353719379820603F0EF030E4A48BFDE
:1023500043F0100310F4007093710D4B0ED0917880
:1023600041F0A00191700B4A9C6011780A4A02EB7F
:10237000C10240F247315268116010BD9A68A24212
:1023800008BF9860F9E700BF00C00640D400D842FB
:102390005891FF1F3089FF1F241D0100114B5B6BFB
:1023A000DB0410B519D5104C227902F0FF03AAB94D
:1023B0004FF0E0224FF40031C2F884110B4A0C496F
:1023C000D37040F203108860C8601179D27923700D
:1023D0006370E3680BB101221A7010BD02F06CFC4F
:1023E000E2E700BF008004405891FF1F00C0064094
:1023F00000C0044070B50A4D04462B7903F0FF0677
:10240000002BFAD101212046FEF728FD3146204657
:10241000FEF7EAFC034B53F83430AB6070BD00BFED
:102420005891FF1F241D010010B509B140F0800034
:102430000E4A1378834217D00D4C646BE40412D516
:1024400003F07F03082B02BF0A4B0024DC60002945
:1024500000F07F010CBF44236023082902BF054917
:1024600043F44073CB60107010BD00BF3089FF1F74
:102470000080044000C00440704738B50C4B5B6BD3
:1024800013F480534FF0000410D02128094D0AD8CE
:10249000094B012153F83030EB60FEF7DFFCEB68AD
:1024A00001201C7038BDEC602046FBE71846F9E7B8
:1024B000008004405891FF1F241D01000C4B024670
:1024C000586B10F4805012D00E2A03F5103309D146
:1024D000084A40F2023151605A7B42F001025A73BD
:1024E000012070475A7B02F0FE025A7300207047A9
:1024F0000080044000C00440274B5B6BDA042DE9E8
:10250000F041064622D5254DAB680BB101221A7069
:10251000DFF88C80AC78D8F80430224F01349C422C
:1025200028BF0024EB78A34212D0272C8ABFAA6BC5
:102530002B19A4F12803F6B28CBFD6541E740123C4
:102540002B71184BE4B2AC22AC70DA70BDE8F081AC
:10255000FEF7B1F9402819DC3B791B06E2D5EB7890
:10256000D8F80410DAB201338B4209D2272B09D8EC
:10257000EA18127CD2B2D2B2DBB2FA71EB70D1E7B8
:102580000023F5E7A96B273A8A5CF3E7FF28C9DD4A
:1025900002F092FBC6E700BF008004405891FF1F85
:1025A0003089FF1F00C0064038B504464518AC42CC
:1025B00000D138BD14F8010BFFF79EFFF7E710B507
:1025C000034C237903B910BD02F076FBF9E700BF95
:1025D0005891FF1F084B9978DB789942DAB222BFF5
:1025E000064B5B6803F1FF33C8B22CBF9B1802F1A6
:1025F000FF33181A704700BF5891FF1F3089FF1F23
:10260000064A117852789142D0B23CBF044A92688F
:10261000CBB238BF9B18181A704700BF5891FF1FE4
:102620003089FF1F70B5154A117853789942CCB2A2
:10263000D8B220D0124DA968431C994215D93F2B1E
:1026400015D8D01890F83C00DEB25670D268C0B2EF
:1026500052B19C423CBF0919CB1AE96828BFE31A62
:102660008B4201D80023137070BD0023E9E7D66FB9
:102670003F38305CE8E74FF0FF30F5E75891FF1F37
:102680003089FF1F0D4B187859788842CAB211D093
:102690000B488068511C884206D93F2906D80B4454
:1026A00093F83C00C0B270470021F8E7DB6F3F3A77
:1026B000985CF7E74FF0FF30704700BF5891FF1F5D
:1026C0003089FF1F044B5A78D2B21A70DB680BB105
:1026D00000221A70704700BF5891FF1F70B5304B31
:1026E0001A79960627D52F4A2F4DD8791378A968DD
:1026F00054780133994298BF00239C42C0B20BD05A
:102700003F2B8BBFD66FD418A3F1400484F83C0054
:1027100088BF3055D8B21070D06860B1D478A34269
:10272000E2B22CBF9B1A891A2A6938BF5B18934200
:1027300024BF012303701A4AD3781D06DCB20AD5E0
:102740001379180607D517498D78C8788542C3B222
:1027500010D16C23D37061060BD5114B1A79520638
:1027600007D5104A00211171926802B111702C2214
:10277000DA7070BD0C4840685A1C90420AD9272A6A
:102780000AD88B181B7C0648DBB2DBB2D2B2C3710D
:10279000CA70E0E70022F4E7886B273BC35CF2E7EE
:1027A00000C006405891FF1F3089FF1F074BD867B4
:1027B00048B101F14002064B9A6001F11A0228313A
:1027C000DA60196170474022F5E700BF5891FF1F9A
:1027D0003089FF1F044B986318B12831034B5960AF
:1027E00070472821FAE700BF5891FF1F3089FF1F6B
:1027F0001FB572B6154B70221A704122DA710F2282
:102800009A7180221A701A781206FCD5986862B6FE
:102810000F4B984238BF0A234FF00A0201A938BF74
:102820005843FEF767F80B4801A9002211F8014B45
:102830001346013224B10A2A20F81240F6D1134679
:1028400001335B00037004B010BD00BF0000024004
:10285000809698004489FF1F431E032B10D872B640
:10286000084A52F8230048B102EB4301D0F804C0F3
:1028700042F823C00B8A02889B1A0B8262B670470B
:1028800000207047D891FF1F013803280DD8094B4D
:1028900003EB8000836972B64BB100201A885B6835
:1028A0001044002BFAD162B67047002070471846DA
:1028B000F9E700BFD891FF1F013803280CD872B682
:1028C000074B03EB8000836943B100205B68013054
:1028D000002BFBD162B67047002070471846F9E71D
:1028E000D891FF1F72B62D4A1378190705D52C4BC6
:1028F000196A00293BD0996A41B353781B0706D562
:10290000274B196C002943D0996C00293AD0937851
:10291000190706D5224B196E00293CD0996E002963
:1029200033D0D3781B070AD51D4BD3F880204FF046
:10293000100CF2B1D3F888204FF0110C42B162B6FE
:10294000184B002283F8282000F0C4BD4FF0050C7E
:1029500003EBCC0213490830506091F8282012484C
:1029600043F83C00013A81F8282062B670474FF0E6
:10297000040C03EBCC020B490830506091F828207E
:102980000A48EDE74FF0090CE2E74FF00D0CDFE7E6
:102990004FF0080CEDE74FF00C0CEAE73C1E01008D
:1029A0000080FF1FD891FF1FC80040008800400032
:1029B000421E032A12D81F4B400140F0100010B5F0
:1029C000184472B61C4B03EB020C9CF82CC0BCF1F3
:1029D000030F22D8DFE80CF01619031D70474FF0E3
:1029E000050CB1F800E010F0080F134414BFC82222
:1029F000882242EA0E420831C0E9002183F82CC047
:102A000062B610BD4FF0030CEBE708304FF0020C3C
:102A1000E7E708304FF0040CE3E703EB8200920095
:102A2000846924B1006B41601A441163E8E7816155
:102A3000FAE700BF0080FF1FD891FF1F00F1FF3CA5
:102A4000BCF1030F1CD80F4B400140F0100010B533
:102A5000184472B60C4B03EB0C0494F82C4064B190
:102A600008304FF0000E6344120442F08002C0E9C7
:102A7000002183F82CE062B610BD4FF0010EF2E7A2
:102A8000704700BF0080FF1FD891FF1F00BE00BF2E
:102A90002DE9F04FDFF8D0B2B44C85B03FE0B44E32
:102AA0008F0806EBC708551ED8F8042011F008015E
:102AB000EDB2A2F1080340F0EC8056F837004FEA7F
:102AC000104E000C22F808EC00F0DC8022F8061C06
:102AD00042F8041C54F82510002900F0448204EB4D
:102AE0008502A900D26D536004EB450521442A8A72
:102AF000CB6572442A8200F0CFFC002800F02B82C4
:102B00009C499D4A18F0080F00F1080008BF0A46CA
:102B1000C8F8040046F8372008228BF880209BF87C
:102B200080205607D5B21CD594F84820B2B194F84D
:102B3000491001F0FF0231B1013AD2B284F84920C4
:102B4000002A00F061848D48017801F0FF0229B16C
:102B5000013AD2B20270002A00F0308204228BF8CF
:102B6000802015F0080200F011829BF89020D1B26D
:102B7000120994D1DFF8F891890809EBC10659F8D8
:102B800031007668C0F38300092800F0B08010D8C7
:102B90000138012809D8B4F84C5042F2210085428E
:102BA00000F02482744849F8310001228BF8942007
:102BB000B2E70D28F9D1D6E900766F4849F831001F
:102BC00040F2816CB9B201206145C4E913766265B7
:102BD000C9F81020C9F8182084F8580000F2EB80DA
:102BE000B1F5D06F80F0EE82B1F5817F00F0CE823A
:102BF00040F2C88040F20230814240F0AF8006F0DF
:102C00007F06042E00F2EB81380C40F0E8815C4B2B
:102C100013F8261041F0020103F826100146B4F81B
:102C2000526094F86CC0B0424CF0020828BF3046A5
:102C300009EBC806402871604FF00107064628BF1F
:102C400040264FF0C80E4EEA064549F83850314448
:102C50008CF00105861B84F8582084F86C5040F0F5
:102C6000BF803F2840F2D88045F0020509EBC5003F
:102C7000012F416084F8587084F86CC040F02E82B7
:102C800088212CE23B493C4A18F0080F08BF0A464D
:102C900040E7184600F01EFC04EB8500816900291E
:102CA00000F065814A688261601901F1080290F8BC
:102CB0002C00C8F80420032807D8DFE800F0120F22
:102CC00015022544042285F82C2018F0080F0988E5
:102CD00014BFC822882242EA01421BE7254402228F
:102CE000F1E725440322EEE725440522EBE7606D7A
:102CF00038B3B4F86E7094F8586094F86C50402F64
:102D0000394628BF4021002E86F0010684F858601D
:102D100045F0020685F0010584F86C5009EBC60504
:102D2000686014BFC825882545EA01450844791A1A
:102D300089B249F83650A4F86E10002900F041819C
:102D40006065B4F84C20B2F5A06F01BF94F84E2036
:102D5000002184F84D108BF8982026E7B1F5A06F7C
:102D600040F03D81002059E700200740D891FF1F27
:102D70000080FF1F88004000C8004000D592FF1F60
:102D8000C0200740802900F01182822940F027816D
:102D900006F07F06042E00F222810021AC4BA4F83D
:102DA000401013F826108D0702D5012184F8401039
:102DB000A849022033E742F2210C61452CD033D9D7
:102DC00042F2212081422BD1B6B2002ECAD1A249B3
:102DD0000E68A2490E60A249C7F307400870C1E718
:102DE00045F00205402E304684F8587028BF402038
:102DF000012F09EBC50784F86CC0796014BFC827A0
:102E0000882747EA00470144301A49F8357000F036
:102E100061816165A4F86E0001228BF89420C4E6FC
:102E200042F2213081429BE7B1F5086F00F0C48186
:102E3000B1F5106F40F0D380D9F82010C7F30740E8
:102E400084F84800080600F1D881D9F8281009064E
:102E500000F16482D9F830100A0600F15982D9F8DD
:102E600038100B0600F14E82D9F840100F0600F121
:102E70004382D9F848100E0600F13882D9F8501074
:102E80000D0600F12D82D9F85810080600F12282B3
:102E9000D9F86010090600F11782D9F868100A06FF
:102EA00000F15482D9F870100B0600F14982D9F86C
:102EB00078100F0600F13E82D9F880100E0600F15E
:102EC0003382D9F888100D0600F14C82D9F89010A1
:102ED000080600F14182D9F89810090600F1EE8148
:102EE000604E06F12C03019306F13003039306F1C3
:102EF0005C03002506F1100A06F11808029356F843
:102F0000047B2FB138467F6800F0E4FA002FF9D136
:102F1000029BD8F8007043F8045B46F8045C029307
:102F20002FB138467F6800F0D5FA002FF9D1039B06
:102F300048F8045B43F8045B0393019B2AF8025BA7
:102F400019780239032900F2D480DFE811F01C015E
:102F5000CE001C01CE0094F8282046F8370001323C
:102F600084F82820D8E544F82530A900BCE525449C
:102F700095F82C20022A00F0A2807FF6CDAD032A1E
:102F800040F0A080012285F82C20C5E5E8076FD429
:102F900029061AD4AA0708D5334B93F888200221B2
:102FA000D2B283F8882083F88010EB0603D52E4B2D
:102FB000102283F8802005B0BDE8F08F00F008FCF7
:102FC000CCE53F2F98BF0020BAE6274B80220D2189
:102FD00083F8C01083F88020AA07E6D5DCE70F222B
:102FE0008BF8C02001228BF89420DEE5B4F8500065
:102FF000A0B91E483578057075784570B57885702C
:10300000F578C570056837790771862D7779B679B7
:103010004771867104BF0F2084F8490094F8585016
:1030200094F86C00002D85F0010584F8585040F0AC
:10303000020580F0010084F86C0018BFC82609EB77
:10304000C50008BF882649F8356000254560A9E518
:10305000C02007401892FF1F3C90FF1FD892FF1F0F
:10306000D692FF1FD891FF1F00200740DC92FF1F60
:10307000C64BC749C748C84C022583F8945080F80E
:103080006C200C608C6000F1B00470304860CC6043
:10309000FF200D2483F8C04083F888009F240A6134
:1030A00083F880008A6183F89820012283F88C00DD
:1030B00083F8844083F8942005B0BDE8F08F85F84C
:1030C0002C1029E518F0080F14BF0322022285F8FE
:1030D0002C2021E53F2E3FF69CAE9DE6C821012223
:1030E00049F835108BF894205FE5019B4FF0010201
:1030F0001A70019B01330193A84B9E427FF4FFAEEF
:10310000A74D002184F8281029788BF8C4100A07ED
:1031100000F1BD8069788BF8C81000200B07C9F852
:103120003000C9F8380000F18580A9788BF8CC1000
:1031300000200F07C9F85000C9F8580063D4E97897
:103140008BF8D01000200E07C9F87000C9F878007D
:1031500000F1878094F86CC094F858704CF0020825
:1031600009EBC8000021C9F89010C9F89810416017
:1031700087F00102002F40F0488139463E4638462C
:103180004FF0880E5FE5019B1D70B2E706F07F06E9
:10319000042E3FF624AF3B0C7FF421AF814B13F894
:1031A000261021F0020103F82610DBE50021A4F827
:1031B000401002207C4932E594F8481084F8401011
:1031C00079492CE57948416800293FF408AF3F0C64
:1031D000B6B204E001690C3000293FF400AFB0F84A
:1031E00000C0BC45F6D1B0F802C0B445F2D13F0AE8
:1031F000032F0CBF0878008911E5D9F8240008389E
:1032000000F068F921E600F047F9002800F0E880B6
:103210000830C9F864006048C9F8600000F03CF963
:10322000002800F0D5806249C9F868100830C9F854
:103230006C0084E700F030F9002800F0DF800830EF
:10324000C9F844005448C9F8400000F025F90028A6
:1032500000F0CC805649C9F848100830C9F84C0035
:1032600063E700F019F9002800F08A800830C9F8F7
:1032700084004948C9F8800000F00EF9002877D092
:103280004B49C9F888100830C9F88C0062E700F093
:1032900003F9002800F096800830C9F824003E4861
:1032A000C9F8200000F0F8F8002800F083804049B9
:1032B000C9F828100830C9F82C002BE7D9F89C0071
:1032C000083800F007F90BE6D9F86400083800F078
:1032D00001F9E2E5D9F85C00083800F0FBF8D7E521
:1032E000D9F85400083800F0F5F8CCE5D9F84C00CE
:1032F000083800F0EFF8C1E5D9F84400083800F0CC
:10330000E9F8B6E5D9F83C00083800F0E3F8ABE599
:10331000D9F83400083800F0DDF8A0E5D9F82C0021
:10332000083800F0D7F895E5D9F88400083800F09F
:10333000D1F8C6E5D9F87C00083800F0CBF8BBE539
:10334000D9F87400083800F0C5F8B0E5D9F86C0079
:10335000083800F0BFF8A5E5D9F89400083800F067
:10336000B9F8B8E5D9F88C00083800F0B3F8ADE545
:1033700094F82810C9F88800013184F82810E9E68B
:1033800094F82810013184F8281073E700200740D2
:103390000080FF1FD891FF1F88004000E891FF1FA9
:1033A0003C1E0100C02007401892FF1F401E010074
:1033B000C800400094F82810C9F82800013184F8AA
:1033C0002810A7E694F82810013184F8281067E740
:1033D00094F82810C9F86800013184F82810AEE686
:1033E00094F82810013184F8281015E794F8281073
:1033F000C9F84800013184F8281096E694F828109E
:10340000013184F828101EE700BE0E46084618E475
:1034100070B5FFF7EDF91B48002200F1A00103464B
:10342000C3E9002208338B42FAD1174C174B616B6A
:10343000174D41F480216163C0F3072483F89C4059
:10344000144CFF214FF0010CC0F30746000E83F827
:10345000B0604FF0E02E83F8B40083F8801083F85A
:103460008810197483F894C0227083F884C0702384
:1034700085F849304FF400721023CEF808212372EA
:1034800070BD00BF0080FF1F008004400020074087
:1034900000E400E00021074072B60C480268B2FA6E
:1034A00082F30B2B02DD62B6002070474FF0004123
:1034B000D94022EA0102026062B60549482253431C
:1034C000C8180022CA504260704700BFE489FF1F3D
:1034D000BC83FF1F0D4BC31AB3F5587F14D20C4A9F
:1034E000127822B10B4A12780AB1FFF7FBB972B613
:1034F000094A48201168B3FBF0F34FF0004020FA6E
:1035000003F30B43136062B6704700BFBC83FF1F19
:103510000092FF1F2092FF1FE489FF1F38B5104C57
:10352000236863B120684388C2180133157A028882
:103530009A4212D8FFF7CEFF0023236004E0094B24
:103540001B781BB94FF0FF35284638BD0320FFF725
:1035500083F920600028E5D1F4E74380F4E700BF59
:10356000C892FF1F2092FF1F10B50B4C236823B198
:1035700023686BB94FF0FF3010BD084B1B78002B50
:10358000F8D00320FFF768F920600028F0D1F1E7B8
:103590005A881344187AEFE7C892FF1F2092FF1F42
:1035A000044B9888044B1A681AB1138852889B1AE6
:1035B00018447047E891FF1FC892FF1F2DE9F0479C
:1035C000DFF87C901F4F06460D464FF0000815B9F6
:1035D0004046BDE8F08799F80030002BF8D03B68F2
:1035E00053B90320FFF738F938600028F0D003887A
:1035F00013B9FFF76FFFF4E7D7F800A05346BAF806
:10360000021033F8084B641AAC4228BF2C462246FD
:103610001944304602F0FAFDBAF80220BAF8003038
:103620002644A0442D1B1444A4B2A342AAF802408D
:10363000CDD85046FFF74EFF00233B60C7E700BFE1
:103640002092FF1FC892FF1F10B5094B1B786BB16A
:10365000084C206818B1FFF73DFF002323600320CA
:10366000FFF7FAF810B1FFF735FFF8E710BD00BF1C
:103670002092FF1FC892FF1F2DE9F0472A4CDFF868
:10368000AC80012781460D4627710E4616B926717A
:1036900028460BE0A3680BBB47F2095A98F80030A4
:1036A00003F0FF0223B922714FF0FF30BDE8F0872D
:1036B0000420FFF701F9072805D82771FFF7ECFE72
:1036C000A06058B92071BAF1010A01D0237B13B16F
:1036D00001232373E8E701F0EFFADFE7A168002395
:1036E00023734B88C3F14002B24228BF3246981878
:1036F0000B444880B61A073309EB020AD1450DD1B5
:103700004B883F2B06D940230B800420FFF750F94C
:103710000023A36005236373D146B7E719F8012B93
:1037200003F8012FEAE700BFC892FF1F2092FF1F96
:1037300007B501218DF807000DF10700FFF79CFF89
:1037400003B05DF804FB10B50D4C01232371A36891
:103750007BB90C4B1B7813B90020207110BD0420DD
:10376000FFF7AAF80728F7D8FFF796FEA060002811
:10377000F2D0A36858880023C0F140002371EDE720
:10378000C892FF1F2092FF1F70B50F4B1B787BB1B3
:103790000E4CA568012626715DB16B880026667304
:1037A00029462B800420FFF703F9A660002323712C
:1037B00070BDFFF771FE014620B104206573FFF76D
:1037C000F7F8F3E76673F1E72092FF1FC892FF1F37
:1037D00038B50D4C237903F0FF053BB9A16831B131
:1037E0004B880B800420FFF7E3F8A56038BDFFF796
:1037F00053FE014620B1BDE838400420FFF7D8B899
:1038000001236373F2E700BFC892FF1FC029F0B520
:1038100028BFC02172B6134B0022C3E90222C3E9BC
:103820000422C3E9062218609A80012791420BD036
:10383000550903EB850502F01F04AE6807FA04F48E
:103840003443AC600132F1E7002302304FF482745C
:103850009A4204D004FB03F143520133F8E762B605
:10386000F0BD00BFE492FF1F70B572B61B4B988885
:1038700003F1080202EB800503F12006B542294658
:1038800002D362B6002070BD55F8044B0CB901306C
:10389000F4E7B4FA84F64FF00045F54024EA050455
:1038A0000C6004B901301C8C98800134A5B21D84D1
:1038B00062B60B48891A41F67C7200FB0622891019
:1038C0004FF4025000FB0122196801268E5488181B
:1038D0005A8CA24238BF5D84D5E700BFE492FF1F37
:1038E000FCFEFFFF10B5438872B60278012A03D9A7
:1038F000013A027062B610BD0A4A580902EB800410
:10390000DB434FF0004103F01F0321FA03F3A168EA
:103910000B43A36093888342138C88BF9080013B44
:103920001384E7E7E492FF1F30B5C3687BB1187AD0
:1039300090420AD158685C7A006950F8245025B941
:1039400040F82410087801300870DB68EEE730BDDD
:10395000437A8B4288BF02694FF0000386BF52F85A
:10396000210042F821301846704738B5437A8B421F
:1039700002D80024204638BD036953F821400022B4
:1039800043F82120002CF4D02378012BF2D9FFF743
:103990006BFF054628B14FF48072211D043002F000
:1039A00035FC2378013B23702C46E3E7037C30B5DC
:1039B00033BB4368427A5B7A9A4221D872B6036875
:1039C000DA6872B9D8600022C2609A7A01329A72BB
:1039D00001221A724368997A1A7211449972027418
:1039E0000DE01146D26862B10C68A342F9D1456876
:1039F0004C68A542F5D10C8901898C42F1D162B69F
:103A000030BDC860DFE7037C10B504464BB14368A6
:103A1000427A5B7A9A4204D872B60368DA680AB9C5
:103A200062B610BD904204BFC268DA604368427A51
:103A30001B6953F8220040B1FFF754FF72B6636868
:103A4000627A1B69002143F822102268937A013BB5
:103A5000DBB2937203B913726268937A013BDBB2F3
:103A6000937203B9137200232374D9E7094B93F8B7
:103A700024206AB9084AD02182F85E104FF0E02273
:103A80004FF080410120C2F8081183F824007047EC
:103A900000207047E492FF1F00E400E04FF0E023B5
:103AA0004FF08042C3F88821024B002283F8242083
:103AB000704700BFE492FF1F4FF0E0222DE9F04174
:103AC000D2F8FC3D174D184E43F08073C2F8FC3D10
:103AD0002B68B46A43F001032B606F68A4B1237AAA
:103AE00083B12368D5F804801B68204698476A682C
:103AF000E388A2EB0802C2F30F11B3EB121FA180FF
:103B000038BFE1806469E9E7064BF18D5B68DB1B38
:103B1000C3F30F12B1EB131FB28538BFF285BDE8B6
:103B2000F08100BF001000E0E492FF1F10B5EFF33A
:103B3000108472B6427F5AB9037F012B10D1134B08
:103B4000196841B9C0E9051118605860012343772D
:103B500004B962B610BD42615A6882615061F4E7EF
:103B6000032BF3D1094B996851B9C0E9051198604D
:103B7000D8604FF0E0234FF08052C3F8042DE5E702
:103B80004261DA6882615061F2E700BF1493FF1F5F
:103B900038B50B4C0025EFF3108272B6A06858B10F
:103BA0004369A36033B19D6102B962B6836845770A
:103BB0009847F0E7E360F7E702B962B638BD00BFA7
:103BC0001493FF1FFFF7E4BF30B50346EFF31084F3
:103BD00072B6407F88B11A7F012A11D1D3E905124C
:103BE00022B15161596921B18A6104E00C4D29600B
:103BF000F8E70B494A6000225A7704B962B630BD33
:103C0000032AF8D1D3E9051232B15161596900296B
:103C1000EAD10349CA60EEE7014DA960F6E700BFAB
:103C20001493FF1F037F012B11D1437F63B1D0E9B0
:103C3000052323B15A61426922B1936104E00D4921
:103C40000A60F8E70B4A5360002303777047032BA1
:103C50000FD1437F002BF7D0D0E9052333B15A6150
:103C60004269002AE9D1034AD360EDE701498A603D
:103C7000F6E770471493FF1F0023C360EFF3108231
:103C800072B6044B1969186101238160037502B98A
:103C900062B670471493FF1F16494B6970B52BB974
:103CA000C0E9023348610223037570BD04681A68D5
:103CB000944206D20025121B8360C560D8601A604A
:103CC000F0E7194605680E689B68AC1B046063B199
:103CD0001A68A242F5D9D968C1608360D860C1680A
:103CE0003244521B88601A60DDE7C0E90231886007
:103CF000D9E700BF1493FF1F10B5EFF3108172B620
:103D0000037D022BDAB212D183682BB1C26804683A
:103D1000DA601A6822441A60C2682AB193600023EC
:103D2000037501B962B610BD0A4A5361F7E7012A6B
:103D3000F7D1084A1369834203D183681361EEE720
:103D40001346002BEBD09A688242F9D182689A60C0
:103D5000E5E700BF1493FF1F037D70B505460C46D1
:103D600016460BB1FFF7C8FF64B1022C38BF02241E
:103D7000023C00232E612C606B602846BDE8704039
:103D8000FFF77ABF70BD037D70B504460D46164639
:103D90000BB1FFF7B1FF65B1022D2B4638BF0223EF
:103DA000023BC4E9003526612046BDE87040FFF7BC
:103DB00063BF70BD70B5154D6C6900261CB12368DA
:103DC0007BB1013B2360EFF3108372B600222869B8
:103DD0002A6103B962B6B8B18468FFF75DFF204677
:103DE000F9E7A26802B1D36020696A6103682675A9
:103DF0001B6822460021984763681BB12360204658
:103E0000FFF74AFF6C69D9E770BD00BF1493FF1F2D
:103E1000024A136801331360704700BF3C90FF1FD4
:103E2000024A136801331360FFF7C4BF3C90FF1FC1
:103E30007047036830B5EBB100249C600124DC605E
:103E40000468194B226023441B110322174DA26002
:103E5000174A45F823100179995444335A1102F155
:103E600038224032920003F01F03012000FA03F3CE
:103E7000136017E00F4CE36B43F40003E36300BFF0
:103E80000D4B01241C6003F580730C4C0360036828
:103E90009D68002DD4D01033A3420360F7D90023CE
:103EA0000360184630BD00BF008FFCBFE889FF1FCC
:103EB00044E400E000800440007003403F71034090
:103EC00030B50468B4B10C4A2244121102F1440125
:103ED0004B1103F1382360339B0001F01F010125D2
:103EE00005FA01F11960054B054943F8221000233A
:103EF000A360036030BD00BF008FFCBFE889FF1FD7
:103F0000313E0000034B0122C3F80C21024B1B6819
:103F1000184700BF00700340E889FF1F034B0122D0
:103F2000C3F81C21024B5B68184700BF00700340B8
:103F3000E889FF1F034B0122C3F82C21024B9B6829
:103F4000184700BF00700340E889FF1F034B0122A0
:103F5000C3F83C21024BDB68184700BF00700340E8
:103F6000E889FF1FFFFFFFFFF8B507460C4659B170
:103F70008D180026AC4208D03B6814F8011B1B6862
:103F8000384698470644F5E70E463046F8BDF0B58A
:103F9000012A8BB008BF0A22A9B930228DF825204A
:103FA00021243BB1631E0AAADCB252FA83F32D220C
:103FB00003F8242C036801A95B68C4F122022144A0
:103FC00098470BB0F0BD2124B1FBF2F602FB1617A7
:103FD000FDB2092F0AAF94BF303537352744EDB213
:103FE0008A4207F8245CDCD8013CE4B23146EBE7B6
:103FF0002DE9F04100268D688AB004460F46B04690
:1040000095B13346212201A9384600F094FC23687B
:10401000202D2A465B6828BF202201A9204616448D
:10402000AD1A98478044EBE740460AB0BDE8F081FE
:104030000029BABF49422D2300230A22A7E707B56A
:1040400040F60D23ADF80430036802225B6801A935
:10405000984703B05DF804FB10B5036814465B682D
:104060009847204610BD0EB403B503AA52F8041BAE
:10407000019206F0C5F802B05DF804EB03B070479A
:104080000EB403B503AA52F8041B019206F0B8F867
:1040900002B05DF804EB03B0704730B422B9036896
:1040A00030BC1B68C9B2184730BC70E72DE9F04737
:1040B00092B080469DF868909DF86CA0B9F1010F10
:1040C00017461E4637D952EA06031AD130238DF817
:1040D00045304125BAF1000F07D06B1E12AADDB2A0
:1040E00052FA83F32D2203F8442CD8F8003001A9AA
:1040F0005B68C5F1420229444046984712B0BDE8CA
:10410000F08741254A4600233846314601F062FDDA
:10411000D4B2092C12AB94BF303437342B44E4B200
:104120004F4503F8444C76F10003D3D3013DEDB283
:1041300007460E46E6E70020E0E713B51C1E0BDA43
:104140000A2352424FF0010CCDE9003C64EB4403DA
:10415000FFF7ACFF02B010BD0A210024CDE9001426
:10416000F6E72DE9F04F85B00546194610469DF853
:10417000386092461C4601F0C7F840B14E492846C7
:1041800000F0AAF80446204605B0BDE8F08F24F000
:1041900000474A4B4FF0FF325046394601F0B4F821
:1041A00048B9464B4FF0FF325046394601F088F887
:1041B00008B94349E3E7434B4FF06042504621467C
:1041C00001F096F808B14049D9E7404B4FF0604202
:1041D0005046214601F068F80028F4D1002200235F
:1041E0005046214601F060F8074610B104F1004442
:1041F00001270FF2BC09D9E9008935494FF0000BBE
:1042000000205FFA8BF39E4206D942464B460DF0E2
:10421000CFFA0BF1010BF4E702460B46504621465C
:1042200000F0C4FD8946804601F0B8F83B460146DF
:1042300082460A222846FFF7AAFE0446002EA2D094
:10424000504600F03BFF0B4602464946404600F010
:10425000ABFD0F2E4FF02E0328BF0F268DF8003038
:104260000DF1010A3746013FFFB2FF2F15D00022A2
:10427000184B0DF09DFA8946804601F08FF8C0B2C8
:1042800000F130030AF8013B00F02AFF02460B461A
:104290004046494600F088FDE5E72B68721C5B68E4
:1042A000D2B26946284698476DE700BFAFF3008059
:1042B0009A9999999999B93F941E0100FFFFEF7F50
:1042C000981E0100FFFFEF419C1E0100FFFFEFC1A0
:1042D0000000E03F0000244070B5044608460D464B
:1042E00002F01CFD23680246294620465B68BDE8B3
:1042F0007040184710B50446FFF7E2FD204610BD98
:104300000448054A054900230361802303751030E2
:1043100001F04CBD4093FF1F1888FF1FF5420000BD
:1043200010B50446006801F059FF204610BD38B5AD
:1043300004460D460068013102F078FA10B1C4E974
:104340000005012038BD43688B4210B5044601D3F7
:10435000012010BDFFF7EBFF0028FAD0A368002B67
:10436000F6D122681370F3E7F8B504460F461546F8
:1043700032B9036803B11A700023A3602046F8BD68
:104380001146FFF7E0FF064638B9206810B101F08A
:1043900025FF266000236360EFE72068A5603946AB
:1043A00002F044FCEAE738B50023C0E900330446D4
:1043B000836003730D4639B1084602F0AFFC29460D
:1043C00002462046FFF7D0FF204638BD38B50546E7
:1043D00008460C4602F0A2FC214602462846BDE8EB
:1043E0003840FFF7C1BF13B504460023C4E90033CA
:1043F000A36023730A22084601A905F0C1FE2046E6
:1044000001A9FFF7E3FF204602B010BD10B5044636
:1044100086B00023C4E90033A3602373084601A9D2
:1044200001F09AFE204601A9FFF7D0FF204606B012
:1044300010BD10B5044686B00023C4E90033A36064
:104440002373084601A905F09BFE204601A9FFF74A
:10445000BDFF204606B010BD10B504468AB000234B
:10446000C4E90033A3602373084601A9FCF766FA88
:10447000204601A9FFF7AAFF20460AB010BD10B5DB
:1044800004468AB00023C4E90033A36023730846BE
:1044900001A9FCF72FFA204601A9FFF797FF204654
:1044A0000AB010BD38B50023C0E90033044683606C
:1044B000037308460D4602F031FC294602462046A9
:1044C000FFF752FF204638BD38B5054600680C4658
:1044D00068B16A688B689A4207D3096802F0A6FB44
:1044E000A368AB600023A36038BD01F077FE2368AA
:1044F0002B6063686B60A368AB600023C4E9003382
:10450000F1E710B50023C0E900330446836003736C
:10451000FFF7DAFF204610BD10B50023C0E90033D5
:10452000044683600373FFF7CFFF204610BD81422E
:1045300003D08A680968FFF717BF704710B50023DA
:104540000446C0E9003383600373FFF7F0FF2046A1
:1045500010BD884210B5044601D0FFF7B5FF2046D4
:1045600010BD884210B5044601D0FFF7ADFF2046CC
:1045700010BD10B5044619B1FFF728FF204610BD45
:104580008160FBE710B504468AB00023C4E900331C
:10459000A360237308466B46911CFCF7DFF90146C4
:1045A0002046FFF7E6FF20460AB010BD38B50446A6
:1045B00008460D4602F0B2FB294602462046FFF7A8
:1045C000D3FE204638BD07B500238DF80410012224
:1045D00001A98DF80530FFF7C7FE03B05DF804FBB5
:1045E00010B500230446C0E9003383600373FFF76E
:1045F000EAFF204610BD2DE9F843036885688B4229
:1046000004460E4617461ED85A1991421BD2A1EBFA
:1046100003094FF001089FB13D4429462046FFF7AA
:1046200092FE68B12168A0680844B8F1000F0DD06F
:104630003A46494401F0EAFD236800225A55A56034
:104640002046BDE8F8834FF00008E4E7314602F069
:10465000EDFAF4E78A680968FFF7CDBF38B505467B
:104660000C4639B1084602F059FB2146024628465D
:10467000FFF7C1FF284638BD13B500238DF804109D
:10468000012201A904468DF80530FFF7B4FF20464A
:1046900002B010BD1FB504460A22084601A9FCF766
:1046A0004DF901A802F03AFB01A902462046FFF7A6
:1046B000A2FF204604B010BD1FB504460A220846DA
:1046C00001A9FCF717F901A802F028FB01A902468D
:1046D0002046FFF790FF204604B010BDFFF7DABF79
:1046E000FFF7EABF10B588B004466B4602220846C1
:1046F0000421FCF733F9684602F010FB69460246D4
:104700002046FFF778FF204608B010BD10B58A6834
:1047100009680446FFF76FFF204610BD38B505460F
:104720000C4639B1084602F0F9FA214602462846FD
:10473000FFF761FF284638BD38B5044608460D46E8
:1047400002F0ECFA294602462046FFF754FF2046C5
:1047500038BD10B50446FFF78FFF204610BD10B5D9
:104760000446FFF797FF204610BD10B50446FFF73B
:1047700091FF204610BD10B50446FFF79DFF20466F
:1047800010BD10B50446FFF785FF204610BD10B5DB
:104790000446FFF791FF204610BD10B50446FFF711
:1047A000A1FF204610BD10B519460446104600F082
:1047B0001FFE01462046FFF795FF204610BD02462A
:1047C00000680B46096858B141B9916851B1007849
:1047D0007047986838B109784842704702F014B9B8
:1047E0000029F6D10846704708B582688B689A425E
:1047F00005D1FFF7E4FFB0FA80F0400908BD0020C2
:10480000FCE7826808B53AB921B10878B0FA80F0BF
:10481000400900E0012008BD006809B90078F5E70B
:1048200002F0F2F8F2E708B5FFF7C9FFC00F08BDC4
:1048300008B5FFF7C4FF0028D4BF0020012008BD41
:1048400008B5FFF7BCFF0028CCBF0020012008BD41
:1048500008B5FFF7B4FFC043C00F08BD884270B56C
:1048600015D083688A6893420FD183B104680E68BB
:10487000013C14F8010F50B105F0DCFB054616F8B9
:10488000010B05F0D7FB8542F3D0002070BD01205D
:10489000FCE7134610B58A688468A41A9C420AD3C0
:1048A000006838B1096841B1184402F067FAB0FAFB
:1048B00080F0400910BD0020FCE70846FAE7826856
:1048C0008B689A4202D30022FFF7E3BF00207047B3
:1048D00008B58A68836893420BD3006840B10968C1
:1048E00049B19B1A184402F08FF8B0FA80F04009E1
:1048F00008BD0020FCE70846FAE783688B4284BFC6
:1049000003685A54704783688B4201D9006818B90C
:104910000248002303707047084470475893FF1FF4
:1049200083688B4203D9006810B1405C7047002057
:104930007047FFF7F5BF58B50E462AB121B184681C
:104940009C4202D800230B7058BDE41A013A01685A
:10495000944228BF144619442246304602F080FA99
:1049600000233355F0E78368934210B506D90468F5
:10497000A01801F0A1FF08B1001B10BD4FF0FF30DF
:10498000FBE70022FFF7EFBF8368934210B507D91A
:1049900004680968A01802F003FD08B1001B10BDEF
:1049A0004FF0FF30FBE70022FFF7EEBFF8B583685A
:1049B0009342054602D84FF0FF30F8BD0368541CFF
:1049C00000221F5D1A550668304602F0AFFA3755CF
:1049D0000028F0D02B68C01AEFE78268013AFFF791
:1049E000E5BF2DE9F04115468A680E46CAB18368D5
:1049F000BBB19A4215D80768AB4298BF03F1FF35A7
:104A000038464FF0FF3407EB050840450BD83168B6
:104A100002F0C6FC38B1C31BAB4298BF1C46013044
:104A2000F3E74FF0FF342046BDE8F08182688B68E1
:104A3000D21AFFF7D6BF9A42F8B50E4682BF11468A
:104A40001A460B46002181600173B5689542C0E9A2
:104A5000001104460BD39D4228BF1D4633685F5D9D
:104A6000595531681144FFF784FD33685F5520467E
:104A7000F8BD10B58B680446FFF7DDFF204610BD7A
:104A8000036810B53BB1013B13F8014F1CB18C42D8
:104A9000FAD11A70F8E710BD2DE9F74FD0F808A049
:104AA00005460F461646BAF1000F46D0D1F808B0B9
:104AB000BBF1000F41D093680468A3EB0B08B8F179
:104AC000000F0DD12046396802F06AFC0446002828
:104AD00033D0B268316801F099FBB0680444F1E763
:104AE0000BDB0968D1462046019102F059FC40B326
:104AF000019900EB0B04C144F5E7A1463968204653
:104B000002F04EFC8246A0B1A0EB040B21465A46AF
:104B10004846D94401F07AFB4846B268316801F052
:104B200075FBB368BC689944AB6843445444AB60BC
:104B3000E4E72146484602F079F8284603B0BDE88C
:104B4000F08FCA45F9D06B684B4523D3AC684FF062
:104B50000009621E002AF0DB39462846FFF741FFB4
:104B6000041EEADBBB682968AA6823441944D21AE8
:104B700001EB080001F0DAFBAB682A684344AB6044
:104B800002F803902868B2683168204401F03EFBC7
:104B9000621EDFE749462846FFF7C9FB0028D5D14A
:104BA000CBE783688B4281BF0368816000225A543F
:104BB000704738B504460846A3688B4211D982B1C4
:104BC00011448B4238BF1A1A2568991A1318A1602C
:104BD0000A1AE918284401F0A9FB2268A3680021F9
:104BE000D154204638BD38B5046805463CB1013C77
:104BF00014F8010F18B105F01DFA2070F8E72846E7
:104C000038BD38B5046805463CB1013C14F8010FC5
:104C100018B105F027FA2070F8E7284638BD2DE9CD
:104C2000F0410668054606B38468F4B1B0464746CD
:104C300018F8010B01F052FA0028F8D1013C344475
:104C4000207801F04BFA18B1A74201D8013CF7E7F0
:104C5000621CD21BBE42AA6003D23946304601F024
:104C6000D5FA2A68AB680021D1542846BDE8F08106
:104C7000006808B101F0A8B87047006810B10021C1
:104C800004F0DAB80020704708B501210D20FCF7C8
:104C9000E5F8074C2025C4F884504FF4FA70FCF76F
:104CA00099FAC4F888504FF4FA70FCF793FAF2E7D7
:104CB00000F00F407047FFFF2DE9F8431B4C2378AD
:104CC000002B31D01A4D2A7872BB0122D9072A70E5
:104CD0000BD5FEF765FC08B1FFF7ECFF154B1B7811
:104CE0001BB1237823F00103237023789A0714D58E
:104CF000DFF84480DFF84490002698F80020F3B2F3
:104D00009A420AD959F823703B6838461B6998477C
:104D100008B13B6998470136EFE700232B702378F1
:104D20005B0701D500F00CF8BDE8F883F989FF1F97
:104D30005993FF1FF889FF1F3093FF1F3493FF1F04
:104D4000114938B50B684BB1EFF3058333B9EFF375
:104D5000108272B6086810B902B962B638BD0B4C41
:104D60002578002DF8D10123237043690B6043B1EE
:104D70009D6102B962B60025836845779847257022
:104D8000ECE703490B60F4E71493FF1F2F93FF1F19
:104D90001893FF1F00009FE51EFF2FE10000C07F5A
:104DA000021121E2000000EA023123E230402DE945
:104DB0008140A0E18350A0E1050034E10200300110
:104DC00000C0941102C09511C4CAF011C5CAF011F7
:104DD0008C00000AA44AA0E1A55A74E0005065B214
:104DE000060000DA054084E0022020E0033021E0E4
:104DF000000022E0011023E0022020E0033021E047
:104E0000360055E33040BD881EFF2F81020111E3BB
:104E10000116A0E101C6A0E321168CE10100000A01
:104E2000000070E20010E1E2020113E30336A0E1AA
:104E300023368CE10100000A002072E20030E3E238
:104E4000050034E16900000A014044E220E075E217
:104E5000050000BA12CEA0E1320590E00010A1E2F8
:104E6000130E90E05315B1E0060000EA205045E231
:104E700020E08EE2010052E313CEA0E102C08C23B9
:104E8000530590E0C31FB1E0025101E20200005A55
:104E900000C07CE20000F0E20010E1E2010651E314
:104EA0000F00003A020651E30600003AA110B0E1FB
:104EB0006000B0E16CC0A0E1014084E2842AA0E17E
:104EC000010572E36B00002A02015CE3A0C0B0019F
:104ED0000000B0E2041AA1E0051081E13040BDE815
:104EE0001EFF2FE18CC0B0E10000B0E00110A1E096
:104EF000014054E201065123F2FFFF2A000031E392
:104F00001430A0133430A0030010A0010000A0034F
:104F10000120A0E1010852E32228A0211030432201
:104F2000010C52E32224A02108304322100052E356
:104F30002222A02104304322040052E30230432203
:104F4000A2304330A23143E0202053E2070000AA00
:104F50000C2092E2040000DA14C082E20C2062E22B
:104F6000110CA0E13112A0E1040000EA142082E259
:104F700020C062D21112A0E1301C81D11002A0D158
:104F8000034054E0041A81A0051081A13040BDA85F
:104F90001EFF2FA10440E0E11F4054E20F0000AAD1
:104FA0000C4094E2060000CA144084E2202064E22F
:104FB0003004A0E1110280E1311485E13040BDE808
:104FC0001EFF2FE10C4064E2202064E23002A0E1E9
:104FD000110480E10510A0E13040BDE81EFF2FE183
:104FE0003104A0E10510A0E13040BDE81EFF2FE133
:104FF000000034E3013623E201162102014084025D
:10500000015045128FFFFFEAC4CAF0E1C5CAF01192
:105010001D00000A050034E1020030010400000A0E
:1050200000C094E10310A0010200A0013040BDE8DF
:105030001EFF2FE1030031E10010A0130000A013B8
:105040003040BD181EFF2F11A4CAB0E10400001AA1
:105050008000B0E10110B1E0021181233040BDE8D1
:105060001EFF2FE1014594E2011681323040BD3828
:105070001EFF2F31025101E27F1485E30F1681E3F9
:105080000000A0E33040BDE81EFF2FE1C4CAF0E1FC
:105090000310A0110200A011C5CAF0010130A01137
:1050A0000020A011014690E1035692010300310156
:1050B000021781133040BDE81EFF2FE1000030E3EE
:1050C0000010A0031EFF2F0130402DE9014BA0E38B
:1050D000324084E20050A0E30010A0E386FFFFEA24
:1050E000000030E30010A0031EFF2F0130402DE927
:1050F000014BA0E3324084E2025110E20000604222
:105100000010A0E37CFFFFEA8020B0E1C211A0E123
:105110006110A0E1020EA0E1FF341212FF0433136C
:105120000E1321121EFF2F11FF24D2E31EFF2F01A9
:10513000FF0433E3021781031EFF2F0130402DE9E6
:105140000E4DA0E3025101E20211C1E36AFFFFEA42
:10515000012090E11EFF2F0130402DE90050A0E317
:10516000060000EA012090E11EFF2F0130402DE9EA
:10517000025111E20100005A000070E20010E1E269
:10518000014BA0E3324084E221CBB0E142FFFF0AB1
:105190000320A0E3ACC1B0E103208212ACC1B0E1B6
:1051A00003208212AC2182E0203062E210C3A0E131
:1051B0003002A0E1110380E13112A0E1024084E05D
:1051C00035FFFFEA00C0E0E3020000EA01C0A0E30F
:1051D000000000EA01C0A0E304C02DE581C0A0E109
:1051E000CCCAF0E183C0A0E1CCCAF0110E00000AE5
:1051F00004D08DE281C090E183C09201030031119F
:10520000020030010000A0031EFF2F01000070E328
:10521000030031E10300515102005001C30FA021EE
:10522000C30FE031010080E31EFF2FE181C0A0E148
:10523000CCCAF0E10100001A01C690E10400001A96
:1052400083C0A0E1CCCAF0E1E8FFFF1A03C692E1F7
:10525000E6FFFF0A04009DE41EFF2FE100C0A0E16D
:105260000200A0E10C20A0E101C0A0E10310A0E138
:105270000C30A0E1FFFFFFEA01402DE9D4FFFFEB76
:10528000000050E3000070430140BDE81EFF2FE125
:1052900008E02DE5F7FFFFEB0100A0030000A013DD
:1052A00008E09DE41EFF2FE108E02DE5F1FFFFEB94
:1052B0000100A0330000A02308E09DE41EFF2FE1C1
:1052C00008E02DE5EBFFFFEB0100A0930000A083B9
:1052D00008E09DE41EFF2FE108E02DE5DEFFFFEB77
:1052E0000100A0930000A08308E09DE41EFF2FE1D1
:1052F00008E02DE5D8FFFFEB0100A0330000A0235C
:1053000008E09DE41EFF2FE181C0A0E1CCCAF0E1DE
:105310000100001A01C690E10600001A83C0A0E156
:10532000CCCAF0E10100001A03C692E10100001AA4
:105330000000A0E31EFF2FE10100A0E31EFF2FE10C
:105340008120A0E1022692E20C00002A0900005A06
:105350003E3EE0E3C22A53E00A00009A8135A0E114
:10536000023183E3A03A83E1020111E33302A0E1B9
:10537000000060121EFF2FE10000A0E31EFF2FE1DE
:10538000010690E10200001A020111E20201E003AD
:105390001EFF2FE10000A0E31EFF2FE18120B0E1FE
:1053A0000A00002A022692E20A00002A0700005A98
:1053B0003E3EE0E3C22A53E00800004A8135A0E106
:1053C000023183E3A03A83E13302A0E11EFF2FE123
:1053D0000000A0E31EFF2FE1010690E10100001A8A
:1053E0000000E0E31EFF2FE10000A0E31EFF2FE11D
:1053F0008120A0E1073252E202C653227FC57C22FF
:105400000600009A02C101E28021A0E1A00E8CE119
:10541000020152E30301A0E00100C0031EFF2FE1DF
:10542000010111E30F00001A2E2693E2020101B2DE
:105430001EFF2FB1011681E3A22AA0E1182062E22B
:1054400020C062E2103CB0E13002A0E10100801314
:105450008135A0E1A335A0E1130C80E13332A0E156
:105460008330A0E1E6FFFFEAC23AF0E10300001A50
:10547000013690E17F04A013030580131EFF2F1156
:10548000020101E27F0480E3020580E31EFF2FE1B9
:10549000020120E2000000EA021121E28020B0E1D6
:1054A0008130B0110300321142CCF01143CCF01125
:1054B0004700000A222CA0E1233C72E0032082C0B6
:1054C000011020C0000021C0011020C0003063B2D4
:1054D000190053E31EFF2F81020110E3020580E350
:1054E000FF04C0E300006012020111E3021581E332
:1054F000FF14C1E300106112030032E12E00000A24
:10550000012042E2510390E0203063E21113A0E158
:10551000023100E20100005A001071E20000E0E2F6
:10552000020550E30B00003A010450E30400003A86
:10553000A000B0E16110A0E1012082E2FE0052E390
:105540003800002A020151E3820BA0E00100C003F1
:10555000030080E11EFF2FE18110B0E10000A0E018
:10556000012052E202055023F5FFFF2A20C6B0E1D8
:105570000006A0010C204202FF0810E30004A00175
:10558000082042020F0610E30002A001042042029C
:10559000030510E30001A00102204202020550E3CE
:1055A0008000A0310020D2E2820B80A0002062B2F5
:1055B000030080A1300283B11EFF2FE1000032E31F
:1055C000021521E20205200201208202013043126D
:1055D000CAFFFFEA8130A0E142CCF0E143CCF011F8
:1055E0001300000A030032E10200000A000032E367
:1055F0000100A0011EFF2FE1010030E10000A01317
:105600001EFF2F11FF0412E30200001A8000B0E118
:10561000020180231EFF2FE1022492E20205803264
:105620001EFF2F31023100E27F0483E3020580E395
:105630001EFF2FE1422CF0E10100A011433CF001DC
:105640000010A0118024B0E18134B00101003001CC
:10565000010580131EFF2FE10030A0E3010000EAE6
:10566000023110E20000604200C0B0E11EFF2F01D5
:105670004B3483E30010A0E10000A0E30F0000EA38
:10568000012090E11EFF2F010030A0E3050000EA99
:10569000012090E11EFF2F01023111E20100005AAA
:1056A000000070E20010E1E201C0B0E100C0A00122
:1056B0000010A0010000A0035B3483E30132430229
:1056C000023543E21720A0E301085CE32CC8A021C7
:1056D00010204222010C5CE32CC4A02108204222AD
:1056E00010005CE32CC2A0210420422204005CE3F1
:1056F00002204222AC204230AC2152E0823B43E007
:10570000060000BA113283E010C2A0E1202062E25C
:1057100002015CE33002A3E00100C0031EFF2FE1A1
:10572000202082E211C2A0E1202062E28C0090E100
:105730003102A3E0AC0FC0011EFF2FE1FFC0A0E3C8
:10574000A02B1CE0A13B1C100C0032110C003311EB
:105750003E00000A032082E001C020E08004B0E1A6
:105760008114B0111000000A0233A0E3A00283E10B
:10577000A11283E1903181E002010CE2020551E3C4
:105780008110A031A31F81318330A031010080E15D
:105790007F20C2E2FD0052E30F00008A020153E3C2
:1057A000820BA0E00100C0031EFF2FE1000030E3E8
:1057B00002C10CE28114A001A0048CE1A10480E1EB
:1057C0007F2052E2FF3072C2820B80C11EFF2FC1C8
:1057D000020580E30030A0E3012052E2350000CA58
:1057E000190072E3020100D21EFF2FD1002062E2F5
:1057F0008010B0E13112A0E1202062E210C2A0E1ED
:105800006100B0E10000A0E28C3093E1AC0FC00178
:105810001EFF2FE1000032E302C100E28000A00180
:105820000205100301204202FBFFFF0A0C0080E189
:10583000000033E302C101E28110A001020511035F
:1058400001304302FBFFFF0A0C1081E1C0FFFFEAB9
:10585000A13B0CE00C0032E10C0033110500000A02
:1058600002C1D0E302C1D113E9FFFF1A010020E019
:10587000020100E21EFF2FE1000030E302013013BD
:105880000100A00100003113020131130D00000AD4
:105890000C0032E10100001A8024B0E10900001A76
:1058A0000C0033E10200001A8134B0E10100A011C4
:1058B0000400001A010020E0020100E27F0480E3FE
:1058C000020580E31EFF2FE17F0480E3030580E3F0
:1058D0001EFF2FE1FFC0A0E3A02B1CE0A13B1C108A
:1058E0000C0032110C0033113A00000A032042E090
:1058F00001C020E08114B0E18004A0E11C00000A96
:105900000132A0E3211283E1203283E102010CE2A3
:10591000010053E18330A0317D20A2E202C5A0E363
:10592000010053E1013043200C008021A10053E12C
:10593000A1304320AC008021210153E121314320DB
:105940002C018021A10153E1A1314320AC01802130
:105950000332B0E12CC2B011F0FFFF1AFD0052E398
:105960009DFFFF8A010053E1820BA0E00100C0030C
:105970001EFF2FE102C10CE2A0048CE17F2092E225
:10598000FF3072C2820B80C11EFF2FC1020580E36F
:105990000030A0E3012052E28FFFFFEA000032E373
:1059A00002C100E28000A0010205100301204202B2
:1059B000FBFFFF0A0C0080E1000033E302C101E2BB
:1059C0008110A0010205110301304302FBFFFF0A11
:1059D0000C1081E1C4FFFFEAA13B0CE00C0032E1B6
:1059E0000500001A8024B0E1B6FFFF1A0C0033E175
:1059F000AFFFFF1A0100A0E1B2FFFFEA0C0033E1A4
:105A00000300001A8134B0E197FFFF0A0100A0E112
:105A1000ACFFFFEA02C1D0E302C1D113DEFFFF1ADF
:105A20000221D0E3A2FFFF1A0231D1E38EFFFF1A59
:105A3000A4FFFFEA00C0E0E3020000EA01C0A0E327
:105A4000000000EA01C0A0E304C02DE58020A0E131
:105A50008130A0E142CCF0E143CCF0110700000A14
:105A600004D08DE2A3C092E1010030110300525036
:105A7000C10FA081C10FE031010080131EFF2FE193
:105A800042CCF0E10100001A80C4B0E10300001A2A
:105A900043CCF0E1F1FFFF1A81C4B0E1EFFFFF0A50
:105AA00004009DE41EFF2FE100C0A0E10100A0E181
:105AB0000C10A0E1FFFFFFEA0F402DE9E0FFFFEB34
:105AC000000050E3000070430F40BDE81EFF2FE1CF
:105AD00008E02DE5F7FFFFEB0100A0030000A01395
:105AE00008E09DE41EFF2FE108E02DE5F1FFFFEB4C
:105AF0000100A0330000A02308E09DE41EFF2FE179
:105B000008E02DE5EBFFFFEB0100A0930000A08370
:105B100008E09DE41EFF2FE108E02DE5E1FFFFEB2B
:105B20000100A0930000A08308E09DE41EFF2FE188
:105B300008E02DE5DBFFFFEB0100A0330000A02310
:105B400008E09DE41EFF2FE18020A0E18130A0E16C
:105B500042CCF0E10100001A80C4B0E10500001A57
:105B600043CCF0E10100001A81C4B0E10100001A49
:105B70000000A0E31EFF2FE10100A0E31EFF2FE1C4
:105B80008020B0E10800002A7F0452E30600003ABA
:105B90009E30A0E3222C53E00500004A0034A0E12F
:105BA000023183E33302A0E11EFF2FE10000A0E3F6
:105BB0001EFF2FE1610072E30100001A8024B0E1B2
:105BC0000100001A0000E0E31EFF2FE10000A0E347
:105BD0001EFF2FE1000053E3000052030400001AEF
:105BE000000051E3000050030010E0130000E01338
:105BF000500000EA08D04DE200602DE9030000EB00
:105C000004E09DE508D08DE20C00BDE81EFF2FE109
:105C1000F0472DE90360A0E1020050E10630D1E039
:105C20000040A0E10000A0330150A0E120709DE5FC
:105C30000010A0313B00003A0610A0E10200A0E1F4
:105C40000280A0E13C0000EB0510A0E10090A0E183
:105C50000400A0E1380000EB00C049E0163CA0E1E0
:105C600020604CE2183683E120E06CE2182CA0E1C1
:105C7000383E83E1020054E10310D5E00000A03378
:105C80000010A0310500003A0100A0E3024054E0FA
:105C90001016A0E1301E81E10350C5E0100CA0E118
:105CA00000005CE31F00000AA220A0E1832F82E134
:105CB0000C80A0E1A330A0E1070000EA024054E01C
:105CC0000350C5E0044094E00550A5E0014094E293
:105CD0000050A5E2018058E20600000A020054E1EB
:105CE0000390D5E0F4FFFF2A044094E00550A5E0BE
:105CF000018058E2F8FFFF1A040090E0344CA0E164
:105D0000154E84E1354684E10510A1E0355CA0E143
:105D1000153CA0E1143683E114CCA0E1343E83E1CC
:105D20000C0050E00310C1E0000057E3300087187A
:105D3000F047BDE81EFF2FE11EFF2FE110402DE9C7
:105D4000000051E30200001A050000EB200080E291
:105D5000010000EA0100A0E1010000EB1040BDE8F5
:105D60001EFF2FE11C10A0E3010850E32008A02132
:105D700010104122010C50E32004A0210810412200
:105D8000100050E32002A0210410412208208FE2DD
:105D90000000D2E7010080E01EFF2FE104030202B1
:105DA0000101010100000000000000000130A0E13D
:105DB00010402DE90010A0E10300A0E10D0000EB70
:105DC0001040BDE81EFF2FE110402DE90A20A0E39E
:105DD0000010A0E3FE0C00EB1040BDE81EFF2FE119
:105DE00010402DE90A30A0E30020A0E3CF0C00EB27
:105DF0001040BDE81EFF2FE101C0A0E110402DE9D9
:105E000000E0A0E10230A0E10E10A0E10200A0E35A
:105E10000C20A0E11F1100EB1040BDE81EFF2FE198
:105E200004E02DE50CD04DE210C09DE500C08DE5ED
:105E300000C0A0E304C08DE5A81100EB0CD08DE2FA
:105E400004E09DE41EFF2FE170402DE908D04DE2F3
:105E50000250A0E10360A0E10140A0E1A9FCFFEB3A
:105E600000C0A0E30530A0E10420A0E100608DE5C2
:105E700004C08DE5991100EB08D08DE27040BDE8BB
:105E80001EFF2FE1F0412DE90340A0E110D04DE2CB
:105E90000250A0E10030A0E30020A0E30170A0E1E7
:105EA0000060A0E1FFFCFFEB000050E30410A01134
:105EB0002D30A0130410A00100E0A0E367C0A0E310
:105EC00048809FE50130C11444009FE50150451210
:105ED00008808FE0000098E704108DE500508DE504
:105EE0000620A0E1000090E50730A0E10CE08DE580
:105EF00008C08DE5051200EB000050E30400A0117E
:105F00000000A00310D08DE2F041BDE81EFF2FE19C
:105F1000DC30FF1F34000000F0412DE910D04DE2CD
:105F20000240A0E10150A0E10070A0E175FCFFEB90
:105F30000130A0E10020A0E10010A0E30700A0E1F3
:105F40000260A0E10370A0E1E6FEFFEB000050E379
:105F50000410A0112D30A0130410A00100E0A0E354
:105F600067C0A0E348809FE50130C11444009FE56D
:105F70000150451208808FE0000098E704108DE57D
:105F800000508DE50620A0E1000090E50730A0E17B
:105F90000CE08DE508C08DE5DC1100EB000050E35E
:105FA0000400A0110000A00310D08DE2F041BDE874
:105FB0001EFF2FE13830FF1F3400000004E02DE504
:105FC0000CD04DE210C09DE500C08DE500C0A0E3FF
:105FD00004C08DE5881100EB0CD08DE204E09DE457
:105FE0001EFF2FE170402DE908D04DE20250A0E1E4
:105FF0000360A0E10140A0E142FCFFEB00C0A0E390
:106000000530A0E10420A0E100608DE504C08DE52D
:10601000791100EB08D08DE27040BDE81EFF2FE142
:1060200010309FE510209FE503308FE0023093E7AA
:10603000000093E51EFF2FE1842FFF1F34000000B6
:10604000F0412DE97C709FE57C209FE57C309FE549
:1060500007708FE0026097E7035097E7056046E01E
:106060004661B0E10600000A0040A0E3043095E478
:10607000014084E20FE0A0E113FF2FE1040056E1AC
:10608000F9FFFF1ACA3000EB44209FE544309FE53A
:10609000026097E7035097E7056046E04661B0E18C
:1060A0000600000A0040A0E3043095E4014084E2C9
:1060B0000FE0A0E113FF2FE1040056E1F9FFFF1A02
:1060C000F041BDE81EFF2FE15C2FFF1F38000000EC
:1060D00050000000300000004800000018309FE52C
:1060E00018209FE503308FE0023093E7003083E013
:1060F0000100D3E5080000E21EFF2FE1C82EFF1FBC
:1061000044000000023042E2220053E30030A0834A
:1061100010402DE90300A0810140A0E10030C185BD
:106120000A00008AA03FA0E10A0052E30030A01359
:1061300001300302000053E32D30A0130410A0012E
:106140000130C11400006012D10F00EB0400A0E187
:106150001040BDE81EFF2FE1023042E2220053E36F
:106160000030A08310402DE90300A0810140A0E190
:106170000030C1850A00008AA03FA0E10A0052E376
:106180000030A01301300302000053E32D30A013B0
:106190000410A0010130C11400006012BC0F00EB1C
:1061A0000400A0E11040BDE81EFF2FE110402DE9E2
:1061B0001C309FE51C209FE503308FE0023093E701
:1061C0000010A0E1000093E5420100EB1040BDE8A3
:1061D0001EFF2FE1F42DFF1F3400000010402DE9B9
:1061E0001C309FE51C209FE503308FE0023093E7D1
:1061F0000010A0E1000093E5E80000EB1040BDE8CE
:106200001EFF2FE1C42DFF1F340000000F0052E3DA
:106210003600009A013080E1030013E33F00001ACA
:1062200010C042E2F0402DE9204081E20FE0CCE3D3
:10623000103081E2106080E20E4084E02C52A0E138
:106240000CE013E508C013E5107013E50CE006E55B
:10625000103083E214E013E5040053E1005006E936
:10626000107006E5106086E2F4FFFF1A01C085E2B7
:106270000C0012E30F3002E20C1281E00320A001B7
:106280000CC280E00D00000A0140A0E1043043E2AE
:106290000360C3E323E1A0E106608CE004304CE23C
:1062A000045094E40450A3E5060053E1FBFFFF1AF9
:1062B00001308EE2032002E203C18CE0031181E091
:1062C000000052E3013042E20130831201204C12FF
:1062D000033081100300000A01C0D1E4030051E142
:1062E00001C0E2E5FBFFFF1AF040BDE81EFF2FE111
:1062F000000052E300C0A0E1013042E21EFF2F0186
:10630000013083E201204CE2033081E001C0D1E49E
:10631000030051E101C0E2E5FBFFFF1A1EFF2FE180
:1063200000C0A0E1013042E2F4FFFFEA010050E1C9
:106330000A00009A023081E0000053E10700009A51
:10634000000052E3022080E01EFF2F0101C073E530
:10635000030051E101C062E5FBFFFF1A1EFF2FE1C0
:106360000F0052E30B00008A000052E300C0A0E1DE
:10637000012042E21EFF2F01012082E201C04CE217
:10638000023081E00120D1E4030051E10120ECE57D
:10639000FBFFFF1A1EFF2FE1013080E1030013E332
:1063A0003400001A10C042E270402DE90F30CCE3F7
:1063B00020E081E2104081E2105080E203E08EE0B4
:1063C0002CC2A0E1103014E5103005E50C3014E5C6
:1063D0000C3005E5083014E5083005E5104084E28E
:1063E000143014E50E0054E1043005E5105085E248
:1063F000F3FFFF1A01C08CE20C0012E30F3002E23F
:106400000C1281E00320A0010CC280E00D00000A04
:106410000140A0E1043043E20360C3E323E1A0E1D3
:1064200006608CE004304CE2045094E40450A3E590
:10643000060053E1FBFFFF1A01308EE2032002E267
:1064400003C18CE0031181E0000052E3012042E22D
:106450000120821201C04C12023081100300000A98
:106460000120D1E4030051E10120ECE5FBFFFF1A1C
:106470007040BDE81EFF2FE100C0A0E1012042E214
:10648000BCFFFFEA030010E34000000A000052E3F3
:10649000012042E21EFF2F010030A0E1FFC001E217
:1064A000020000EA012042E2010072E31EFF2F0118
:1064B00001C0C3E4030013E3F9FFFF1A030052E332
:1064C0002800009A30402DE9FFE001E20EE48EE161
:1064D0000F0052E30EE88EE12E00009A10C042E257
:1064E0000F40CCE3205083E2045085E02C42A0E131
:1064F00010C083E210E00CE50CE00CE508E00CE5D0
:1065000004E00CE510C08CE205005CE1F8FFFF1A26
:1065100001C084E20C0012E30CC283E00F2002E20F
:106520001800000A043042E20330C3E3043083E27F
:1065300003308CE004E08CE40C0053E1FCFFFF1A14
:10654000032002E2000052E30400000AFF1001E20F
:10655000022083E00110C3E4030052E1FCFFFF1AB4
:106560003040BDE81EFF2FE1000052E31EFF2F0167
:10657000FF1001E2022083E00110C3E4030052E1B6
:10658000FCFFFF1A1EFF2FE10C30A0E1ECFFFFEA39
:106590000030A0E1C8FFFFEA03C0A0E1E0FFFFEA8E
:1065A00070402DE924619FE5000051E306608FE013
:1065B0002400000A043011E5044041E2000053E3E6
:1065C000034084B00050A0E1BB1600EB00319FE512
:1065D000032096E7003092E5000053E33100000A03
:1065E000040053E11900008A0310A0E1043093E590
:1065F000002053E20120A013040053E10020A083F7
:10660000000052E3F7FFFF1A002091E5020081E04D
:10661000040050E11A00000A2700008A002094E5D7
:10662000020084E0000053E100009305043093056C
:10663000022080000C00840804308415044081E5A9
:106640000500A0E19D1600EB7040BDE81EFF2FE1A4
:10665000001094E5010084E0000053E10000930580
:1066600004309305011080000A0084080500A0E1B1
:1066700004308415004082E5901600EB7040BDE8C0
:106680001EFF2FE1000094E5002082E00100A0E160
:10669000022080E6000053E10900930802208000F8
:1066A0000C008108E5FFFFEA0500A0E1043084E565
:1066B000004082E5811600EBE2FFFFEA0C30A0E328
:1066C0000500A0E1003085E57C1600EBDDFFFFEA68
:1066D000002AFF1F4C00000070402DE9035081E2AA
:1066E0000350C5E3085085E20C0055E30C50A0337D
:1066F000050051E10010A0930110A083A53F91E196
:106700000060A0E10C30A0130000A013003086153B
:106710002000001A681600EB00319FE503209FE778
:10672000000052E31D00000A0240A0E1040000EA5C
:10673000043094E5000053E30420A0E11700000AB0
:106740000340A0E1003094E5053053E0F7FFFF4A35
:106750000B0053E3003084850350A4870500008AB2
:10676000043094E5020054E104308215B0209F0506
:1067700002208F00003082050600A0E14F1600EBDA
:106780000B0084E2043084E20700C0E3032050E001
:1067900000304310023084177040BDE81EFF2FE127
:1067A00080409FE504408FE0041094E5000051E331
:1067B0001600000A0510A0E10600A0E1280000EB89
:1067C000010070E30010A0E10A00000A034080E22B
:1067D0000340C4E3040050E10400000A0600A0E105
:1067E000011044E01E0000EB010070E30100000A0C
:1067F000005084E5DFFFFFEA0C30A0E30600A0E1D3
:10680000003086E52D1600EB0000A0E3E1FFFFEA73
:106810000600A0E1120000EB040084E5E4FFFFEABB
:10682000382CFF1FE42BFF1FB02BFF1F00C0A0E17F
:1068300010402DE920309FE50120A0E11C109FE5CC
:1068400003308FE0013093E70C10A0E1000093E5E6
:10685000211A00EB1040BDE81EFF2FE16C27FF1F3F
:106860003400000070402DE900E0A0E33C309FE5DB
:106870003C209FE503308FE0025093E70040A0E109
:106880000100A0E100E085E5F1E7FFFB010070E316
:106890000100000A7040BDE81EFF2FE1003095E5C1
:1068A000000053E3003084157040BDE81EFF2FE167
:1068B0003827FF1F04000000FF1011E20030A0E1A4
:1068C000032000E22D00000A000052E32500001A18
:1068D00070402DE900C090E5015481E11C419FE525
:1068E000055885E10C2025E0043082E00230C3E148
:1068F00004208CE008619FE50C20C2E1023083E1B6
:10690000060013E10800001A04C0B0E505E02CE021
:1069100004308CE004208EE00C30C3E10E20C2E194
:10692000023083E1060013E1F6FFFF0A0030D0E5F4
:10693000000053E30300001A2D0000EA0130F0E5E7
:10694000000053E32A00000A030051E1FAFFFF1A96
:10695000280000EA010052E11EFF2F01030013E3AB
:106960000300A0E1D9FFFF0A0300A0E10120D3E466
:10697000000052E3F6FFFF1A0200A0E11EFF2FE124
:10698000000052E30700000A0300A0E10020D0E568
:10699000000052E3013083E21EFF2F01030013E3E6
:1069A0000300A0E1F7FFFF1A002090E54CC09FE52F
:1069B0004C109FE50C3082E00230C3E1010013E18E
:1069C0000400001A0420B0E50C3082E00230C3E17C
:1069D000010013E1FAFFFF0A0030D0E5000053E3A5
:1069E0001EFF2F010130F0E5000053E3FCFFFF1A0A
:1069F0001EFF2FE10300A0E17040BDE81EFF2FE164
:106A0000FFFEFEFE8080808001C020E003001CE3CA
:106A10002100001A03C010E20300C0E30310C1E329
:106A2000042090E4043091040600000A03C02CE224
:106A3000FF34E0E38CC1A0E133CCA0E1043091E469
:106A40000C2082E10C3083E104402DE50140A0E3FD
:106A5000044484E1044884E104C042E0030052E1BC
:106A600002C0CC0184031C01042090040430910472
:106A7000F8FFFF0A020CA0E12224A0E1010050E38C
:106A8000030C50212334A001F9FFFF0AFF3003E279
:106A9000200C63E004409DE41EFF2FE1030010E39F
:106AA0000600000A0120D0E40130D1E4010052E3E5
:106AB00003005221F8FFFF0A030042E01EFF2FE10E
:106AC00030002DE90140A0E3044484E1044884E15E
:106AD000042090E4035001E20310C1E3043091E488
:106AE000020055E31700000A2D00008AFF54C2E39C
:106AF000230455E104C042E002C0CCE10700001AC3
:106B000084C31CE0043091040600001A025025E002
:106B1000030C55E10800001A042090E4F2FFFFEA9C
:106B20002334A0E1360000EAFFC4DCE33100001AA0
:106B30000030D1E5225CA0E1310000EA225CA0E156
:106B4000FF3003E22E0000EA0258A0E104C042E058
:106B50002558A0E102C0CCE1230855E10E00001A3F
:106B600084C31CE0043091040400001A025025E0A4
:106B7000030855E10600001A042090E4F1FFFFEA43
:106B80000CC8B0E11B00001AB030D1E12258A0E1DE
:106B90001B0000EA0338A0E12258A0E12338A0E15D
:106BA000170000EAFF5002E2230C55E104C042E066
:106BB00002C0CCE10700001A84C31CE00430910439
:106BC0000600001A025025E0030455E10600001AF1
:106BD000042090E4F2FFFFEA233CA0E1080000EA71
:106BE000FF0012E30300000A043091E42254A0E104
:106BF000FF34C3E3020000EA0000A0E33000BDE878
:106C00001EFF2FE1FF2005E2FF0003E2010050E339
:106C1000020050212554A0012334A001F8FFFF0AEF
:106C2000000042E03000BDE81EFF2FE1012020E01F
:106C300000C0A0E1030012E33200001A030011E3D8
:106C40002100001A04502DE50150A0E3055485E110
:106C5000055885E104402DE5040011E3043091E47A
:106C60000500000A052043E00320D2E1850312E17C
:106C700004308C04043091040C00001A044091E4A8
:106C8000052043E00320D2E1850312E1052044E022
:106C90000600001A04308CE40420D2E1850312E1DE
:106CA0000430910404408C04F3FFFF0A0430A0E197
:106CB0000130CCE4FF0013E36334A0E1FBFFFF1AD3
:106CC00004409DE404509DE41EFF2FE1010011E308
:106CD0000300000A0120D1E40120CCE4000052E3CB
:106CE0001EFF2F01020011E3D5FFFF0AB220D1E001
:106CF000FF0012E3B220CC100020CC05FF0C1213D1
:106D0000CFFFFF1A1EFF2FE10120D1E40120CCE4C8
:106D1000000052E3FBFFFF1A1EFF2FE10310C0E348
:106D2000030010E2000060E2043091E404C080E25D
:106D30008CC1A0E10020E0E3323C831101C0A0E35C
:106D40000CC48CE10CC88CE10C2043E00320C2E1B0
:106D50008C2312E00430910404008002F9FFFF0A42
:106D6000FF0013E301008012FF0C131301008012D7
:106D7000FF081313010080121EFF2FE1000052E3F1
:106D80002F00000AF0402DE901E080E103001EE33E
:106D900000C0A0E10130A0E11500001A030052E399
:106DA0001300009AAC509FE5AC609FE5070000EA35
:106DB000042052E21F00000A060014E11D00001A20
:106DC000030052E30C00A0E10310A0E10800009AC8
:106DD0000310A0E10C00A0E1007091E504E09CE448
:106DE00005408EE007005EE1043083E20E40C4E11E
:106DF000EEFFFF0A00C0D0E50040D1E50C0054E1F1
:106E00001100001A010052E3000054130900000AA7
:106E100000E0A0E101C0FEE50140F1E502304EE0F6
:106E200004005CE1013083E20700001A030050E136
:106E300000005C13F6FFFF1A0000A0E3F040BDE87D
:106E40001EFF2FE10200A0E11EFF2FE104004CE035
:106E5000F040BDE81EFF2FE1FFFEFEFE8080808037
:106E6000013080E1030052E3033003E200C0A0934D
:106E700001C0A083000053E300C0A01300005CE346
:106E800000C0A00170402DE91500001A01E041E2A8
:106E9000070000EA0C30A0E10110FEE5000051E31C
:106EA0000110C3E4014042E20500000A03C0A0E172
:106EB0000420A0E1000052E3F5FFFF1A7040BDE896
:106EC0001EFF2FE1000054E302208C10FAFFFF0A9E
:106ED0000110C3E4020053E1FCFFFF1A7040BDE85B
:106EE0001EFF2FE10130A0E100C0A0E130609FE56E
:106EF00030509FE50310A0E1044093E406E084E0F5
:106F000004E0CEE105001EE1DFFFFF1A042042E2AB
:106F1000030052E30310A0E104408CE4F4FFFF8A75
:106F2000D9FFFFEAFFFEFEFE8080808070402DE9E1
:106F3000004051E20030A0110050A0130200001ADE
:106F4000090000EA0050A0E1013080E20410A0E155
:106F50000300A0E157FEFFEB000050E3F8FFFF1A2B
:106F60000500A0E17040BDE81EFF2FE151FEFFEBE0
:106F70000050A0E10500A0E17040BDE81EFF2FE138
:106F8000F04F2DE9010053E341DE4DE20350A0E153
:106F900000B0A0E10170A0E10280A0E104D04DE2C8
:106FA000FA00009A0130A0E30010A0E303E0A0E1A2
:106FB0000090E0E30320A0E1050000EA0310A0E157
:106FC0000120A0E309E043E0013082E0030055E145
:106FD0000C00009A090088E00200D0E703C0D8E75F
:106FE00000005CE1F4FFFF3A6400000A01E0A0E366
:106FF0000E20A0E10190A0E10E1081E0013082E0BE
:10700000030055E1F2FFFF8A00E08DE501E0A0E317
:107010000000A0E300C0E0E30E10A0E10E30A0E10C
:10702000050000EA0300A0E10110A0E30CE043E04A
:10703000013080E0030055E10C00009A012088E057
:107040000340D8E70C20D2E7020054E1F4FFFF8AA6
:107050004F00000A01E0A0E30E10A0E100C0A0E193
:107060000E0080E0013080E0030055E1F2FFFF8A6E
:1070700001C08CE2019089E20C0059E100309DE5ED
:107080000E30A0910C90A09100308DE5012B8DE287
:107090000C308DE20C2082E20450A3E5020053E1A3
:1070A000FCFFFF1A000055E3014045E201204812B1
:1070B000040088100800000A0110F2E50230E0E147
:1070C00041CE8DE2053083E001118CE0033088E091
:1070D000000052E1003401E5F6FFFF1A00309DE5A3
:1070E0000920A0E10800A0E1031088E0C71300EB2D
:1070F00000A050E26200001A0A60A0E1013049E2FB
:107100000C308DE500309DE5033045E004308DE521
:1071100006E08BE00430DEE7412E8DE2033182E0B1
:10712000003413E5000053E31E00000A00209DE533
:1071300000005AE30200531104309D3500A0A0E383
:10714000036086E0053047E0060053E1EFFFFF2AC9
:1071500007008BE0021B85E3411800EB007087E01D
:10716000053047E0060053E1E8FFFF2A0000A0E3F6
:1071700041DE8DE204D08DE2F04FBDE81EFF2FE12D
:1071800002005EE10120A003012082120E108100A6
:107190008CFFFFEA01005EE10110A00301108112E3
:1071A0000E008000A1FFFFEA0A0059E10930A0218A
:1071B0000A30A031040053E10E00002A011043E21E
:1071C000062083E0011088E002208BE0020000EA44
:1071D000013083E2040053E10600002A0100D2E4FA
:1071E00001C0F1E500005CE1F8FFFF0A012069E25F
:1071F000066082E0D0FFFFEA0A0059E10C309DE50D
:107200006000009A062089E008908DE502208BE05E
:10721000091088E0020000EA0A0053E1013043E26D
:107220000D00000A01C071E5010072E500005CE19B
:10723000019083E2F7FFFF0A0930A0E108909DE585
:1072400001A08AE203005AE10800008A00309DE5AF
:1072500004A09DE5036086E0B9FFFFEA0A30A0E1E3
:1072600001A08AE203005AE108909DE5F6FFFF9A2B
:107270000E00A0E141DE8DE204D08DE2F04FBDE8CA
:107280001EFF2FE1093045E0090053E10930A0312C
:1072900000A0A0E3012049E200208DE5013083E257
:1072A000012069E204208DE508308DE5026B85E35D
:1072B0000AE08BE00430DEE7412E8DE2033182E00C
:1072C000003413E5000053E30B00000A03A08AE03A
:1072D000053047E003005AE1F4FFFF9A07008BE016
:1072E0000610A0E1DE1700EB007087E0053047E0F4
:1072F00003005AE1EDFFFF9A9BFFFFEA040059E10A
:107300001000002A00309DE50A2089E0031088E083
:1073100002208BE00930A0E1020000EA013083E2A4
:10732000040053E10700002A0100D2E401C0F1E5A6
:1073300000005CE1F8FFFF0A04209DE50AA082E05E
:1073400003A08AE0E1FFFFEA000059E3C7FFFF0A5C
:107350000A1089E001108BE0092088E0020000EAB1
:10736000013043E2080053E1C0FFFF0A0230A0E110
:10737000010071E501C072E500005CE1F7FFFF0A62
:1073800008309DE5D0FFFFEA0930A0E1ABFFFFEA3E
:107390000130A0E30090A0E300308DE53AFFFFEA62
:1073A000F0412DE90150A0E10010D1E5000051E3CA
:1073B0000040A0E140D04DE24100000A0120D5E5A7
:1073C000000052E35E00000A0230D5E5000053E3FE
:1073D0003F00000A03E0D5E500005EE37300000A09
:1073E0000400D5E5000050E35B00000A0500A0E1C1
:1073F00049FEFFEB0060A0E10400A0E1021C86E36F
:10740000971700EB000056E13E00008AFE0056E3AD
:107410007700008A060040E04020A0E3007084E08E
:10742000011086E20D00A0E115FCFFEB000056E321
:107430000B00000A012045E2FFC006E2060082E0E0
:107440000130F2E540108DE23F3003E2033081E08D
:10745000021045E001108CE0000052E1401043E5CD
:10746000F6FFFF1A014044E20630D4E740208DE2E7
:107470003F3003E2033082E0400053E5004084E007
:10748000040057E10300002A230000EA084084E0DA
:10749000040057E12000003A06C0D4E740308DE2F6
:1074A0003FC00CE20CC083E00400A0E10620A0E194
:1074B0000510A0E140805CE5D41200EB000050E331
:1074C000F1FFFF1A0400A0E140D08DE2F041BDE8D9
:1074D0001EFF2FE100C0D0E500005CE3012882E13F
:1074E0000800000A03388CE10400A0E101C0F4E5C3
:1074F000030052E100005C13F9FFFF1A030052E1A0
:1075000001404002EEFFFF0A0040A0E30400A0E1BA
:1075100040D08DE2F041BDE81EFF2FE10630D7E7F5
:10752000000053E3060087E0F6FFFF0A021BA0E31A
:107530004B1700EB007087E0040057E1C8FFFF2AFB
:10754000F0FFFFEADBFCFFEB0040A0E10400A0E15C
:1075500040D08DE2F041BDE81EFF2FE100C0D4E530
:1075600000005CE3E7FFFF0A022481E10010A0E1D4
:10757000033882E10E3C83E1632823E02224A0E16A
:10758000FF2CC2E3633422E001148CE10400A0E18B
:1075900001C0F4E500005CE303005111F9FFFF1A9C
:1075A000030051E103404002C5FFFF0AD5FFFFEA97
:1075B0000228A0E1012C82E10010D0E5000051E397
:1075C000033482E1CFFFFF0A0E2081E10400A0E135
:1075D0000110F4E502E4A0E1000051E303005E11B4
:1075E000F8FFFF1A0E0053E102404002B4FFFF0A09
:1075F000C4FFFFEA0010A0E10630A0E10520A0E1F1
:107600000400A0E140D08DE2F041BDE85BFEFFEA5E
:1076100000C0A0E3F04F2DE9B8AF9FE584D04DE264
:107620001C208DE570C08DE50340A0E1A83F9FE5DB
:107630000AA08FE003309AE7003093E50080A0E1D4
:107640000300A0E10160A0E120308DE5B2FDFFEB79
:107650000010A0E30020A0E10000A0E30630A0E1BC
:1076600010008DE514108DE56C608DE50390A0E1B0
:1076700001B0D3E42D005BE30BF18F902D0000EA05
:10768000840100EA2B0000EA2A0000EA290000EA4F
:10769000280000EA270000EA260000EA250000EAA8
:1076A000240000EA860100EA850100EA840100EA7C
:1076B000830100EA820100EA1E0000EA1D0000EAE0
:1076C0001C0000EA1B0000EA1A0000EA190000EAA8
:1076D000180000EA170000EA160000EA150000EAA8
:1076E000140000EA130000EA120000EA110000EAA8
:1076F000100000EA0F0000EA0E0000EA0D0000EAA8
:107700006F0100EA0B0000EA0A0000EA090000EA43
:10771000080000EA070000EA060000EA050000EAA7
:10772000040000EA030000EA020000EADC0200EACA
:10773000000000EAD10200EA0030A0E328308DE525
:1077400030005BE30030A01324308D155E01000A89
:1077500030304BE2090053E34403008A0070A0E399
:107760000900A0E10750A0E10740A0E1010080E28C
:107770006C008DE5080054E300B0D0E5077187C0C8
:10778000051185E0815083D0877083C030304BE293
:10779000090053E3014084E2F3FFFF9A20109DE5C6
:1077A00020208DE574FDFFEB000050E320209DE5D7
:1077B0009A01000A20B0CBE345005BE35001000AC8
:1077C0000030A0E330408DE520308DE534308DE58C
:1077D00030609DE5000054E30640A0010500A0E1F3
:1077E000100056E306B0A0B110B0A0A332F6FFEB34
:1077F0000020A0E10130A0E134C09DE520E09DE53E
:10780000090056E30EC04CE010208DE514308DE5E4
:107810002CC08DE5110000DA083E9FE503309AE7A1
:107820008B3183E0483043E20C0093E8DF2700EB24
:107830000020A0E10700A0E10260A0E10170A0E14A
:107840001DF6FFEB0020A0E10130A0E10600A0E161
:107850000710A0E154F5FFEB10008DE514108DE545
:1078600030309DE50F0053E37F0100CA2C309DE5C9
:10787000000053E3E302000A2C309DE5A80300DA80
:10788000160053E3DF0300DA30309DE52C209DE540
:10789000253063E2020053E130309DE5ED0300AA9C
:1078A0000BB043E02C309DE503B08BE00F001BE2F2
:1078B0000800000A6C1D9FE501109AE7801181E025
:1078C00010308DE20C0093E8030091E8B72700EB3D
:1078D00010008DE514108DE50F60DBE38902001ABE
:1078E0000030A0E324308DE530309DE50420A0E198
:1078F0000910A0E10800A0E100508DE55C1200EB4A
:10790000003050E24C308DE56503000A2C309DE5D7
:1079100020209DE534109DE5000053E3012042B096
:107920000020A0A30090A0E3C33FC3E134208DE575
:1079300020908DE548308DE54C409DE50800A0E1A4
:10794000041094E5DE1100EB00A050E2C701000A2C
:10795000102094E5022082E20221A0E10C1084E2D2
:107960000C008AE228FAFFEB10108DE2030091E888
:1079700001C0A0E138108DE578108DE204108DE58E
:1079800074108DE20020A0E144008DE50C30A0E1F0
:107990000800A0E100108DE5F71400EB000050E3B3
:1079A00070008DE5A801000A0110A0E30800A0E125
:1079B000B31200EB009050E2AC01000A74309DE578
:1079C000000053E334209DA548209DB5027083A09C
:1079D000036042B024209DE578409DE5023043E0FD
:1079E000043083E0F4BB9FE5013043E248609DA58D
:1079F00034709DB50B0053E1364064E2650100AA86
:107A000003B04BE01F005BE30130A0D30B4044E028
:107A100001B0A0C313BBA0D10030A0D3C02B9FC521
:107A2000033042C01B33A0C13C308DE524309DE5BE
:107A3000046086E0044087E0040057E1066083E0CC
:107A40000430A0A10730A0B1060053E10630A0A188
:107A5000000053E3034044C0036046C0037047C0C6
:107A600034309DE5000053E35E0100CA000054E39A
:107A70006E0100CA2C309DE5000053E3750100CA79
:107A8000000056E38F0100CA000057E3050000DA4A
:107A90000910A0E10720A0E10800A0E1771300EBA6
:107AA000009050E27101000A0A20A0E10800A0E164
:107AB00070109DE5DB1300EB003050E220308DE5C7
:107AC0006A01000A0050A0E320309DE50C2093E5F8
:107AD0000910A0E10C5083E530208DE5B91300EBCF
:107AE000050050E1CB0300BA14409DE56903000A8C
:107AF0000910A0E120009DE5F21400EB0020A0E3B6
:107B00000131A0E30060A0E10170A0E1EBF5FFEB23
:107B1000000050E32301000A30309DE5000053E3EC
:107B20007401000A0060A0E3B83A9FE53C508DE57F
:107B300040308DE5AC7A9FE5005B9FE5A83A9FE574
:107B400005B004E003005BE18501000A24309DE5F7
:107B5000003053E20130A0136A065BE30030A083DB
:107B6000000053E31B00000A3C509DE540409DE5AA
:107B70000500A0E10410A0E1702A9FE5703A9FE59E
:107B8000CEF5FFEB000050E31000000A0410A0E166
:107B90000500A0E100F6FFEB010050E30100A03377
:107BA00045F5FFEB30309DE5000053E33C008DE5EB
:107BB00040108DE5CC01000A3C208DE20C0092E8DB
:107BC00058208DE55C308DE558708DE2C00097E857
:107BD0006B3687E20B7043E044509DE538409DE5ED
:107BE0000500A0E10410A0E1111400EB0020A0E1C9
:107BF0000130A0E10600A0E10710A0E1EB2600EBB8
:107C00000520A0E10430A0E167F4FFEB0150A0E102
:107C100010008DE514108DE5203A9FE524209DE5A8
:107C2000053003E00B0053E1000052033402000A68
:107C30000800A0E170109DE5441100EB0A10A0E1DE
:107C40000800A0E1411100EB0910A0E10800A0E14B
:107C50003E1100EB0800A0E120109DE53B1100EB78
:107C600034FFFFEA0030A0E301C0A0E30350A0E12D
:107C70000340A0E10370A0E120308DE52030CBE38C
:107C8000450053E39C01001A24209DE5003084E167
:107C9000023093E11E00001A00A0A0E30AB0A0E1A8
:107CA0001C309DE5000053E31C309D1500608315DA
:107CB0000A00A0E10B10A0E184D08DE2F04FBDE8F6
:107CC0001EFF2FE16C308DE567FEFFEA0130D9E53C
:107CD000DF3003E2580053E35A02000A019089E2C0
:107CE0006C908DE500B0D9E530005BE3FAFFFF0A48
:107CF00000005BE33E00000A0130A0E324308DE584
:107D000092FEFFEA0000A0E300C0A0E12C408DE558
:107D100020008DE56C609DE5013086E26C308DE5DC
:107D200001B0D6E52B005BE32202000A2D005BE3E5
:107D300000E0A0130300001A01E0A0E3023086E295
:107D40006C308DE502B0D6E530304BE2090053E3EC
:107D50002501008A30005BE30500001A6C309DE5C8
:107D6000013083E26C308DE500B0D3E530005BE399
:107D7000FAFFFF0A31304BE2080053E35E01008A4C
:107D80006C109DE5013081E26C308DE530204BE2D6
:107D900001B0D1E530108DE530104BE2090051E320
:107DA0006E02008A013083E26C308DE5022182E0B0
:107DB00082208BE000B0D3E530104BE2090051E3A4
:107DC000302042E2F6FFFF9A30109DE5013043E09B
:107DD000080053E3610200DA3C389FE534308DE55A
:107DE00000005EE334309D150030631234308D1591
:107DF000000100EA00A0A0E30AB0A0E11C209DE57C
:107E0000000052E36C309D150030821528309DE54E
:107E1000000053E302318B1203B0A011A3FFFFEA6D
:107E20006C309DE5021083E06C108DE52C408DE5F3
:107E300002B0D3E720008DE530104BE2090051E39A
:107E400001C0A0838CFFFF8A000051E301B0A0E1D4
:107E50006CC09DE5010080E21602001A01308CE240
:107E60006C308DE501B0DCE5F2FFFFEA30309DE5D6
:107E70000BB043E02C309DE503B08BE000005BE3EA
:107E800089FEFFCA95FEFF0A00606BE20F2016E232
:107E90000800000A8C379FE503309AE7823183E0BF
:107EA00010108DE2030091E80C0093E8E32600EB4C
:107EB00010008DE514108DE54662B0E187FEFF0AE3
:107EC0001F0056E32E0000CA103016E26A30A013DD
:107ED00024308DE50030A0E318779FE510108DE287
:107EE000030091E807708FE0287087E2010016E335
:107EF0000200000A0C0097E82C2600EB0130A0E3FA
:107F0000C660B0E1087087E2F7FFFF1A000053E394
:107F100010008D1514108D1524309DE5000053E3DD
:107F20001000000A18379FE510108DE2030091E859
:107F3000213A03E06B2063E2000052E3090000DA1B
:107F40001F0052E32C0300DA340052E30020A0E3C8
:107F500010208DE50020E0D33736A0C34B3063D22C
:107F6000123301D014308DE50020A0E30030A0E3EF
:107F700010108DE2030091E8C4F4FFEB000050E321
:107F800058FEFF0A2230A0E300A0A0E3003088E5FD
:107F90000AB0A0E198FFFFEA0030A0E301B0A0E33F
:107FA0003C308DE5A0FEFFEA70369FE50600A0E1BB
:107FB0000710A0E10020A0E3FC2500EB30309DE598
:107FC000000053E33C008DE540108DE54400001AAD
:107FD000023181E250008DE554308DE550708DE224
:107FE000C00097E8D3FEFFEA0910A0E10320A0E15A
:107FF0000800A0E1D51100EB009050E21B00000A40
:108000000910A0E10800A0E170209DE5481100EBF7
:10801000005050E21500000A0800A0E170109DE534
:108020004A1000EB000054E370508DE590FEFFDA3B
:108030000420A0E10800A0E170109DE50F1200EB04
:10804000000050E370008DE589FEFF1A0050A0E1AA
:108050000A60A0E1070000EA0A10A0E10800A0E120
:1080600048209DE5B91100EB00A050E283FEFF1A05
:108070000A60A0E170509DE52230A0E300A0A0E3DB
:10808000003088E5B4B59FE50510A0E10800A0E147
:108090002E1000EB0610A0E10800A0E12B1000EB71
:1080A0000910A0E10800A0E1281000EB0800A0E101
:1080B0004C109DE5251000EB0800A0E120109DE587
:1080C000221000EB4CFFFFEA0A10A0E10620A0E11D
:1080D0000800A0E1E91100EB00A050E269FEFF1AE0
:1080E000E2FFFFEA3C208DE20C0092E850208DE593
:1080F00054308DE5B8FFFFEA10309DE5000053E3F2
:108100006A00001AFF34C4E30F36C3E3000053E3F0
:108110006B00001A0020A0E30600A0E10710A0E118
:10812000C0349FE55FF4FFEB000050E3C001001A8C
:10813000E8349FE50600A0E10710A0E10020A0E3DD
:108140009A2500EB023181E23C008DE540108DE57F
:1081500060008DE564308DE560708DE2C00097E8C9
:1081600074FEFFEA353644E214308DE510408DE2AE
:10817000180094E80300A0E10410A0E1AC1200EBA9
:108180000020A0E10130A0E10600A0E10710A0E17D
:10819000862500EB10308DE20C0093E802F3FFEB34
:1081A00054249FE50130A0E110008DE514108DE509
:1081B000051001E0020051E14800009A38209DE5D9
:1081C00074349FE5030052E10200001A44309DE53B
:1081D000010073E3A5FFFF0A5C349FE514308DE5D1
:1081E0000030E0E310308DE590FEFFEA0030A0E3C0
:1081F0006C608DE534308DE5000054E39B02001A7D
:1082000024309DE5003093E1F9FEFF1A00005CE3A5
:10821000A0FEFF1A69005BE37F00000A140000CA99
:1082200049005BE37C00000A4E005BE399FEFF1A05
:10823000C8139FE56C408DE20400A0E101108FE0BF
:10824000500E00EB000050E392FEFF0A6C309DE5FB
:108250000030D3E5280053E3CB01000AA0039FE5DB
:1082600000008FE0C31300EB00A0A0E101B0A0E18B
:10827000E1FEFFEA6E005BE3ECFFFF0A85FEFFEA2A
:108280000130A0E328308DE5013089E26C308DE5C6
:1082900001B0D9E500005BE37EFEFF0A0390A0E198
:1082A00026FDFFEA0030A0E328308DE5F5FFFFEA68
:1082B00010309DE5010053E30100001A000054E373
:1082C0005F02000A0030A0E33C308DE514339FE5E7
:1082D0000060A0E340308DE528739FE515FEFFEABE
:1082E000355683E214508DE54AFEFFEA023181E201
:1082F00058008DE55C308DE532FEFFEA0030A0E3EA
:1083000034308DE5BBFFFFEA4D0F56E3E40000CAB1
:10831000100056E34662A0E1E50100DA0030A0E378
:1083200010239FE502B09AE70370A0E10BA0A0E143
:1083300010108DE2030091E8010016E3C660A0E191
:108340000200000A0C009AE8182500EB0130A0E3B7
:10835000010056E3017087E208A08AE2F5FFFF1AE8
:10836000000053E310008D1514108D1514309DE599
:10837000353643E214308DE587718BE010308DE2A5
:108380000C0093E8030097E8082500EBAC329FE56A
:1083900074229FE5013003E0020053E110008DE5F7
:1083A00014108DE5BE00008A012642E2020053E16E
:1083B00084329F8514308D850030E083353681927C
:1083C00010308D8514308D950030A0E324308DE57C
:1083D00044FDFFEA78309DE510308DE574309DE571
:1083E0007C209DE5433E83E2033083E20126C2E325
:1083F000033A82E114308DE5080014E314309D1532
:108400000231831314308D1510408DE2180094E86A
:1084100003A0A0E104B0A0E177FEFFEAEC119FE524
:108420006C408DE20400A0E101108FE0D50D00EB5F
:10843000000050E317FEFF0A6C309DE5D0119FE568
:10844000013043E20400A0E101108FE06C308DE5C3
:10845000CC0D00EB000050E36C309D050130830231
:1084600000A0A0E36C308D05D0B19FE562FEFFEA6D
:1084700020109DE50900A0E120208DE53EFAFFEBEC
:10848000003050E22C308DE520209DE5EE01001AF1
:108490006C109DE5023081E06C308DE502B0D1E7D3
:1084A00030005BE32C009D150600001A012063E2FA
:1084B000020083E0013083E26C308DE500B0D3E54B
:1084C00030005BE3F9FFFF0A31304BE2080053E371
:1084D000E3FDFF8A0050A0E36CC09DE50140A0E3EE
:1084E0000C90A0E10570A0E1013080E220308DE524
:1084F00030B04BE2055185E00000A0E385508BE0F1
:1085000055FEFFEA40409DE53C609DE50410A0E17A
:108510000600A0E1CC2500EB11F3FFEB0020A0E169
:108520000130A0E10600A0E10410A0E11DF2FFEB84
:1085300030C09DE510E09DE5FF54C5E30F56C5E34F
:108540000EC08CE105C09CE10040A0E10150A0E11B
:108550000B00001A64308FE20C0093E851F3FFEB3C
:10856000000050E3B1FDFF0A10408DE2180094E8CE
:108570000A60A0E104B0A0E103A0A0E170509DE575
:10858000C0FEFFEA3C308FE20C0093E845F3FFEBBE
:10859000000050E3F3FFFF1A0400A0E10510A0E182
:1085A00028308FE20C0093E850F3FFEB000050E31B
:1085B0009EFDFF0AEBFFFFEA00E0A0E3DEFDFFEA1D
:1085C0009535A094FFFFCF3F9535A094FFFFDF3F87
:1085D00035E5AF350000E03F7C19FF1F3C0000008F
:1085E00002FCFFFFE2FBFFFF0000F03F0000E07F26
:1085F0000000C0FFFFFFDF41C49F0000FFFF9F7C22
:10860000689C000094A000000000F0BF0000A07C67
:10861000709A0000549A0000449800001F4E000019
:108620000000E03F0000E0BF0C000000FFFF0F0073
:1086300000005039189500001C000000FFFFEF7F7C
:108640000000F07FFF07000028309DE53C201FE57B
:1086500004308DE570308DE208408DE500308DE509
:108660000800A0E102208FE074308DE26C108DE2F2
:10867000E10A00EB075010E20040A0E1DCFDFF0A38
:10868000060055E34000001A00A0A0E31C309DE561
:10869000019089E2000053E30AB0A0E10090831545
:1086A00082FDFFEA2230A0E300A0A0E374B01FE542
:1086B000003088E5D0FDFFEA20309DE5003083E002
:1086C00020308DE5010050E3013084E20320A0E179
:1086D0000F00000A040080E001E040E2000000EA30
:1086E000013083E20420A0E1050185E0080052E3A7
:1086F0000340A0E18050A0910200009A100053E3D3
:10870000077187D08770A0D103005EE1F3FFFF1AE5
:10871000022082E2080054E3150000CA0240A0E1F2
:1087200073FFFFEA160073E3CFFDFFBA20309DE52B
:1087300034209DE5022043E018311FE503309AE71D
:10874000823183E010108DE2030091E80C0093E881
:10875000BA2400EB00A0A0E101B0A0E1A6FDFFEA71
:108760004C311FE5030052E10230A0B134308DE5F9
:108770009AFDFFEA100052E3077187D00240A0E1A2
:108780000000A0E3877081D0B3FDFFEA70209DE573
:10879000000052E30500000A3510A0E378008DE2E6
:1087A000021200EB0800A0E170109DE5670E00EBDF
:1087B000015045E2040055E305F18F900DFFFFEAFB
:1087C00003FFFFEA0A0000EA060000EA000000EAF0
:1087D000FFFEFFEA0231E0E314308DE50030E0E314
:1087E00010308DE503FFFFEAB0311FE514308DE551
:1087F00000FFFFEA78309DE510308DE57C309DE587
:1088000014308DE5FBFEFFEAE8111FE52C009DE525
:1088100001109AE7801181E010308DE20C0093E89E
:10882000030091E8E12300EB00A0A0E101B0A0E18A
:1088300071FDFFEA0020A0E330309DE53C308DE57E
:1088400028321FE540308DE52C321FE560208DE594
:1088500064308DE53FFEFFEA38121FE501409AE7DC
:108860000F8063E2881184E010308DE20C0093E801
:10887000030091E8CD2300EB2C309DE5088043E018
:10888000884184E00C0094E8C82300EB00A0A0E13C
:1088900001B0A0E158FDFFEA30309DE578221FE5E8
:1088A000000053E30A60A0E10B00A0E10450A0E146
:1088B0003C709DE544A09DE538B09DE5023004E0A4
:1088C0004400000A020053E17D00000A000057E363
:1088D0007300000A050017E11B00000A30309DE517
:1088E000000053E30A00A0E10B10A0E19300000A8E
:1088F000CF1000EB24C09DE500005CE30020A0E168
:108900000130A0E10B00000ACCC21FE525CA0CE033
:108910006BC06CE200005CE3060000DA0CCAA0E168
:10892000FF358CE20020A0E3033683E29F2300EBB7
:108930000020A0E10130A0E10A00A0E10B10A0E1BD
:1089400019F1FFEB00A0A0E101B0A0E124309DE50A
:10895000000053E370509DE5CAFDFF0A0A00A0E144
:108960000B10A0E13C331FE50020A0E38F2300EBB8
:108970000030A0E1033091E12230A00300A0A0E18B
:1089800001B0A0E100308805BEFDFFEA60131FE5DD
:1089900001108FE00400A0E1141081E278208DE244
:1089A0008D0C00EB050050E32BFEFF1A7C309DE59B
:1089B0007F3483E30F3683E314308DE578309DE513
:1089C00010308DE510408DE2180094E803A0A0E17E
:1089D00004B0A0E108FDFFEA10209DE5023093E11C
:1089E000B9FFFF1A0520A0E124309DE5000053E304
:1089F000B8331FE5032002E00230A0E17100000A55
:108A00006B0652E36F0000CA370652E3670000DAD4
:108A100070509DE5D0FFFFEA30209DE510408DE2CB
:108A2000180094E8032092E10A60A0E138B09DE5C7
:108A300044A09DE5C4FFFF1AFF34C4E30F36C3E32F
:108A4000050053E10450A0E1BFFFFF1A0231C4E367
:108A5000233AA0E1033AA0E16B0653E3BAFFFF9A81
:108A600020209DE5143092E5000053E30200001A37
:108A7000103092E5010053E3B3FFFFDA0120A0E3D9
:108A800020109DE50800A0E17C0F00EB0910A0E19B
:108A900020008DE5CB0F00EB000050E3AAFFFFDACA
:108AA000CFFFFFEA10209DE5020010E1A6FFFF0ABC
:108AB00089FFFFEA84341FE50070A0E303B09AE762
:108AC00029FEFFEA24309DE5000053E310109DE5E8
:108AD0004700000A9C341FE5043003E06A0653E3B4
:108AE0004300008A0020E0E3233AA0E16B3063E218
:108AF0001233A0E1030051E173FFFF1AC8341FE5F0
:108B0000030055E1010071030130A0030030A01300
:108B100057FDFF0A0510A0E1E0241FE5021001E067
:108B2000012681E214208DE510308DE510408DE2A4
:108B3000180094E803A0A0E104B0A0E182FFFFEADE
:108B40003B1000EB24C09DE500005CE30020A0E1A9
:108B50000130A0E12D00000A1CC51FE525CA0CE06C
:108B60006BC06CE200005CE3060000DA0CCAA0E116
:108B7000FF358CE230209DE5033683E20B2300EBCA
:108B80000020A0E10130A0E10A00A0E10B10A0E16B
:108B900084F0FFEB0020A0E30030A0E300A0A0E100
:108BA00001B0A0E1B9F1FFEB000050E397FFFF0A2D
:108BB0002230A0E300A0A0E3003088E50AB0A0E1E5
:108BC00070509DE52FFDFFEA013643E2233AE0E1D4
:108BD000033AE0E114308DE50030E0E310308DE53C
:108BE00010408DE2180094E803A0A0E104B0A0E1D9
:108BF00055FFFFEA0030E0E3BDFFFFEA0030E0E3AD
:108C000010109DE5133201E010308DE5D5FCFFEA30
:108C10000A00A0E10B10A0E162F0FFEB0020A0E34E
:108C20000030A0E30150A0E100A0A0E101B0A0E16C
:108C300096F1FFEB000050E370509D0511FDFF0A17
:108C4000DAFFFFEA0A60A0E1D8FFFFEA0030A0E304
:108C500003C0A0E10370A0E10350A0E10300A0E184
:108C60000340A0E12C308DE520308DE502FCFFEAC9
:108C700030408DE52C409DE5D4FAFFEA0C309FE5AD
:108C80000CC09FE503308FE00C3093E75FFAFFEAFA
:108C90002803FF1F5400000004E02DE501C0A0E1FF
:108CA00000E0A0E10230A0E11C209FE51C109FE540
:108CB00002208FE0012092E70E10A0E1000092E573
:108CC00004E09DE40C20A0E150FAFFEAFC02FF1F43
:108CD0003400000000C0A0E10120A0E11C109FE5CD
:108CE0001C009FE501108FE0000091E714309FE524
:108CF000000090E5033091E70C10A0E143FAFFEA91
:108D0000C802FF1F3400000054000000F0412DE9AC
:108D100001C0A0E100E0A0E10230A0E1FC209FE55D
:108D2000FC109FE502208FE0017092E70E10A0E199
:108D30000C20A0E1000097E534FAFFEB0140A0E130
:108D40000050A0E10430A0E10520A0E10500A0E171
:108D50000410A0E16BF1FFEB000050E32300001AC8
:108D60000410A0E10500A0E1A0F1FFEB0281C0E347
:108D70000060A0E1AC109FE50800A0E171F3FFEBFB
:108D8000000050E31600001A0800A0E194109FE5CF
:108D90005AF3FFEB000050E31100001A0241C4E354
:108DA0000500A0E10020E0E30410A0E178309FE599
:108DB00054F1FFEB000050E30600001A0500A0E1AB
:108DC0000020E0E30410A0E15C309FE53BF1FFEB05
:108DD000000050E30200000A2220A0E3003097E5E3
:108DE000002083E50600A0E1F041BDE81EFF2FE171
:108DF000000054E3040000AA30009FE500008FE06B
:108E0000E3EFFFEB026180E2F5FFFFEA20009FE560
:108E100000008FE0DEEFFFEB0060A0E1F0FFFFEA73
:108E20008802FF1F34000000FFFF7F7FFFFFEF7FFE
:108E3000F8940000E494000000C0A0E1F0412DE9A6
:108E40000120A0E100119FE500019FE501108FE0E6
:108E5000007091E7F8309FE5000097E5033091E757
:108E60000C10A0E1E9F9FFEB0140A0E10050A0E106
:108E70000430A0E10520A0E10500A0E10410A0E17C
:108E800020F1FFEB000050E32300001A0410A0E1E2
:108E90000500A0E155F1FFEB0281C0E30060A0E115
:108EA000B0109FE50800A0E126F3FFEB000050E3BF
:108EB0001600001A0800A0E198109FE50FF3FFEBE1
:108EC000000050E31100001A0241C4E30500A0E1D4
:108ED0000020E0E30410A0E17C309FE509F1FFEB06
:108EE000000050E30600001A0500A0E10020E0E3C6
:108EF0000410A0E160309FE5F0F0FFEB000050E3CC
:108F00000200000A2220A0E3003097E5002083E55C
:108F10000600A0E1F041BDE81EFF2FE1000054E390
:108F2000040000AA34009FE500008FE098EFFFEBFB
:108F3000026180E2F5FFFFEA24009FE500008FE078
:108F400093EFFFEB0060A0E1F0FFFFEA6001FF1F7D
:108F50003400000054000000FFFF7F7FFFFFEF7F21
:108F6000CC930000B8930000F04F2DE90190A0E1F0
:108F700002A0A0E10370A0E10150A0E1A4C19FE51F
:108F8000A4E19FE50CC08FE00E409CE70CD04DE2C1
:108F900004008DE5014084E20530A0E101C0D5E484
:108FA00004E0DCE708E01EE2FAFFFF1A2D005CE3B4
:108FB0000C40A0E14600000A2B005CE30E60A0011B
:108FC0000E60A0110281E0E30040D505025083024B
:108FD0001030D7E30300001A300054E34100000AC8
:108FE000000057E30A70A00307B0A0E10B10A0E156
:108FF0000800A0E1932100EB0020A0E300E0A0E145
:109000000200A0E1090000EA00304EE0002073E217
:109010000320A2E00C0051E10020A0A3000052E3D5
:109020001400001A0120A0E39BC020E00140D5E419
:1090300030C044E209005CE30700009A41C044E20A
:1090400019005CE337C044920300009A61C044E217
:1090500019005CE30900008A57C044E20C0057E1A4
:10906000060000DA00005EE10040A0230140A033CA
:10907000A23F94E1E3FFFF0A0020E0E3EAFFFFEAFA
:10908000010072E30900000A000056E300006012CC
:1090900000005AE30200000A000052E31F00001A19
:1090A00000908AE50CD08DE2F04FBDE81EFF2FE165
:1090B0002220A0E304309DE500005AE30800A0014F
:1090C000002083E5F6FFFF0A0800A0E1019045E2D9
:1090D000F2FFFFEA0040D5E50281A0E30160A0E3D2
:1090E000025083E2B9FFFFEA0020D5E5DF2002E26B
:1090F000580052E30400001A1070A0E30140D5E5C7
:1091000007B0A0E1025085E2B7FFFFEA000057E395
:109110000870A00307B0A001B3FFFF0AB1FFFFEA88
:109120000080A0E1E7FFFFEA2800FF1F44000000E5
:1091300010402DE901E043E200C07EE20EC0ACE049
:10914000240053E301C08C8300005CE31040BD08A1
:1091500084FFFF0AB1F3FFEB1630A0E31040BDE837
:10916000003080E50000A0E31EFF2FE10230A0E107
:10917000012042E200C072E202C0ACE0240053E3EE
:1091800001C08C8310402DE93CE09FE500005CE3CA
:109190000EE08FE00600001A0120A0E12C109FE5F0
:1091A00001C09EE70010A0E11040BDE800009CE572
:1091B0006CFFFFEA99F3FFEB1630A0E31040BDE827
:1091C000003080E50000A0E31EFF2FE11CFEFE1F23
:1091D000340000000230A0E1012042E200C072E24F
:1091E00002C0ACE0240053E301C08C8310402DE9A1
:1091F0003CE09FE500005CE30EE08FE00600001A13
:109200000120A0E12C109FE501C09EE70010A0E125
:109210001040BDE800009CE552FFFFEA7FF3FFEB42
:109220001630A0E31040BDE8003080E50000A0E368
:109230001EFF2FE1B4FDFE1F3400000010402DE999
:1092400090309FE590209FE503308FE0023093E758
:10925000003093E5000053E30040A0E10200000A63
:10926000382093E5000052E30800000A000054E3B0
:109270000A00000A010054E31100000A020054E34E
:10928000200044120900000A1040BDE81EFF2FE133
:109290000300A0E13D0700EB000054E3F4FFFF1AD8
:1092A00038309FE51040BDE803009FE71EFF2FE127
:1092B0002C309FE503308FE0080093E51040BDE8B7
:1092C0001EFF2FE11C309FE503308FE0040093E583
:1092D0001040BDE81EFF2FE164FDFE1F34000000BA
:1092E000B400FF1FA800FF1F9400FF1FF0432DE9EB
:1092F0000380A0E30040A0E39C509FE514D04DE222
:1093000005508FE004508DE50160A0E30C808DE5F1
:1093100004708DE208408DE50600A0E10710A0E191
:10932000563412EF0090A0E10430A0E304508DE524
:1093300068509FE505508FE00C808DE5009085E535
:1093400008308DE50600A0E10710A0E1563412EFC9
:109350000060A0E10010E0E30430A0E1086085E5D2
:10936000046085E50C2085E2831182E7013083E209
:10937000140053E3FBFFFF1A0030A0E3002095E543
:10938000146085E50C2085E5103085E5183085E50D
:1093900014D08DE2F043BDE81EFF2FE1F88B0000F2
:1093A0002800FF1F70402DE9B8309FE5B8C09FE549
:1093B00003308FE00C3093E7003093E5000053E377
:1093C0000040A0E10160A0E10250A0E110D04DE218
:1093D0000200000A382093E5000052E31200000A60
:1093E000000054E31400000A010054E31900000ACD
:1093F000020054E3204044121200000A50008DE99C
:109400000C508DE50640A0E304508DE20400A0E17D
:109410000510A0E1563412EF0040A0E10400A0E1E5
:1094200010D08DE27040BDE81EFF2FE10300A0E1E7
:10943000D60600EB000054E3EAFFFF1A2C309FE54C
:1094400003409FE7ECFFFFEA24309FE503308FE005
:10945000084093E5E8FFFFEA18309FE503308FE00E
:10946000044093E5E4FFFFEAFCFBFE1F340000002C
:109470001CFFFE1F10FFFE1F00FFFE1FF0402DE926
:1094800014D04DE20060A0E10170A0E10250A0E123
:1094900069FFFFEBC0C09FE50CC08FE00040A0E378
:1094A0000CC08CE2020000EA014084E2140054E3A4
:1094B0000200000A84319CE7030050E1F9FFFF1A23
:1094C0000600A0E15CFFFFEB0660A0E308708DE5FD
:1094D0000C508DE504008DE504708DE20600A0E1DE
:1094E0000710A0E1563412EF0060A0E1000056E33F
:1094F0000C0000BA140054E30600000A5C309FE53B
:1095000003308FE0844183E0103094E5063043E07F
:10951000053083E0103084E5060045E014D08DE28C
:10952000F040BDE81EFF2FE1BCF2FFEB1350A0E3BB
:109530000060A0E30040A0E10500A0E10610A0E16A
:10954000563412EF0050A0E10000E0E3005084E543
:1095500014D08DE2F040BDE81EFF2FE1C4FEFE1FD7
:109560005CFEFE1FF0472DE908D04DE20250A0E15D
:109570000070A0E10160A0E12FFFFFEB04219FE557
:1095800002208FE00040A0E30CC082E2020000EA6B
:10959000014084E2140054E32000000A84319CE777
:1095A000030050E1F9FFFF1A010055E30190A013F9
:1095B0001D00001A842182E0000056E3108092E52D
:1095C0001200000A0590A0E10DA0A0E1068088E04D
:1095D0000700A0E118FFFFEB0A50A0E304808DE52F
:1095E00000008DE50500A0E10A10A0E1563412EF5D
:1095F0000050A0E1000055E30090A0130190090283
:10960000000059E31500001A000055E31B00001A82
:109610000800A0E108D08DE2F047BDE81EFF2FE171
:10962000010055E31500000A0090A0E3020055E395
:109630000680A0110DA0A011E4FFFF1A0C80A0E38A
:109640000DA0A0E100008DE50800A0E10A10A0E156
:10965000563412EF0080A0E1088086E0DBFFFFEACD
:109660000800A0E120309FE503308FE0844183E0D3
:10967000108084E508D08DE2F047BDE81EFF2FE1A1
:109680000080E0E3E1FFFFEADCFDFE1FF4FCFE1FCB
:10969000F0412DE9B2FFFFEB010070E30040A0E1D3
:1096A0000200000A0400A0E1F041BDE81EFF2FE126
:1096B0005AF2FFEB1360A0E30070A0E30050A0E1BA
:1096C0000600A0E10710A0E1563412EF0060A0E10F
:1096D0000400A0E1006085E5F041BDE81EFF2FE138
:1096E00070402DE9B8309FE5B8C09FE503308FE0AA
:1096F0000C3093E7003093E5000053E30040A0E115
:109700000160A0E10250A0E110D04DE20200000A89
:10971000382093E5000052E31200000A000054E3F1
:109720001400000A010054E31900000A020054E387
:10973000204044121200000A50008DE90C508DE5C3
:109740000540A0E304508DE20400A0E10510A0E173
:10975000563412EF0040A0E10400A0E110D08DE2E9
:109760007040BDE81EFF2FE10300A0E1070600EBFB
:10977000000054E3EAFFFF1A2C309FE503409FE707
:10978000ECFFFFEA24309FE503308FE0084093E5CB
:10979000E8FFFFEA18309FE503308FE0044093E5CF
:1097A000E4FFFFEAC0F8FE1F34000000E0FBFE1FEC
:1097B000D4FBFE1FC4FBFE1FF0402DE914D04DE288
:1097C0000060A0E10170A0E10250A0E19AFEFFEB71
:1097D000C4C09FE50CC08FE00040A0E30CC08CE249
:1097E000020000EA014084E2140054E30200000A8F
:1097F00084319CE7030050E1F9FFFF1A0600A0E165
:109800008DFEFFEB0560A0E308708DE50C508DE543
:1098100004008DE504708DE20600A0E10710A0E1D0
:10982000563412EF0060A0E1010076E30500561106
:109830000C00000A140054E30600000A5C309FE5A7
:1098400003308FE0844183E0103094E5063043E03C
:10985000053083E0103084E5060045E014D08DE249
:10986000F040BDE81EFF2FE1ECF1FFEB1350A0E349
:109870000060A0E30040A0E10500A0E10610A0E127
:10988000563412EF0050A0E10000E0E3005084E500
:1098900014D08DE2F040BDE81EFF2FE188FBFE1FD3
:1098A0001CFBFE1FF0402DE9F8209FE502208FE011
:1098B0000040A0E314D04DE20C2082E2020000EA56
:1098C000014084E2140054E32400000A843192E74A
:1098D000010073E3F9FFFF1A2158A0E1015005E2EE
:1098E000020011E302508513020C11E304508513AA
:1098F000010B11E304508513080011E30450C51354
:109900000850851304008DE503F5FFEB0160A0E32B
:1099100008508DE50C008DE504508DE20600A0E1B5
:109920000510A0E1563412EF0050A0E1000055E30D
:109930000F0000BA70309FE503308FE0844183E070
:109940000C5084E5205085E20020A0E30500A0E152
:10995000102084E514D08DE2F040BDE81EFF2FE119
:109960000050E0E30500A0E114D08DE2F040BDE836
:109970001EFF2FE1A9F1FFEB1360A0E30070A0E34D
:109980000040A0E10600A0E10710A0E1563412EF6C
:109990000060A0E10500A0E1006084E514D08DE244
:1099A000F040BDE81EFF2FE1B0FAFE1F24FAFE1FB3
:1099B0000E002DE9F0402DE914109DE5B8FFFFEBF6
:1099C000010070E30040A0E10300000A0400A0E1F0
:1099D000F040BDE80CD08DE21EFF2FE18FF1FFEBD0
:1099E0001360A0E30070A0E30050A0E10600A0E136
:1099F0000710A0E1563412EF0060A0E10400A0E1DE
:109A0000006085E5F040BDE80CD08DE21EFF2FE13F
:109A100030402DE90CD04DE207FEFFEB5CC09FE526
:109A20000CC08FE00030A0E304008DE50C108CE248
:109A3000020000EA013083E2140053E30500000A4B
:109A4000832191E7020050E1F9FFFF1A0020E0E3D3
:109A500083318CE00C2083E50240A0E304508DE2CA
:109A60000400A0E10510A0E1563412EF0040A0E18F
:109A70000400A0E10CD08DE23040BDE81EFF2FE1D4
:109A80003CF9FE1FF0412DE9E0FFFFEB010070E320
:109A90000040A0E10200000A0400A0E1F041BDE89E
:109AA0001EFF2FE15DF1FFEB1360A0E30070A0E368
:109AB0000050A0E10600A0E10710A0E1563412EF2B
:109AC0000060A0E10400A0E1006085E5F041BDE890
:109AD0001EFF2FE1060051E31840A0E304E02DE54E
:109AE0000400000A20509FE50400A0E10510A0E159
:109AF000563412EF0040A0E110509FE50400A0E1B1
:109B00000510A0E1563412EF0040A0E1260002004B
:109B10002300020004E02DE51840A0E30C509FE56F
:109B20000400A0E10510A0E1563412EF0040A0E1CE
:109B3000260002000100A0E31EFF2FE190209FE518
:109B400002208FE00030A0E1AC0092E584109FE598
:109B5000000050E301108FE010402DE91700000ACB
:109B60000D20A0E1033080E0020053E10C00008AE8
:109B700064209FE502208FE060109FE5002092E5C1
:109B8000010052E10100000A020053E10400008AD2
:109B90004C209FE502208FE0AC3082E51040BDE80C
:109BA0001EFF2FE11DF1FFEB0C20A0E30030A0E130
:109BB0001040BDE80000E0E3002083E51EFF2FE138
:109BC00020009FE5001091E70100A0E1AC1082E5C4
:109BD000E2FFFFEA1CF8FE1F58F4FE1FB8F2FE1F5A
:109BE000ADDEFECAC8F7FE1F2000000010402DE9C0
:109BF0000140A0E15820A0E30400A0E10010A0E390
:109C00001FF2FFEB022AA0E3013BA0E30000A0E368
:109C1000042084E5483084E51040BDE81EFF2FE1B4
:109C2000F0412DE90150A0E10010A0E31CFFFFEB83
:109C3000010070E30040A0E10F00000A000050E3C3
:109C4000190000BA5820A0E30500A0E10010A0E32D
:109C50000BF2FFEB812CA0E3013BA0E30400A0E1A9
:109C6000042085E5483085E50040A0E367FFFFEB71
:109C70000400A0E1F041BDE81EFF2FE1E7F0FFEB9B
:109C80001360A0E30070A0E30050A0E10600A0E193
:109C90000710A0E1563412EF0060A0E10400A0E13B
:109CA000006085E5F041BDE81EFF2FE10040E0E3E4
:109CB000EEFFFFEA10402DE9D8F0FFEB5820A0E3BB
:109CC0000030A0E11040BDE80000E0E3002083E5A3
:109CD0001EFF2FE1F0402DE90CD04DE200008DE594
:109CE0000DF4FFEB0E40A0E30D50A0E104008DE564
:109CF0000400A0E10510A0E1563412EF0040A0E1FD
:109D0000010074E30600000A004054E20140A01381
:109D1000004064E20400A0E10CD08DE2F040BDE818
:109D20001EFF2FE1BDF0FFEB1360A0E30070A0E386
:109D30000050A0E10600A0E10710A0E1563412EFA8
:109D40000060A0E10400A0E1006085E50CD08DE298
:109D5000F040BDE81EFF2FE11EFF2FE1F0402DE98E
:109D6000004050E20150A0E10800000A1160A0E3A9
:109D70000070A0E30600A0E10710A0E1563412EF46
:109D80000060A0E1C63FA0E1880084E9006084E5AE
:109D9000000055E30030A0130000A0E3003085155B
:109DA00004308515F040BDE81EFF2FE170402DE91D
:109DB0001050A0E30060A0E30040A0E10500A0E196
:109DC0000610A0E1563412EF0050A0E1060054E165
:109DD0000500A0E160008418086084150C608415FB
:109DE0007040BDE81EFF2FE1F0402DE9E8309FE50F
:109DF000E8209FE503308FE0023093E7003093E5E1
:109E0000000053E30040A0E10CD04DE20200000A44
:109E1000382093E5000052E31300000A000054E3E9
:109E20001500000A010054E31A00000A020054E37E
:109E3000204044121300000A04408DE50950A0E3BD
:109E400004408DE20500A0E10410A0E1563412EFB9
:109E50000040A0E1010074E31200000A0400A0E148
:109E60000CD08DE2F040BDE81EFF2FE10300A0E121
:109E7000460400EB000054E3E9FFFF1A60309FE561
:109E800003409FE7EBFFFFEA58309FE503308FE088
:109E9000084093E5E7FFFFEA4C309FE503308FE091
:109EA000044093E5E3FFFFEA5CF0FFEB1360A0E3FF
:109EB0000070A0E30050A0E10600A0E10710A0E1BF
:109EC000563412EF0060A0E10400A0E1006085E5D7
:109ED0000CD08DE2F040BDE81EFF2FE1B8F1FE1F6F
:109EE00034000000DCF4FE1FD0F4FE1FC0F4FE1F9F
:109EF000F0402DE9003050E20150A0030CD04DE2BB
:109F00001400000A00308DE583F3FFEB1240A0E35C
:109F10000D50A0E104008DE50400A0E10510A0E1D2
:109F2000563412EF0040A0E1010074E30450A0E1B8
:109F30000F00000AFF0054E30600008A000054E30B
:109F40000400000A8450A0E14534A0E1FF3003E2A0
:109F5000040053E10300001A0500A0E10CD08DE2DB
:109F6000F040BDE81EFF2FE18550B0E1F5FFFF1A7C
:109F7000F8FFFFEA29F0FFEB1360A0E30070A0E315
:109F80000040A0E10600A0E10710A0E1563412EF66
:109F90000060A0E1006084E5EEFFFFEAF0402DE9FB
:109FA00014D04DE20140A0E100008DE55AF3FFEB33
:109FB0000030A0E10400A0E118008DE956F3FFEBAA
:109FC0000F40A0E30D50A0E10C008DE50400A0E1DE
:109FD0000510A0E1563412EF0040A0E1010074E347
:109FE0000600000A004054E20140A013004064E271
:109FF0000400A0E114D08DE2F040BDE81EFF2FE187
:10A0000006F0FFEB1360A0E30070A0E30050A0E1B6
:10A010000600A0E10710A0E1563412EF0060A0E1B5
:10A020000400A0E1006085E514D08DE2F040BDE8B9
:10A030001EFF2FE120309FE520209FE503308FE0B9
:10A04000023093E7013083E20330D0E7033003E2CC
:10A05000010053E3200080021EFF2FE170EFFE1F7E
:10A060004400000020309FE520209FE503308FE072
:10A07000023093E7013083E20330D0E7033003E29C
:10A08000020053E3200040021EFF2FE140EFFE1FBD
:10A0900044000000F0432DE92CD04DE20DC0A0E1BA
:10A0A000D4E09FE5023042E20EE08FE0220053E36D
:10A0B0000140A0E10280A0E10070A0E10F00BEE835
:10A0C0000F00ACE80F00BEE80F00ACE80030A08342
:10A0D00003009EE804008CE40030C4850300A081E6
:10A0E0000010CCE52100008A016044E20690A0E166
:10A0F0000050A0E30700A0E10810A0E1511D00EB13
:10A100000720A0E128308DE2011083E0283051E5DE
:10A11000020058E105C0A0E10070A0E10130E9E5CE
:10A12000015085E2F2FFFF9A0030A0E303005CE1FA
:10A130000530C4E7050084100B00000A0620A0E1EA
:10A140000110F6E50630E0E1022082E2043083E00F
:10A1500001E070E5042042E00C3083E0030052E1AE
:10A1600000E0C6E50010C0E5F3FFFFBA0400A0E17F
:10A170002CD08DE2F043BDE81EFF2FE1547E00009D
:10A18000C3FFFFEAF0402DE90160A0E1021CA0E35B
:10A1900085DF4DE210708DE200308DE50C108DE50D
:10A1A0000230A0E10710A0E10C208DE20050A0E1F8
:10A1B0003D0C00EB004050E20E00000A0610A0E14A
:10A1C0000420A0E10500A0E10C309DE51A0000EBA1
:10A1D000070054E10C008DE50300000A0500A0E132
:10A1E0000410A0E1EDF0FFEB0C009DE585DF8DE2B2
:10A1F000F040BDE81EFF2FE10000E0E3FAFFFFEAB8
:10A2000004E02DE501C0A0E100E0A0E10230A0E102
:10A210001C209FE51C109FE502208FE0012092E7A3
:10A220000E10A0E1000092E504E09DE40C20A0E106
:10A23000D3FFFFEA94EDFE1F3400000070402DE9CB
:10A2400001E0A0E10210A0E10020A0E300C0A0E135
:10A2500038009FE538409FE500008FE0045090E70C
:10A26000002085E50E00A0E10320A0E10C40A0E164
:10A2700078E7FFFA010070E30200001A003095E56C
:10A28000000053E3003084157040BDE81EFF2FE14D
:10A2900054EDFE1F0400000010402DE988C09FE52A
:10A2A00088E09FE50CC08FE00EC09CE700E09CE5D5
:10A2B00048C19EE500005CE353CF8E0248C18E0585
:10A2C00004E09CE51F005EE3150000CA000050E3B7
:10A2D0000600001A0000A0E301308EE202E08EE2E8
:10A2E00004308CE50E118CE71040BDE81EFF2FE115
:10A2F000020050E30100A0E30E418CE0882084E5D9
:10A30000102EA0E188019CE5020080E188018CE527
:10A31000083184E58C319C05022083018C218C0559
:10A32000EBFFFFEA0000E0E3EEFFFFEA08EDFE1FAF
:10A3300014000000FFFFFFFF02C0A0E370402DE902
:10A3400028D04DE20150A0E120108DE238409DE57B
:10A3500010108DE51C108DE20C108DE524108DE29F
:10A3600008108DE5011084E200C08DE504108DE534
:10A370003C60DDE5EF0C00EB24E09DE550319FE50E
:10A3800003005EE14C00000A00C0A0E10520A0E14E
:10A390000130DCE4000054E30130C2E4110000DAD3
:10A3A0000130D0E5000053E30130A00340308D05BB
:10A3B0000C00000A2E30A0E30130C5E50130D0E5E5
:10A3C000022085E20130C2E40130FCE5014044E2B4
:10A3D000000053E3000054130110A0C30010A0D3E9
:10A3E000F7FFFFCA40108DE5670056E36560A003E4
:10A3F0000F00000A470056E34560A0030C00000A66
:10A40000000054E30A0000DA40309DE5000053E309
:10A410002E10A013013082E20230A0010010C215FC
:10A420003010A0E3042083E00110C3E4020053E1F4
:10A43000FCFFFF1A01305EE22D00A0432B00A05369
:10A440000210A0E101306E42630053E30260C1E4F8
:10A450000100C2E50F0000CA00C0A0E374009FE540
:10A4600093E0C0E0C32FA0E1402162E0300082E22F
:10A470000000C1E5820E62E0002162E0823083E0EC
:10A48000303083E20130C1E502C0C1E528D08DE261
:10A490007040BDE81EFF2FE13C009FE593C080E0C7
:10A4A000A002A0E130C080E202C0C2E5031082E257
:10A4B0006320E0E3923023E0E6FFFFEA0010A0E132
:10A4C0000500A0E1D8F1FFEB28D08DE27040BDE897
:10A4D0001EFF2FE10F270000676666661F85EB51A0
:10A4E000F0472DE90190A0E104119FE50080A0E173
:10A4F00020D04DE2FC009FE501108FE044509DE527
:10A50000001091E7000055E30240A0E10360A0E1E4
:10A51000007091E52500000A40109DE50C108DE5C6
:10A520000310A0E300108DE51C108DE20820A0E1CF
:10A530000930A0E10700A0E150008DE910108DE581
:10A540007C0C00EB1C309DE5002096E5030050E1FB
:10A55000002062E20530A0E10600002A001042E07F
:10A560000120D0E40120C3E41CC09DE500005CE1B3
:10A57000002081E0F9FFFF8A020054E11A0000DAAE
:10A580003010A0E3022044E0022083E00110C3E485
:10A59000030052E1FCFFFF1A0030A0E30030C2E5E7
:10A5A0000500A0E120D08DE2F047BDE81EFF2FE1BD
:10A5B000502097E5233084E2030052E1545097E5A0
:10A5C000D4FFFFCA24A084E20510A0E10A20A0E184
:10A5D0000700A0E1C00A00EB005050E2EFFFFF0AC5
:10A5E00050A087E5545087E5CAFFFFEA0320A0E1A9
:10A5F000E8FFFFEAB4EAFE1F34000000F0472DE94F
:10A600000170A0E1FC109FE50060A0E120D04DE2C8
:10A61000F4009FE501108FE044509DE5001091E7A4
:10A62000000055E30240A0E10380A0E1009091E525
:10A630002400000A40109DE50C108DE50210A0E3F7
:10A6400000108DE51C108DE20730A0E10620A0E18E
:10A650000900A0E108808DE504408DE510108DE52E
:10A66000340C00EB1C309DE5030050E100C0A0E37A
:10A670000530A0E10500002A0120D0E40120C3E458
:10A680001C209DE5000052E101C08CE2F9FFFF8A29
:10A690000C0054E1190000DA3020A0E30CC044E0C3
:10A6A0000CC083E00120C3E403005CE1FCFFFF1A5F
:10A6B0000030A0E30030CCE50500A0E120D08DE221
:10A6C000F047BDE81EFF2FE1503099E5020053E14D
:10A6D000545099E5D6FFFFCA01A082E20510A0E11F
:10A6E0000A20A0E10900A0E17B0A00EB005050E243
:10A6F000F0FFFF0A50A089E5545089E5CCFFFFEA3E
:10A7000003C0A0E1E9FFFFEA98E9FE1F3400000062
:10A71000F0432DE90310A0E12CD04DE20350A0E15D
:10A720000260A0E10030A0E30080A0E10200A0E10F
:10A730000020A0E3DBEAFFEB000050E302518512AA
:10A740000600A0E10510A0E10020A0E30030A0E396
:10A75000CEEAFFEB48408DE2000050E3900094E821
:10A760005090DDE50700000A3020A0E30030A0E3B0
:10A770000020C7E50130C7E50700A0E12CD08DE23D
:10A78000F043BDE81EFF2FE10600A0E10510A0E1A7
:10A790001F3E8FE20C0093E8C8EAFFEB000050E395
:10A7A0000600001A0400A0E1E70900EB0620A0E182
:10A7B0000530A0E1C1EAFFEB000050E30D00000A04
:10A7C00054109DE5014044E20800A0E108108DE529
:10A7D0000620A0E10530A0E10710A0E104908DE57E
:10A7E00000408DE5D3FEFFEB0700A0E12CD08DE209
:10A7F000F043BDE81EFF2FE10210A0E300108DE53D
:10A8000024108DE210108DE520108DE20C108DE5E6
:10A810001C108DE20620A0E10530A0E10800A0E1B7
:10A8200004408DE508108DE5C20B00EB1C209DE572
:10A8300058319FE5030052E14D00000A0010D0E5B9
:10A84000000051E30730A0E10600001A380000EADA
:10A850000110C3E41C208DE50110F0E5000051E378
:10A86000014044E23200000A000052E3012042E2CB
:10A87000F6FFFFCA54209DE5000052E30500001AD0
:10A880000020D0E5000052E30200001A0020A0E3FF
:10A890000020C3E5B7FFFFEA030057E1012083E290
:10A8A0000230A0013010A0030720A0010210C20452
:10A8B0002E10A0E30010C3E51C309DE5000053E31B
:10A8C000290000AA3010A0E3033042E00110C2E4E6
:10A8D000020053E1FCFFFF1A0020A0E31C208DE5DD
:10A8E0000020D0E5000052E300005413050000DA18
:10A8F0000120C3E40120F0E5014044E2000052E3FE
:10A9000000005413F9FFFFCA54209DE5000052E3F4
:10A91000DDFFFF0A000054E3DBFFFFDA3020A0E395
:10A92000044083E00120C3E4030054E1FCFFFF1A6C
:10A93000D5FFFFEA000054E3000052C3CCFFFFDA6A
:10A9400030C0A0E3012042E20210A0E1014044E255
:10A95000000054E3000051C301C0C3E4012042E2FF
:10A96000F8FFFFCA1C108DE5C1FFFFEA0230A0E12D
:10A97000DAFFFFEA0010A0E10700A0E1AAF0FFEB78
:10A980007CFFFFEA0000A0E12D431CEBE2361A3FFA
:10A990000F270000F0402DE92CD04DE248E0DDE526
:10A9A00045C04EE20150A0E140409DE54C609DE570
:10A9B00022005CE30CF18F90250000EA210000EA00
:10A9C000310000EA260000EA210000EA200000EA47
:10A9D0001F0000EA1E0000EA1D0000EA1C0000EA59
:10A9E0001B0000EA1A0000EA190000EA180000EA59
:10A9F000170000EA160000EA150000EA140000EA59
:10AA0000130000EA120000EA110000EA100000EA58
:10AA10000F0000EA0E0000EA0D0000EA0C0000EA58
:10AA20000B0000EA0A0000EA090000EA080000EA58
:10AA3000070000EA060000EA050000EA010000EA5B
:10AA4000110000EA060000EA10408DE808608DE57C
:10AA500038FEFFEB0500A0E12CD08DE2F040BDE810
:10AA60001EFF2FE1000054E30140A0030C608DE5C0
:10AA700030008DE808E08DE524FFFFEB0500A0E144
:10AA80002CD08DE2F040BDE81EFF2FE10310A0E3C3
:10AA900000108DE524108DE210108DE520108DE260
:10AAA0000C108DE51C108DE2000054E304408DE590
:10AAB00008108DE50160A0131E0B00EB1C209DE526
:10AAC00078319FE5030052E15800000A00C0D0E54C
:10AAD00000005CE30070A0010530A0014700000AFF
:10AAE0000530A0E10070A0E1050000EA012042E28B
:10AAF00001C0C3E41C208DE501C0F7E500005CE364
:10AB00003E00000A000052E3F7FFFFCA000056E3D0
:10AB10003000000A070050E13010A0030110C30408
:10AB2000000054E30010A0D30110A0C3000052E3C2
:10AB30000000A00301000112000050E32E20A0132A
:10AB40001CC09DE50120C314AC2F11E00B00000ACE
:10AB50003020A0E301C08CE2014044E2000054E355
:10AB60000C10A0E10000A0D30100A0C3A10F10E0D1
:10AB70000120C3E401C08CE2F6FFFF1A1C108DE532
:10AB80000010D7E5000051E30A00000A000054E37A
:10AB9000130000DA0720A0E1010000EA000054E3FE
:10ABA0000F00000A0110C3E40110F2E5000051E3B8
:10ABB000014044E2F8FFFF1A000054E33020A0C334
:10ABC000044083C0060000DA0120C3E4040053E11E
:10ABD000FCFFFF1A030000EA0010D7E5000051E374
:10ABE000CBFFFF1A0340A0E10030A0E30500A0E185
:10ABF0000030C4E52CD08DE2F040BDE81EFF2FE10F
:10AC0000000052E3C0FFFFDA30C0A0E302E083E0BF
:10AC100001C0C3E403005EE1FCFFFF1A0020A0E3D3
:10AC2000000056E31C208DE5B9FFFF1AE9FFFFEA9B
:10AC30000010A0E10500A0E1FBEFFFEB84FFFFEABD
:10AC40000F2700000000A0E31EFF2FE110402DE9B8
:10AC500014309FE514209FE503308FE0021093E746
:10AC60000A0100EB1040BDE81EFF2FE154E3FE1F78
:10AC7000100000000000A0E31EFF2FE1F0472DE9C7
:10AC800003C0A0E30040A0E30410A0E300A0A0E103
:10AC90002C319FE5045090E503308FE03C3080E597
:10ACA000BB3F80E2E4C280E5E04280E5E83280E537
:10ACB0000820A0E30C1085E5644085E50410A0E1C0
:10ACC000004085E5044085E5084085E5104085E5C0
:10ACD000144085E5184085E55C0085E2E4609FE569
:10ACE000E7EDFFEB1C5085E5DC309FE506608FE06B
:10ACF000039096E7209085E5D0309FE5038096E7A6
:10AD0000CC309FE5248085E5037096E7C4309FE54D
:10AD1000287085E5036096E7BC309FE52C6085E5EB
:10AD200008509AE50410A0E1644085E5004085E5FF
:10AD3000044085E5084085E5104085E5144085E53B
:10AD4000184085E50C3085E50820A0E35C0085E22D
:10AD5000CBEDFFEB209085E5248085E5287085E527
:10AD60002C6085E574309FE51C5085E50C509AE514
:10AD70000410A0E10C3085E5644085E5004085E5E0
:10AD8000044085E5084085E5104085E5144085E5EB
:10AD9000184085E55C0085E20820A0E3B8EDFFEBF4
:10ADA0000130A0E3209085E51C5085E5248085E5F1
:10ADB000287085E52C6085E538308AE5F047BDE8E8
:10ADC0001EFF2FE1ACFFFFFFC0E2FE1F28000000C6
:10ADD00040000000000000002C00000009000100FD
:10ADE00012000200012041E270402DE9824082E021
:10ADF000042182E08241A0E10160A0E1741084E2BC
:10AE000034EEFFEB005050E20600000A0010A0E311
:10AE10000C0085E2046085E5080085E5001085E505
:10AE2000682084E296EDFFEB0500A0E17040BDE8EC
:10AE30001EFF2FE1F0412DE90C319FE50C219FE52C
:10AE400003308FE0023093E7008093E5383098E5D7
:10AE5000000053E30060A0E12500000A0470A0E3B5
:10AE60002E8E88E2180098E9013053E20300005A60
:10AE70001A0000EA010073E3684084E21700000A48
:10AE8000FC50D4E1000055E3013043E2F8FFFF1A23
:10AE9000BC309FE50820A0E30510A0E1645084E5E4
:10AEA000005084E5045084E5085084E50C3084E5C6
:10AEB000105084E5145084E5185084E55C0084E269
:10AEC0006FEDFFEB305084E5345084E5445084E569
:10AED000485084E50400A0E1F041BDE81EFF2FE1E9
:10AEE000005098E5000055E30400000A0580A0E149
:10AEF000DBFFFFEA0800A0E15FFFFFEBD6FFFFEA00
:10AF00006B1FA0E30600A0E1F2EDFFEB004050E272
:10AF10000900000A0C0084E20510A0E1005084E55D
:10AF20001A2EA0E3047084E5080084E554EDFFEBDD
:10AF30000450A0E1004088E5EBFFFFEA0C30A0E3FD
:10AF4000004088E5003086E5E1FFFFEA6CE1FE1F86
:10AF5000140000000100FFFF10402DE920309FE5A4
:10AF600020209FE503308FE0022093E718109FE533
:10AF7000000092E5011093E7440000EB1040BDE8AB
:10AF80001EFF2FE148E0FE1F14000000100000002B
:10AF9000383090E5000053E31EFF2F1136FFFFEA23
:10AFA0001EFF2FE11EFF2FE11EFF2FE11EFF2FE1ED
:10AFB00010402DE920309FE520209FE503308FE0F1
:10AFC000022093E718109FE5000092E501108FE042
:10AFD000120000EB1040BDE81EFF2FE1F0DFFE1F66
:10AFE0003400000070FCFFFF10402DE920309FE589
:10AFF00020209FE503308FE0022093E718109FE5A3
:10B00000000092E501108FE0040000EB1040BDE865
:10B010001EFF2FE1B8DFFE1F3400000068FCFFFFB9
:10B02000F0412DE90060A0E30180A0E12E7E80E2E6
:10B03000045097E5015055E2084097E50D00004A9D
:10B04000BC30D4E1010053E3015045E20600009A10
:10B05000FE30D4E1010073E30300000A0400A0E124
:10B060000FE0A0E118FF2FE1006086E1010075E329
:10B07000684084E2F1FFFF1A007097E5000057E393
:10B08000EAFFFF1A0600A0E1F041BDE81EFF2FE134
:10B09000F0472DE90090A0E30070A0E10180A0E15D
:10B0A0002E6E80E2045096E5015055E2084096E588
:10B0B0000E00004ABC30D4E1010053E3015045E2E8
:10B0C0000700009AFE30D4E1010073E30400000A97
:10B0D0000410A0E10700A0E10FE0A0E118FF2FE1BC
:10B0E000009089E1010075E3684084E2F0FFFF1AF7
:10B0F000006096E5000056E3E9FFFF1A0900A0E1B1
:10B10000F047BDE81EFF2FE1F0412DE9104090E52A
:10B11000C10254E1220000DA14C080E2C162A0E161
:10B120001FE011E204518CE006318CE02200000A9D
:10B1300006219CE7043083E2030055E1322EA0E1B2
:10B1400020806EE21200009A0C70A0E1001093E5DE
:10B15000112882E1042087E4042093E4030055E1F0
:10B16000322EA0E1F8FFFF8A063044E00331A0E16F
:10B17000053043E22331A0E1013083E2000052E3D5
:10B1800003218CE703318CE01400000A043083E2D1
:10B19000120000EA000052E30C30A011142080E5F8
:10B1A000F9FFFF1A0030A0E3103080E50030A0E383
:10B1B000F041BDE8143080E51EFF2FE1030055E1AA
:10B1C00010208082F6FFFF9A041093E4030055E1FB
:10B1D0000410A2E5FBFFFF8A063044E003318CE057
:10B1E0000C2043E04221A0E10C0053E1102080E557
:10B1F000EDFFFF0AF041BDE81EFF2FE1F04F2DE902
:10B2000050C99FE550E99FE50CC08FE00EC09CE758
:10B210000180A0E100C09CE534D04DE21C008DE52A
:10B220000C00A0E10C40A0E110208DE524308DE55C
:10B2300014C08DE5B8EEFFEB005098E50210D5E59F
:10B24000003084E0300051E30020A0E101B053E57C
:10B250008601001A0100E0E3033085E2050040E0CA
:10B260000350A0E1039080E00110D3E4300051E3EB
:10B27000FAFFFF0AE4489FE504408FE00130D4E77D
:10B28000000053E3CE00000A0070A0E30030D5E5D3
:10B290000330D4E70740A0E1C4189FE5000053E362
:10B2A0000560A0E101108FE00300000A0130F6E51F
:10B2B0000330D1E7000053E3FBFFFF1A0600A0E1D3
:10B2C00014109DE504208DE5ABEEFFEB003050E25D
:10B2D00008308DE504209DE58000000A000054E35D
:10B2E000064044100411A0110030D6E508108D1559
:10B2F00008408D05DF3003E2500053E30640A0E133
:10B300008000000A000057E3006088E5A500001AED
:10B31000053044E0013043E2070053E30710A0E1A9
:10B32000030000DAC330A0E1070053E3011081E21B
:10B33000FBFFFFCA1C009DE504208DE5600300EBC8
:10B34000003050E20C308DE504209DE5F001000A4C
:10B350000C309DE5040055E114A083E220A08DE5AA
:10B360008301002A0060A0E3F8379FE503308FE0F7
:10B3700004308DE5013062E20680A0E118308DE5F1
:10B38000120000EA200056E30610A01104608612A5
:10B390000600001A0A30A0E10010A0E3088083E450
:10B3A00007A0A0E10460A0E30370A0E10180A0E198
:10B3B000013054E50940A0E104009DE50330D0E7E9
:10B3C000050054E10F3003E2138188E11400009A74
:10B3D000013054E50B0053E1019044E204708AE22D
:10B3E000E7FFFF1A18309DE5033089E0050053E1BF
:10B3F000E3FFFF3A0300A0E114109DE52C208DE54A
:10B4000028308DE55CEEFFEB000050E328309DE531
:10B410002C209DE5DAFFFF1A0340A0E1050054E16E
:10B42000EAFFFF8A20309DE5037047E00C309DE580
:10B430004771A0E100808AE50800A0E1107083E573
:10B44000D20300EB10309DE58772A0E1004093E548
:10B45000000047E0040050E1880000CA0060A0A39B
:10B46000E60000BA10309DE508209DE5083093E520
:10B47000020053E1360100BA10109DE508209DE559
:10B48000043091E5020053E1660000DA025043E027
:10B49000050054E1920000CA0C2091E5020052E33D
:10B4A0004401000A030052E35C01000A010052E378
:10B4B0004E01000A5050A0E31C009DE50C109DE5D4
:10B4C000220300EB0030A0E30500A0E158209DE539
:10B4D000003082E534D08DE2F04FBDE81EFF2FE151
:10B4E000000054E3D100000A064044E00431A0E12A
:10B4F00008308DE50030D6E5DF3003E2500053E33D
:10B500000640A0E17EFFFF1A0130D4E52B0053E393
:10B51000B800000A2D0053E300E0A013016084127C
:10B520000200001A01E0A0E30230D4E5026084E2E8
:10B5300034069FE500008FE00310D0E7013041E2C0
:10B54000180053E30460A0816DFFFF8A0130D6E547
:10B550000330D0E701C043E218005CE3101041E281
:10B56000016086E20700008A011181E0813083E0FA
:10B57000101043E20130F6E50330D0E701C043E2AA
:10B5800018005CE3F7FFFF9A08309DE500005EE3DA
:10B5900000106112013083E0000057E308308DE5B0
:10B5A000006088E559FFFF0A000059E30050A0132E
:10B5B0000650A0030500A0E134D08DE2F04FBDE8B5
:10B5C0001EFF2FE10500A0E114109DE504208DE58C
:10B5D000E9EDFFEB000050E304209DE55600001A62
:10B5E0000210D5E70130D4E7000053E3024085E0C4
:10B5F0005300000A300051E30450A0E10500001A96
:10B600000130F5E5300053E3FCFFFF0A5C159FE5D0
:10B6100001108FE00330D1E7017073E20070A033B6
:10B620000190A0E31BFFFFEA0150A0E3000056E3F6
:10B630000800000A10309DE50C3093E5020053E34A
:10B640004700000A030053E34800000A010053E3E7
:10B650006000000A105085E30500A0E158309DE528
:10B660000C209DE5002083E524309DE508209DE524
:10B67000002083E534D08DE2F04FBDE81EFF2FE1BE
:10B680000C509DE5047040E00710A0E10500A0E12A
:10B69000690600EB006050E20A00000A0160A0E3C6
:10B6A00020109DE5013047E2C322A0E1022191E78D
:10B6B0001F1003E2162112E00200000A060053E107
:10B6C000B50000CA0260A0E308309DE50710A0E1C4
:10B6D000073083E00C009DE508308DE589FEFFEB27
:10B6E0005FFFFFEA000056E30160A013017045E22E
:10B6F0000100001A000057E3A200001A0120A0E395
:10B7000020109DE5C732A0E1033191E71F7007E2E9
:10B71000123713E00510A0E10C009DE502608613CE
:10B7200078FEFFEB10309DE5043093E5054044E0E2
:10B7300008308DE50250A0E3BBFFFFEA0540A0E121
:10B740000010D5E5DF1001E2500051E300408815FC
:10B7500094FFFF1A0030A0E30170A0E308308DE5EC
:10B7600068FFFFEA5C309DE5013063E25C308DE507
:10B770005C309DE5000053E3B5FFFF0A0C309DE50A
:10B7800020809DE5106093E50000A0E30830A0E173
:10B790000671A0E1061188E0020000EA030051E111
:10B7A000040003E53400009A03C0A0E1042093E400
:10B7B000010072E3F8FFFF0A012082E2020055E374
:10B7C00000208CE59900000A1F4014E2C100001A15
:10B7D0002150A0E39FFFFFEA020016E39CFFFF0A4F
:10B7E00020309DE5003093E5036086E1010016E31B
:10B7F000E1FFFF1A96FFFFEA00E0A0E349FFFFEA3E
:10B8000008309DE5002044E0023043E00C109DE547
:10B810001C009DE508308DE5180400EB143080E233
:10B820000060A0E30C008DE520308DE50CFFFFEA01
:10B830003C039FE50230D6E700008FE00310D0E71D
:10B8400002C086E0000051E30C60A0E1A8FEFF0A00
:10B850000130F6E50310D0E7000051E3FBFFFF1ACB
:10B8600006C04CE00C11A0E108108DE5A0FEFFEA37
:10B870000090A0E3025085E27DFEFFEA0C309DE5DA
:10B88000083093E5030056E10630A0B1750000AA28
:10B890000110A0E30C009DE5012083E0020055E3C8
:10B8A000033180E0102080E5141083E55F00000A7A
:10B8B000020056E1C3FFFFAA000052E37E0000DA57
:10B8C0000C109DE5022188E0143091E5181081E20A
:10B8D000010052E1A330A0E18700009A08C0A0E176
:10B8E000000091E5803F83E104308CE4043091E472
:10B8F000010052E1A330A0E1F8FFFF8A0C109DE5A2
:10B90000012042E0192042E22221A0E1012082E24E
:10B91000000053E3023188E7023188E07A00001A20
:10B920000C209DE5030058E1083043E04331A0E1DD
:10B93000103082E56300000A10309DE508209DE587
:10B94000083093E5012082E2020053E108208DE5F2
:10B950009EFFFFAA0C109DE51C009DE5FB0100EB7E
:10B960000030A0E358209DE5A350A0E3003082E51D
:10B970000FFFFFEA0C309DE50080A0E320A09DE5CD
:10B98000187083E2A6FEFFEA0710A0E10C009DE517
:10B99000A90500EB0060A0E157FFFFEA0500A0E168
:10B9A000021047E2A40500EB000050E30360A0137F
:10B9B00044FFFF1A42FFFFEA5C209DE5000052E3CE
:10B9C000BBFEFF1A0120A0E324109DE5003081E5B5
:10B9D0000C309DE520109DE5102083E5002081E5D9
:10B9E00058209DE56250A0E3003082E5F0FEFFEABA
:10B9F000050054E1AEFEFF1A010054E3F0FFFF0A18
:10BA00000C009DE5011044E28B0500EB000050E3C3
:10BA1000A7FEFF0A10309DE5043093E5E8FFFFEA3A
:10BA20005C209DE5000052E3A1FEFF0AE4FFFFEA6F
:10BA300010309DE5003093E5013043E2040053E10E
:10BA40002250A01303FFFF1A0120A0E3C432A0E19B
:10BA5000033198E71F4004E2123413E02250A003A0
:10BA60002150A013FBFEFFEA0C309DE5041093E586
:10BA70001C009DE5011081E2910100EB008050E285
:10BA80002A00000A0C909DE5102099E5022082E230
:10BA90000221A0E10C1089E20C0088E2DAE9FFEB58
:10BAA0000910A0E11C009DE5A80100EB0C808DE5CC
:10BAB000103098E5148088E274FFFFEA0030A0E3BC
:10BAC0000C209DE5103082E50030A0E30C209DE5C0
:10BAD000143082E597FFFFEA077088E0040017E55D
:10BAE0002A0200EB204064E2040050E137FFFFAA85
:10BAF0000C309DE5102093E56EFFFFEA000053E354
:10BB0000003088E50830A0110F00000A043083E2FD
:10BB100082FFFFEA0320A0E158009FE558309FE52F
:10BB2000DE10A0E303308FE000008FE05A0600EB48
:10BB300048309FE548009FE50820A0E18410A0E37D
:10BB400003308FE000008FE0530600EB0C209DE5F2
:10BB5000103082E5DBFFFFEAA4DDFE1F3C000000A1
:10BB6000006E0000D46D00000C6D0000446B0000FE
:10BB7000686A000040680000146500000465000069
:10BB8000E8640000F864000000C090E510402DE972
:10BB900001C08CE20040A0E1050000EA0130DCE4D5
:10BBA00041E043E219005EE320308392020053E15A
:10BBB0000600001A0120D1E4000052E3F6FFFF1A4C
:10BBC0000100A0E300C084E51040BDE81EFF2FE1A6
:10BBD0000000A0E31040BDE81EFF2FE1F04F2DE96B
:10BBE00014D04DE208008DE50000A0E3001091E5BF
:10BBF000C132A0E1033182E01F1011E20350A01115
:10BC00000430831204308D0504308D150450430236
:10BC10000C108DE508309DE504109DE5003093E59E
:10BC2000040001E50110D3E55CE29FE5000051E16D
:10BC30000EE08FE0014083E27800000A4C329FE57D
:10BC40000560A0E105C0A0E100A0A0E10070A0E1B6
:10BC500000B0A0E103809EE7150000EA200051E358
:10BC60006C00008A07005AE10E0000AA06005CE1A1
:10BC70000030A0230130A033070050E30030A0C300
:10BC8000000053E34100001A0C0052E10800A02319
:10BC90000400002A04604CE204B00CE507A0A0E117
:10BCA00006C0A0E10000A0E30110F4E5000051E3AC
:10BCB0000E00000A0130D8E7000053E3E6FFFF0A58
:10BCC000010080E2080050E3017087E2280000CA0A
:10BCD00000109CE50112A0E10F3003E2013083E186
:10BCE00000308CE50110F4E5000051E3F0FFFF1A8D
:10BCF000000057E34900000A0C0056E10030A09311
:10BD00000130A083070050E30030A0C3000053E3DC
:10BD10004A00001A0C0052E12900003A0C309DE55F
:10BD2000000053E30000E01304C09DE504101CE58F
:10BD3000203063123013011004100C15000051E381
:10BD40000300000A390000EA043035E5000053E33F
:10BD50003600001A050052E1FAFFFF1A0130A0E395
:10BD60000500A0E3003085E514D08DE2F04FBDE87A
:10BD70001EFF2FE10C0052E1CAFFFF2A04B00CE5C0
:10BD80000010A0E30100A0E304C04CE2D1FFFFEAF1
:10BD90000C10A0E1080060E20001A0E100309CE589
:10BDA000209060E204E091E51E3983E1003081E5F6
:10BDB0003E30A0E10430A1E5060051E1F8FFFF3A72
:10BDC000B0FFFFEA0C30A0E1041042E2040093E46B
:10BDD000050053E10400A1E5FBFFFF9A0C3045E0AC
:10BDE000011085E201C08CE20C0051E10330C3E395
:10BDF000043083E20430A0330010A0E3033082E07B
:10BE0000041083E4050053E1FCFFFF9A04309DE534
:10BE1000041013E5C8FFFFEA290051E31600000AE9
:10BE20000400A0E314D08DE2F04FBDE81EFF2FE127
:10BE30000500A0E314D08DE2F04FBDE81EFF2FE116
:10BE4000083060E20C00A0E10331A0E100109CE5A5
:10BE5000204063E204E090E51E1481E1001080E5DB
:10BE60003E13A0E10410A0E5000056E1F8FFFF8AB0
:10BE70000C0052E1D2FFFF3AA7FFFFEA08309DE530
:10BE8000014084E2004083E598FFFFEA7CD3FE1F77
:10BE90001800000010402DE9004052E20500000AA1
:10BEA00058109FE50400A0E101108FE0D5EAFFEBF8
:10BEB000000050E30300001A44009FE500008FE0FB
:10BEC0001040BDE81EFF2FE138109FE50400A0E1FF
:10BED00001108FE0CBEAFFEB000050E3F5FFFF0A13
:10BEE00024109FE50400A0E101108FE0C5EAFFEBFC
:10BEF000000050E3EFFFFF0A0000A0E3EFFFFFEABE
:10BF0000D8620000C0620000AC6200000C64000057
:10BF100008309FE503308FE02801D3E51EFF2FE1B5
:10BF20002CCFFE1F10402DE9004051E20500000A11
:10BF300058109FE50400A0E101108FE0B1EAFFEB8B
:10BF4000000050E30300001A44009FE500008FE06A
:10BF50001040BDE81EFF2FE138109FE50400A0E16E
:10BF600001108FE0A7EAFFEB000050E3F5FFFF0AA6
:10BF700024109FE50400A0E101108FE0A1EAFFEB8F
:10BF8000000050E3EFFFFF0A0000A0E3EFFFFFEA2D
:10BF900048620000306200001C6200007C63000008
:10BFA00004E02DE518C09FE518E09FE50CC08FE088
:10BFB0000EC09CE7E4E09CE50EC0A0E104E09DE437
:10BFC0001CFF2FE100D0FE1F54000000000051E3D1
:10BFD00008D04DE204108D02000052E30200A001DF
:10BFE0000600000A000053E30600000A0030D2E514
:10BFF000003081E50020D2E5000052E20100A013EC
:10C0000008D08DE21EFF2FE10100E0E3FBFFFFEA15
:10C01000030052E310402DE91100009A01E080E195
:10C0200003001EE300C0A0E10130A0E11D00001AE2
:10C030000310A0E10C00A0E100E091E5004090E5D4
:10C040000E0054E1043083E204C08CE21500001AB3
:10C05000042042E2030052E30C00A0E10310A0E13F
:10C06000F2FFFF8A000052E30200A001014042E219
:10C070000A00000A01C040E2011041E2010000EAAA
:10C08000033090E00900000A01E0FCE50120F1E541
:10C0900002005EE10C3044E0F8FFFF0A02004EE0CF
:10C0A0001040BDE81EFF2FE1014042E2F0FFFFEA31
:10C0B0000300A0E11040BDE81EFF2FE11EFF2FE1AD
:10C0C0001EFF2FE14C3090E5000053E370402DE956
:10C0D0000050A0E10140A0E10900000A040193E73B
:10C0E000000050E30F00000A002090E5042183E7E0
:10C0F0000030A0E3103080E50C3080E57040BDE8F2
:10C100001EFF2FE12120A0E30410A0E3E10300EBD8
:10C11000000050E30030A0E14C0085E5EEFFFF1A7F
:10C120000000A0E3F4FFFFEA0110A0E30500A0E196
:10C130001154A0E1052085E20221A0E1D50300EB26
:10C14000000050E3F5FFFF0A300080E9E7FFFFEA57
:10C15000000051E34C309015042091150201931713
:10C1600000008115021183171EFF2FE1F0412DE918
:10C1700000E0A0E30070A0E10340A0E1E4809FE5BF
:10C180000160A0E1105091E5141081E200C091E53A
:10C1900008300CE0924323E02C08A0E123C8A0E182
:10C1A00092C02CE001E08EE2083003E00C3883E01E
:10C1B0000E0055E1043081E42C48A0E1F2FFFFCAF3
:10C1C000000054E30600000A083096E5050053E13C
:10C1D000060000DA053186E0015085E2144083E56F
:10C1E000105086E50600A0E1F041BDE81EFF2FE1FA
:10C1F000041096E50700A0E1011081E2B0FFFFEB1B
:10C20000008050E21000000A102096E5022082E231
:10C210000C1086E20221A0E10C0088E2FAE7FFEBB5
:10C220004C3097E5042096E5021193E7001086E56F
:10C23000026183E70860A0E1053186E0015085E2F4
:10C24000144083E5105086E5E5FFFFEA18309FE5CE
:10C2500018009FE50820A0E1B510A0E303308FE0AF
:10C2600000008FE08C0400EBFFFF0000CC5D0000BD
:10C27000285F000008C19FE5F0472DE90270A0E1AA
:10C28000082083E20350A0E1090053E3923CCCE094
:10C29000C23FA0E10060A0E10140A0E1CC3063E03A
:10C2A0002E0000DA01C0A0E30010A0E38CC0A0E1E2
:10C2B0000C0053E1011081E2FBFFFFCA0600A0E180
:10C2C0007FFFFFEB001050E22600000A20309DE5C2
:10C2D000143081E50130A0E3090057E30970A0D3D1
:10C2E000103081E50A4084D20E0000CA070055E1F3
:10C2F000090000DA075045E0055084E00130D4E43D
:10C300000A20A0E30600A0E1303043E296FFFFEBF5
:10C31000040055E10010A0E1F7FFFF1A0100A0E1C1
:10C32000F047BDE81EFF2FE1099084E20980A0E1FB
:10C33000074084E00130D8E40A20A0E30600A0E131
:10C34000303043E288FFFFEB040058E10010A0E129
:10C35000F7FFFF1A084047E2044089E0E2FFFFEAE6
:10C360000010A0E3D4FFFFEA18309FE518009FE516
:10C370000120A0E103308FE0CE10A0E300008FE0A9
:10C38000450400EB398EE338B45C00000C5E00001D
:10C390002028A0E10228A0E1000052E30030A0E143
:10C3A0001000A0030000A0131330A001FF0413E34A
:10C3B0000334A001080080020F0213E30332A0013E
:10C3C00004008002030113E30331A0010200800294
:10C3D000000053E31EFF2FB1010113E3010080129F
:10C3E0002000A0031EFF2FE1003090E50020A0E117
:10C3F000070013E20800000A010013E31C00001A02
:10C40000020013E3A330A0112331A0010100A01307
:10C410000200A003003082E51EFF2FE10318A0E117
:10C420002118A0E1000051E31000A0033330A00167
:10C43000FF1003E2000051E32334A0010800800252
:10C440000F0013E32332A00104008002030013E372
:10C450002331A00102008002010013E30200001A50
:10C46000A330B0E1010080E20300000A003082E561
:10C470001EFF2FE10000A0E31EFF2FE12000A0E33C
:10C480001EFF2FE14C3090E5000053E370402DE992
:10C490000040A0E10150A0E10B00000A040093E578
:10C4A000000050E31600000A002090E5042083E518
:10C4B0000020A0E30130A0E3145080E50C2080E5CB
:10C4C000103080E57040BDE81EFF2FE12120A0E381
:10C4D0000410A0E3EF0200EB000050E30030A0E105
:10C4E0004C0084E5ECFFFF1A3C309FE53C009FE5E3
:10C4F0000020A0E3051DA0E303308FE000008FE0E3
:10C50000E50300EB1C20A0E30110A0E30400A0E180
:10C51000E00200EB000050E3F2FFFF0A0120A0E37D
:10C520000230A0E30C0080E9E0FFFFEA305B00008E
:10C530008C5C0000F04F2DE9103092E5105091E531
:10C54000030055E10240A0B10140A0A10360A0B1E9
:10C550000560A0A10350A0A10190A0B10A0094E938
:10C56000057086E00290A0A1070053E114D04DE2CF
:10C57000011081B2D2FEFFEB003050E204308DE5B5
:10C580006700000A04309DE514A083E207B18AE049
:10C590000B005AE10A30A0310020A0330200002A2B
:10C5A000042083E403005BE1FCFFFF8A149089E22E
:10C5B000053189E00320A0E1030059E1143084E251
:10C5C00000308DE5066183E04700002A043046E034
:10C5D000153043E2154084E20330C3E3040056E122
:10C5E000043083E20430A03308B08DE50C708DE593
:10C5F00002B0A0E10370A0E140019FE5040000EA61
:10C600002CC8B0E11C00001A09005BE104A08AE21A
:10C610003300009A04C099E400501CE0F7FFFF0AC1
:10C620000AE0A0E10030A0E300409DE504C094E4EE
:10C6300000109EE500200CE0008001E0958228E0DB
:10C640002CC8A0E12128A0E1952C22E0033088E04D
:10C65000232882E0003003E0023883E1040056E141
:10C6600004308EE42238A0E1EFFFFF8A07308AE72A
:10C6700004C019E52CC8B0E1E2FFFF0A00309AE5DA
:10C680000A40A0E10310A0E10020A0E300E09DE546
:10C6900000509EE52118A0E1005005E09C1521E026
:10C6A000003003E0022081E0023883E1043084E4BA
:10C6B00004309EE4001094E52358A0E1003001E02E
:10C6C0009C3523E00E0056E1223883E02328A0E1C8
:10C6D000EEFFFF8A09005BE107308AE704A08AE2E7
:10C6E000CBFFFF8A08B09DE50C709DE5000057E385
:10C6F000020000CA040000EA017057E20200000ACA
:10C7000004303BE5000053E3FAFFFF0A04309DE5E7
:10C710000300A0E1107083E514D08DE2F04FBDE876
:10C720001EFF2FE10320A0E114009FE514309FE5D8
:10C7300014109FE503308FE000008FE0560300EBFC
:10C74000FFFF0000505A0000F45800005D01000097
:10C75000033012E2F0412DE90240A0E10070A0E1B7
:10C760000160A0012500001A4441B0E11900000A4F
:10C77000485097E5000055E32800000A0080A0E338
:10C78000050000EAC440B0E11200000A000095E58F
:10C79000000050E31200000A0050A0E1010014E381
:10C7A000F7FFFF0A0520A0E10610A0E10700A0E1C5
:10C7B0005FFFFFEB000056E3042096154C30971501
:10C7C000021193170010861502618317C440B0E16F
:10C7D0000060A0E1ECFFFF1A0600A0E1F041BDE817
:10C7E0001EFF2FE10520A0E10510A0E10700A0E158
:10C7F0004FFFFFEB000085E5008080E5E5FFFFEAE5
:10C8000068209FE5013043E202208FE0032192E798
:10C810000030A0E354FEFFEB0060A0E1D1FFFFEA8F
:10C820000110A0E30700A0E125FEFFEB005050E25D
:10C830000700000A38309FE50120A0E3143085E5A9
:10C840000030A0E3102085E5485087E5003085E5FD
:10C85000C9FFFFEA1C309FE51C009FE50520A0E111
:10C86000051DA0E303308FE000008FE00A0300EB1A
:10C87000B859000071020000C457000020590000A0
:10C88000F0472DE90140A0E1106094E5083094E5FF
:10C89000C26286E0015086E2030055E10280A0E119
:10C8A0000070A0E1041091E5C292A0E1030000DA5B
:10C8B0008330A0E1030055E1011081E2FBFFFFCAD4
:10C8C0000700A0E1FEFDFFEB000050E33300000A8B
:10C8D000000059E314E080E2090000DA0E30A0E124
:10C8E0000010A0E3052089E202C1A0E1022180E05E
:10C8F000041083E4020053E1FCFFFF1A14304CE201
:10C9000003E08EE0109094E5143084E21F8018E27A
:10C91000099183E01B00000A0E20A0E100C0A0E303
:10C9200020A068E2001093E511C88CE104C082E405
:10C9300004C093E4030059E13CCAA0E1F8FFFF8A78
:10C94000043049E000005CE3153043E2152084E246
:10C950000560A0110330C3E3020059E1043083E213
:10C960000430A03303C08EE74C3097E5042094E5F3
:10C97000021193E7106080E5001084E5024183E72F
:10C98000F047BDE81EFF2FE104104EE2042093E4BF
:10C99000030059E10420A1E5FBFFFF8AF1FFFFEA54
:10C9A0000020A0E110309FE510009FE510109FE5EA
:10C9B00003308FE000008FE0B70200EB78560000F4
:10C9C000D4570000D901000004E02DE5103091E5B6
:10C9D00000E0A0E1100090E5030050E00C00001A18
:10C9E00014E08EE2141081E203218EE0033181E035
:10C9F000010000EA02005EE10500002A04C032E501
:10CA0000041033E501005CE1F9FFFF0A0100A023F7
:10CA10000100003A04E09DE41EFF2FE10000E0E386
:10CA200004E09DE41EFF2FE1F04F2DE9103092E568
:10CA3000105091E5035045E0000055E30140A0E1AE
:10CA40000290A0E10CD04DE25600001A14E081E201
:10CA5000142082E2032182E003318EE0010000EA2B
:10CA600003005EE15600002A04C033E5041032E5FD
:10CA700001005CE1F9FFFF0A4C00003A041094E564
:10CA80008FFDFFEB000050E35C00000A14B080E271
:10CA90000B80A0E10030A0E3107094E510A099E5B0
:10CAA000142084E20C5080E510E084E268519FE598
:10CAB000144089E204208DE50AA184E0072182E088
:10CAC0000460BEE504C094E4051006E0031081E0B4
:10CAD00005300CE0031041E02C38A0E1263863E07B
:10CAE000413883E0051001E003C881E104005AE108
:10CAF00004C088E44338A0E1F0FFFF8A09104AE04F
:10CB0000151041E2159089E209005AE103E0C1E302
:10CB100004E08EE204E0A0330310C1E30010A03370
:10CB200004409DE50E5084E0050052E101108BE0C9
:10CB30000EB08BE01100009A0B40A0E10510A0E1BF
:10CB4000D4E09FE5048091E40EC008E003308CE05F
:10CB50004368A0E1286886E00E3003E006C883E160
:10CB6000010052E104C084E44638A0E1F4FFFF8AEA
:10CB7000011042E2051041E00310C1E301108BE017
:10CB800000005CE30300001A043031E5000053E3C9
:10CB9000017047E2FBFFFF0A107080E50CD08DE2C8
:10CBA000F04FBDE81EFF2FE10050A0A3B2FFFFAA87
:10CBB0000430A0E10150A0E30940A0E10390A0E10E
:10CBC000ADFFFFEA0010A0E33DFDFFEB000050E3E6
:10CBD0000120A0130030A013102080151430801500
:10CBE000EDFFFF1A0020A0E130309FE530009FE507
:10CBF00030109FE503308FE000008FE0260200EB4D
:10CC00000020A0E120309FE520009FE5091DA0E362
:10CC100003308FE000008FE01F0200EBFFFF0000F9
:10CC200034540000905500003202000018540000F7
:10CC30007455000058309FE5013003E00D3543E2A4
:10CC4000000053E3020000DA0000A0E30310A0E1BB
:10CC50001EFF2FE1003063E2050553E3433AA0E1F4
:10CC6000030000AA0227A0E30000A0E35213A0E102
:10CC70001EFF2FE1143043E21E0053E30221A0D334
:10CC80000130A0C33233A0D10010A0E30300A0E123
:10CC90001EFF2FE10000F07FF0412DE9106090E5CC
:10CCA000144080E2066184E0047016E50700A0E10C
:10CCB000B6FDFFEB203060E20A0050E3003081E572
:10CCC000045046E2130000DA050054E10B3040E264
:10CCD0000900002A000053E3082016E51A00001A94
:10CCE000FF5587E3035685E30240A0E10510A0E16C
:10CCF0000400A0E1F041BDE81EFF2FE1000053E376
:10CD00000320A001F5FFFF0A68109FE50020A0E3C3
:10CD1000175381E1F3FFFFEA58209FE5050054E136
:10CD20000B3060E2375382E10020A0230820163543
:10CD30003223A031153080E2174382E10400A0E1E4
:10CD40000510A0E1F041BDE81EFF2FE1200063E2E5
:10CD50003210A0E1177381E11223A0E1083046E20E
:10CD6000FF5587E3030054E1035685E30C30163585
:10CD700033208231DBFFFFEA0000F03F70402DE9F5
:10CD80000110A0E308D04DE20260A0E10340A0E161
:10CD9000CBFCFFEB005050E23F00000A14119FE56E
:10CDA000FF24C4E30F26C2E3244A11E001268213C4
:10CDB000000056E304208DE51500001A04008DE202
:10CDC00088FDFFEB0130A0E304209DE5000054E363
:10CDD0000310A0E1142085E5103085E5200080E2F5
:10CDE0001F00000A433E44E218209DE5033043E261
:10CDF000003083E0003082E51C309DE5350060E2C4
:10CE0000000083E50500A0E108D08DE27040BDE898
:10CE10001EFF2FE10D00A0E100608DE571FDFFEB2D
:10CE2000000050E304309D1500109D150C009D0876
:10CE300020206012132281113330A0111420851597
:10CE400004308D1514208505000053E30210A01353
:10CE50000110A003000054E3183085E5101085E5AB
:10CE6000DFFFFF1A012185E0433E40E2100092E51A
:10CE700018209DE5023043E2003082E543FDFFEBE0
:10CE8000811260E00500A0E11C309DE5001083E503
:10CE900008D08DE27040BDE81EFF2FE118309FE5FD
:10CEA00018009FE50520A0E114109FE503308FE0F6
:10CEB00000008FE0780100EBFF0700007C510000CC
:10CEC000D85200000A030000F0432DE90CD04DE2D7
:10CED0000160A0E10D10A0E10070A0E16DFFFFEB8B
:10CEE0000040A0E10150A0E10600A0E104108DE2A5
:10CEF00068FFFFEB103097E5102096E5022043E035
:10CF000008109DE80C3043E0823283E0000053E3D8
:10CF1000090000DA039A85E00950A0E10020A0E1B1
:10CF20000130A0E10400A0E10510A0E1C31200EB74
:10CF30000CD08DE2F043BDE81EFF2FE1033663E025
:10CF4000037A81E00710A0E1F3FFFFEA170050E346
:10CF500070402DE90060A0E10A0000DA0000A0E3C3
:10CF60000040A0E338109FE538509FE50420A0E181
:10CF70000530A0E10D1200EB016056E2FAFFFF1A46
:10CF80007040BDE81EFF2FE11C309FE503308FE0AD
:10CF9000806183E0101086E2030091E87040BDE8F4
:10CFA0001EFF2FE10000F03F00002440345200003B
:10CFB00001C041E2101092E5143082E2CCC2A0E13F
:10CFC000011183E001C08CE2010053E10CC180E05B
:10CFD0001200002A10402DE904E040E2044093E4EE
:10CFE000030051E10440AEE5FBFFFF8A023041E05F
:10CFF000153043E20330C3E3043083E2030080E0F2
:10D0000000005CE10300009A0030A0E3043080E4FB
:10D0100000005CE1FCFFFF8A1040BDE81EFF2FE12D
:10D0200000005CE11EFF2F910030A0E3043080E49B
:10D0300000005CE1FCFFFF8A1EFF2FE1103090E54D
:10D04000C122A0E1020053E1140080E2033180B06C
:10D050000C0000BA023180E00A0000DA1F1011E271
:10D060000800000A022190E732C1A0E11C0152E150
:10D070000400000A0100A0E31EFF2FE1042033E5B5
:10D08000000052E3FAFFFF1A000053E1FAFFFF8AA3
:10D090000000A0E31EFF2FE170402DE9916285E0C2
:10D0A000000055E30800001A0610A0E189E5FFEB37
:10D0B000004050E20620A0110510A011F0E4FF1B73
:10D0C0000400A0E17040BDE81EFF2FE10C30A0E39A
:10D0D0000040A0E3003080E5F8FFFFEAF0412DE9D1
:10D0E000005051E20240A0E11E00000A000052E39D
:10D0F0001700000A0080A0E1E00800EB000054E106
:10D100000060A0E10200008AA00054E10570A08147
:10D110000C00008A0410A0E10800A0E16DE5FFEB1F
:10D12000007050E20700000A060054E10510A0E17B
:10D130000420A0310620A02133E4FFEB0510A0E17C
:10D140000800A0E115E5FFEB0700A0E1F041BDE814
:10D150001EFF2FE10470A0E110E5FFEB0700A0E146
:10D16000F041BDE81EFF2FE10210A0E159E5FFEB01
:10D170000070A0E1F3FFFFEA0000A0E300109FE5CC
:10D180001EFF2FE10000F87F10402DE90140A0E1D3
:10D19000FE10D1E1680D00EB000050E3503094A583
:10D1A000BC30D4B1003083A0013AC3B3503084A561
:10D1B000BC30C4B11040BDE81EFF2FE10000A0E369
:10D1C0001EFF2FE1FCC0D1E1010C1CE3F0412DE971
:10D1D0000140A0E10050A0E10260A0E10370A0E1E5
:10D1E000FE10D1E10700001A01CACCE30730A0E12C
:10D1F0000620A0E10500A0E1BCC0C4E10EF4FFEBF5
:10D20000F041BDE81EFF2FE10230A0E30020A0E3C3
:10D21000830800EBFCC0D4E1FE10D4E1F1FFFFEA8B
:10D2200010402DE90140A0E1FE10D1E17C0800EBA7
:10D23000BC30D4E1010070E3013AC303013A831327
:10D2400050008415BC30C4E11040BDE81EFF2FE142
:10D2500010402DE9FE10D1E1B30000EB1040BDE815
:10D260001EFF2FE1000051E30030A01101C080102B
:10D270000200001A0A0000EA0C0053E10600000A4E
:10D280000320A0E10010D2E5000051E3013083E269
:10D29000F8FFFF1A000042E01EFF2FE1000043E00C
:10D2A0001EFF2FE10100A0E11EFF2FE110402DE93C
:10D2B0000240A0E100E094E5000051E300005E13AD
:10D2C0000320A0E101C0A01300C0A00368D04DE27C
:10D2D0001F00000A8C309FE500005EE30EC0A0E155
:10D2E00000108DE510108DE5BC30CDE1110000BAC5
:10D2F00000E0E0E370309DE50D10A0E108C08DE591
:10D3000014C08DE5BEE0CDE1150900EB000050E34F
:10D310000020A0A30030A0B300309DA5000084A58C
:10D320000020C3A510309DA50300A0E168D08DE2C8
:10D330001040BDE81EFF2FE18B20A0E30030A0E3EA
:10D34000002080E50300A0E168D08DE21040BDE838
:10D350001EFF2FE1A23FA0E300C08DE510C08DE5C8
:10D36000BC30CDE1E1FFFFEA0806000000C0A0E10B
:10D3700030402DE90140A0E1001091E500005CE3A0
:10D3800000005113A8009FE5A8E09FE500008FE092
:10D390000E0090E76CD04DE201E0A01300E0A00386
:10D3A000005090E51D00000A01E0A0E1000051E3FB
:10D3B00084109FE500C08DE510C08DE5BC10CDE167
:10D3C000100000BA00C0E0E30500A0E10D10A0E1EC
:10D3D00008E08DE514E08DE5BEC0CDE1E00800EB8E
:10D3E000000050E30020A0A30000A0B300309DA5E2
:10D3F000000084A50020C3A510009DA56CD08DE27F
:10D400003040BDE81EFF2FE18B30A0E30000A0E319
:10D41000003085E56CD08DE23040BDE81EFF2FE185
:10D42000A21FA0E300E08DE510E08DE5BC10CDE18A
:10D43000E3FFFFEA20BCFE1F3400000008060000E6
:10D4400004E02DE518C09FE518E09FE50CC08FE0D3
:10D450000EC09CE7E0E09CE50EC0A0E104E09DE486
:10D460001CFF2FE160BBFE1F54000000000051E3D1
:10D470000030A0E10600000AFF0052E38A20A083EA
:10D480000000E083002083850100A0930020C19567
:10D490001EFF2FE10100A0E11EFF2FE104E02DE5BA
:10D4A00060C09FE560E09FE50CC08FE00EC09CE788
:10D4B00000C09CE50C509CE500C052E201E0A0E1F8
:10D4C0000320A0E114D04DE20A00000A3C109FE5C1
:10D4D00001108FE004108DE534109FE50030A0E1CD
:10D4E00008C08DE500E08DE501108FE00500A0E1AA
:10D4F000B80700EBFDCCFFFA18109FE501108FE094
:10D5000001C0A0E1F2FFFFEA04BBFE1F34000000EF
:10D51000184E0000104E0000F84D00000230A0E14F
:10D5200010402DE90020A0E3DBFFFFEB70402DE968
:10D5300000E0A0E334309FE534209FE503308FE026
:10D54000025093E70040A0E10100A0E100E085E582
:10D550004BF1FFEB010070E30200001A003095E58B
:10D56000000053E3003084157040BDE81EFF2FE13A
:10D5700070BAFE1F04000000F04F2DE9103090E556
:10D58000104091E514D04DE2040053E103008DE812
:10D590000000A0B3630000BA014044E2145081E2ED
:10D5A000148080E2047195E7049198E7017087E2A6
:10D5B0000431A0E10710A0E10900A0E108308DE5E9
:10D5C000E30F00EB070059E1043188E00060A0E1BF
:10D5D0000C308DE5047185E02A00003A0010A0E3CC
:10D5E0000590A0E10800A0E10120A0E140C19FE575
:10D5F00004E099E40C300EE0961321E02EE8A0E15F
:10D600002138A0E1963E2EE000A090E50C3001E02C
:10D61000033042E00CB00AE00C200EE00B3083E057
:10D620002A2862E00C1003E0433882E0031881E10D
:10D63000090057E1041080E44328A0E12E18A0E17E
:10D64000EAFFFF2A08309DE5033098E7000053E326
:10D650000C00001A0C309DE5043043E2030058E151
:10D660000300003A050000EA030058E1014044E2EB
:10D670000200002A042013E4000052E3F9FFFF0A2D
:10D6800000309DE5104083E503009DE8CDFCFFEBF5
:10D69000000050E3220000BA0800A0E10020A0E34F
:10D6A0008C109FE5016086E204C095E400E090E5FF
:10D6B00001300CE0032042E02CC8A0E101300EE074
:10D6C000033082E02EC86CE043288CE0013003E098
:10D6D000023883E1050057E1043080E44228A0E1EC
:10D6E000F0FFFF2A042198E7000052E3043188E0AC
:10D6F0000B00001A043043E2030058E10300003A33
:10D70000050000EA030058E1014044E20200002A5B
:10D71000042013E4000052E3F9FFFF0A00309DE506
:10D72000104083E50600A0E114D08DE2F04FBDE883
:10D730001EFF2FE1FFFF0000F04F2DE90260A0E186
:10D740000370A0E164139FE574D04DE201108FE0F7
:10D7500030108DE5401090E5000051E30040A0E15D
:10D7600008608DE50C708DE5A4509DE50700000A6A
:10D770000130A0E3442090E51332A0E1083081E5B8
:10D78000042081E571FAFFEB0030A0E3403084E52E
:10D79000009057E20130A0B30030A0A3003085E52F
:10D7A0003C339FE50291C9B30C908DB50930D3E1AC
:10D7B0009700000A08308DE20C0093E80200A0E117
:10D7C0000310A0E10020A0E30030A0E328008DE5D5
:10D7D0002C108DE5ADDEFFEB008050E20E00000A5C
:10D7E0000130A0E3A8209DE5000052E3A0209DE5C4
:10D7F000003082E56102000AB4729FE507708FE095
:10D80000033087E0A8209DE5003082E50700A0E115
:10D8100074D08DE2F04FBDE81EFF2FE128B08DE2FD
:10D82000000C9BE868308DE204308DE56C308DE2B1
:10D8300000308DE50400A0E10A20A0E10B30A0E15A
:10D840004DFDFFEB295AB0E134008DE58000001A50
:10D8500068809DE56C509DE5055088E0433E85E27B
:10D86000023083E2200053E3411E85C2021081C2D0
:10D87000403063C2203063D23601A0C1190380C199
:10D880001603A0D10CDEFFEB0130A0E34C308DE598
:10D89000015045E21F1641E20020A0E314329FE54B
:10D8A00040DDFFEB7B3F8FE20C0093E8BF0F00EB06
:10D8B0007A3F8FE20C0093E83BDDFFEB0060A0E1D4
:10D8C0000500A0E10170A0E104DEFFEB753F8FE2EF
:10D8D0000C0093E8B50F00EB0020A0E10130A0E1BF
:10D8E0000600A0E10710A0E12FDDFFEB0060A0E142
:10D8F0000170A0E191DEFFEB0020A0E318008DE5B0
:10D900000090A0E10030A0E30600A0E10710A0E134
:10D9100064DEFFEB000050E30700000A0900A0E10D
:10D92000EEDDFFEB0730A0E10620A0E157DEFFEBC4
:10D93000000050E30130490218308D0518609DE564
:10D94000055048E0013045E2160056E31C308DE5F5
:10D950000202008A30109DE590319FE5033091E787
:10D96000863183E00C0093E828108DE2030091E8F3
:10D970004CDEFFEB000050E35D00000A013046E2A0
:10D9800018308DE50030A0E348308DE5013045E2E8
:10D99000000053E30030A0A324308DA5F20100BAAB
:10D9A00018309DE5000053E3570000AA18309DE5AC
:10D9B00024209DE510308DE5032042E0003063E235
:10D9C0003C308DE50030A0E318308DE598309DE5C2
:10D9D000090053E324208DE55500008A050053E338
:10D9E0000150A0D30050A0C3043043C298308DC56D
:10D9F00098309DE5023043E2030053E303F18F903A
:10DA00000B0400EAEE0200EAEA0200EAE00200EAA1
:10DA1000C60200EAA0309FE5A0209DE5FF94C9E37F
:10DA20000F96C9E3003082E5063099E11200001A32
:10DA3000A8309DE584709FE5000053E307708FE0F8
:10DA400071FFFF0A78709FE507708FE0083087E26A
:10DA50006BFFFFEAFF34CBE30F36C3E3FF5F45E222
:10DA6000FF1583E34C808DE50A00A0E168809DE509
:10DA7000035045E2031681E386FFFFEAA8309DE5E7
:10DA8000000053E38802001A38709FE507708FE0AA
:10DA90005DFFFFEA0000A0E161436F63A787D23F0B
:10DAA000B3C8608B288AC63FFB799F501344D33F8D
:10DAB00060B8FE1F3C4B00000000F83F0F2700003D
:10DAC000F0480000E44800009C4800000000F03FDF
:10DAD000B44100001C00000000001440783E00002B
:10DAE0000000E03F0000F07F0000244000001C40E8
:10DAF0000C000000013045E2000053E348008DB502
:10DB0000990100BA48008DE524008DE518309DE5A7
:10DB10001C209DE510308DE5032082E00030A0E35D
:10DB20003C308DE598309DE5090053E31C208DE5E0
:10DB3000A9FFFF9A0030A0E398308DE50030E0E3C4
:10DB40000150A0E320308DE50030A0E338508DE592
:10DB50009C308DE50010A0E320309DE5441084E565
:10DB600060308DE50400A0E155F9FFEB003050E294
:10DB700014308DE5B904000A20309DE50E0053E312
:10DB80000050A0830150059214309DE5000055E33C
:10DB9000403084E5D300000A10109DE5000051E3F9
:10DBA000EE0100DABC301FE530009DE5033090E760
:10DBB0000F2001E2823183E0010C11E3C00093E801
:10DBC0004152A0E15502000AFC301FE5033090E706
:10DBD00028108DE2030091E8203083E20C0093E8E6
:10DBE000960F00EB0380A0E300A0A0E101B0A0E14C
:10DBF0000F5005E2000055E30E00000A30311FE52A
:10DC000030209DE5039092E7010015E30600000A2D
:10DC10000600A0E10710A0E10C0099E8E30E00EB7C
:10DC20000060A0E10170A0E1018088E2C550B0E190
:10DC3000089089E2F3FFFF1A0A00A0E10B10A0E1AF
:10DC40000620A0E10730A0E17C0F00EB00A0A0E1DE
:10DC500001B0A0E148309DE5000053E30600000A52
:10DC60000020A0E30A00A0E10B10A0E1A8311FE50D
:10DC70008CDDFFEB000050E33C03001A0800A0E13C
:10DC800016DDFFEB0A20A0E10B30A0E1C70E00EB90
:10DC9000AC311FE50020A0E343DCFFEB20309DE525
:10DCA000000053E30080A0E10D9541E27A00000AF4
:10DCB00010309DE564308DE520309DE540308DE5E8
:10DCC0000B10A0E10A00A0E158808DE55C908DE585
:10DCD0009ADDFFEB30109DE5F0311FE5033091E751
:10DCE00040109DE5813183E0060013E9307080E249
:10DCF00050108DE554208DE5F8DCFFEB0130A0E1FC
:10DD00000020A0E10B10A0E10A00A0E125DCFFEB60
:10DD100038309DE514609DE5000053E30080A0E1EC
:10DD20000190A0E1015086E2FF7007E22702000A9D
:10DD300050308DE20C0093E80000A0E364121FE570
:10DD40003E0F00EB58308DE20C0093E815DCFFEB42
:10DD50000070C6E50820A0E10930A0E10060A0E164
:10DD60000170A0E161DDFFEB000050E3C003001A89
:10DD700040B09DE500A0A0E340408DE5210000EA11
:10DD800001A08AE20B005AE1D60300AA0600A0E136
:10DD90000710A0E10020A0E3B8321FE5830E00EBDE
:10DDA0000020A0E3C4321FE50060A0E10170A0E103
:10DDB0000800A0E10910A0E17C0E00EB0190A0E1B9
:10DDC0000080A0E15DDDFFEB0040A0E1C3DCFFEBE4
:10DDD0000020A0E10130A0E10800A0E10910A0E1CD
:10DDE000F0DBFFEB304084E20620A0E10730A0E149
:10DDF0000140C5E40080A0E10190A0E129DDFFEB36
:10DE0000000050E39903001A0820A0E10930A0E1C6
:10DE10000000A0E350131FE5E2DBFFEB0620A0E1CA
:10DE20000730A0E11FDDFFEB000050E3D3FFFF0A46
:10DE300064309DE5013083E240409DE514709DE52E
:10DE400010308DE5010000EA070055E16803000A83
:10DE50000520A0E1013075E5390053E3F9FFFF0A21
:10DE6000013083E214208DE5FF3003E20030C5E588
:10DE7000A80000EA0800A0E198DCFFEB0A20A0E17E
:10DE80000B30A0E1490E00EB0020A0E3A8331FE512
:10DE9000C5DBFFEB0080A0E10D9541E20A00A0E1A7
:10DEA0000B10A0E10020A0E3D8331FE5BDDBFFEBA2
:10DEB0000820A0E10930A0E100A0A0E101B0A0E1AC
:10DEC0000ADDFFEB006050E29A02001A0820A0E190
:10DED0000A00A0E10B10A0E1023189E2F1DCFFEBC6
:10DEE000000050E36001001A6C309DE50320E0E182
:10DEF00010109DE50E0051E3A22FA0E10020A0C369
:10DF0000000052E33C01001A38209DE5000052E376
:10DF1000A900000A98209DE5010052E3AF0200DA53
:10DF200020309DE5012043E23C309DE5020053E1B5
:10DF30003C309DB518109DB5033042B0033081B020
:10DF4000026043A018308DB520309DE53C208DB592
:10DF50000060A0B3000053E31C209DA5032082A015
:10DF60001C208DA524209DA50270A0A120208DB28B
:10DF70000C0092B8033082A024308DA5027043B00B
:10DF80000110A0E30400A0E13DF9FFEB0050A0E187
:10DF90001C209DE5000057E3000052C3080000DA92
:10DFA000020057E10730A0B10230A0A124109DE586
:10DFB000037047E0031041E0033042E024108DE598
:10DFC0001C308DE53C309DE5000053E30700000A5E
:10DFD00038309DE5000053E38F02000A000056E34D
:10DFE000340200CA3C309DE5062053E04102001A8D
:10DFF0000110A0E30400A0E121F9FFEB18209DE54A
:10E00000000052E30060A0E1190100CA98309DE5CC
:10E01000010053E34A0200DA0080A0E318309DE5D6
:10E02000000053E30130A0031901001A1C109DE504
:10E03000013083E01F3013E25600000A202063E223
:10E04000040052E38F0300DA24209DE51C3063E2D4
:10E05000032082E0037087E0033081E024208DE517
:10E060001C308DE524309DE5000053E3040000DA08
:10E070000320A0E10400A0E134109DE5FFF9FFEBCF
:10E0800034008DE51C309DE5000053E3040000DA08
:10E090000610A0E10320A0E10400A0E1F7F9FFEBE6
:10E0A0000060A0E198309DE5020053E348309DE513
:10E0B00000A0A0D301A0A0C3000053E3FE00001AFB
:10E0C00020309DE5000053E300A0A0C301A00AD2C8
:10E0D00000005AE33C00000A20309DE5000053E3B5
:10E0E0008701000A9C309DE50330E0E114709DE556
:10E0F000013083E20610A0E10400A0E110308DE5BC
:10E1000012F8FFEB000055E30200000A0510A0E141
:10E110000400A0E10DF8FFEB34109DE50400A0E140
:10E120000AF8FFEBA8309DE5000053E30030A0E3C0
:10E1300014209DE510109DE50030C2E5A0309DE55E
:10E14000001083E5B0FDFF0A0700A0E1A8309DE5BF
:10E15000002083E574D08DE2F04FBDE81EFF2FE173
:10E160000130A0E348308DE507FEFFEA013065E2AB
:10E1700024308DE50030A0E31C308DE507FEFFEA7A
:10E18000B8761FE507708FE00700A0E174D08DE23C
:10E19000F04FBDE81EFF2FE11C30A0E324209DE5D9
:10E1A000032082E024208DE51C209DE5037087E09C
:10E1B000033082E01C308DE5A9FFFFEA3C609DE55D
:10E1C00024709DE538509DE570FFFFEA38309DE5ED
:10E1D000000053E35C01000A000057E3040000DA8A
:10E1E0000510A0E10720A0E10400A0E1A3F9FFEBE6
:10E1F0000050A0E1000058E30580A001A802001A29
:10E2000008309DE5013003E208308DE514309DE5CE
:10E2100020209DE503A0A0E1013043E2023083E02D
:10E2200020308DE534B09DE5320000EA0010A0E119
:10E230000B00A0E11C308DE5E2F9FFEB0020A0E12E
:10E240000910A0E10400A0E118208DE5BFF7FFEB65
:10E2500098309DE518209DE5031082E108309DE58A
:10E26000013093E11C309DE5D702000A000057E31E
:10E2700001908AE2640200BA98109DE5017087E17E
:10E2800008109DE5071091E15F02000A000052E3CB
:10E29000B00200CA20209DE50A0052E10030CAE524
:10E2A000B902000A0B10A0E10030A0E30A20A0E3AD
:10E2B0000400A0E1ACF7FFEB080055E100B0A0E1DD
:10E2C0000510A0E10030A0E30A20A0E30400A0E1D3
:10E2D0009001000AA4F7FFEB0810A0E10050A0E1B4
:10E2E0000030A0E30A20A0E30400A0E19EF7FFEBCA
:10E2F0000080A0E109A0A0E10610A0E10B00A0E1D0
:10E300009CFCFFEB0030A0E10510A0E10B00A0E1B8
:10E310000390A0E124308DE5AAF9FFEB0820A0E1ED
:10E320000070A0E10610A0E10400A0E1BDF9FFEB40
:10E330000C2090E5000052E3303089E20090A0E12B
:10E34000B9FFFF0A0010A0E10400A0E118308DE53C
:10E350007EF7FFEB0120A0E318309DE5C2FFFFEA46
:10E360003A01000A10209DE580381FE530709DE5D8
:10E37000006062E2033097E70F2006E2823183E01B
:10E380000C0093E828108DE2030091E8070D00EBE4
:10E390004662B0E140008DE544108DE5A702000A19
:10E3A0000030A0E30280A0E300A0A0E101B0A0E162
:10E3B000E4281FE5027097E7010016E30700000A52
:10E3C0000A00A0E10B10A0E10C0097E8F70C00EBAD
:10E3D0000530A0E100A0A0E101B0A0E1018088E249
:10E3E000C660B0E1087087E2F2FFFF1A000053E355
:10E3F00040B08D02000C9B0815FEFFEA20609DE5F1
:10E40000000056E30030A0C30130A0D39C109DE56E
:10E41000A13F13E030109DE530391FE5033091E74F
:10E4200010109DE5813183E0000C93E89A01000A09
:10E43000000056E33401001A0020A0E36C391FE508
:10E440000A00A0E10B10A0E1D80C00EB0020A0E135
:10E450000130A0E128108DE2030091E897DBFFEB8B
:10E46000000050E33401000A20609DE50650A0E161
:10E470001BFFFFEA0010A0E10400A0E1B3F8FFEBEE
:10E4800098309DE5010053E30060A0E1F30000DA5D
:10E490000080A0E3103096E5033186E0100093E59C
:10E4A000BAF7FFEB203060E2DFFEFFEAD8791FE524
:10E4B00007708FE0033087E2D1FCFFEA0610A0E18D
:10E4C00034009DE53FF9FFEB000050E3FBFEFFAA9F
:10E4D00060309DE50A20A0E3000053E300A0A0C344
:10E4E00001A00AD20400A0E10030A0E334109DE5B1
:10E4F0001DF7FFEB38309DE5000053E310309DE53C
:10E5000034008DE5019043E23E02001A00005AE318
:10E510003802001A60309DE520308DE58D0000EA5C
:10E520000280A0E328B08DE2000C9BE8B0FDFFEA7A
:10E530000130A0E338308DE59C309DE510209DE54D
:10E54000023083E060308DE5013083E2010053E367
:10E550000300A0A10100A0B320308DE50010A0E3CE
:10E56000170050E3441084E57DFDFFDA0120A0E3AD
:10E570000430A0E30210A0E18330A0E1142083E284
:10E58000000052E1012081E2F9FFFF9A441084E586
:10E5900073FDFFEA0130A0E338308DE59C309DE546
:10E5A000000053E3DF0000DA0300A0E160308DE5F6
:10E5B00020308DE5E8FFFFEA0030A0E338308DE53C
:10E5C000DCFFFFEA0030A0E338308DE5F2FFFFEA20
:10E5D00058308DE20C0093E850108DE2030091E872
:10E5E000720C00EB14309DE50070C3E540309DE5F2
:10E5F000010053E350008DE554108DE50D02000A33
:10E6000000A0A0E340209DE514309DE5023083E0AA
:10E6100040308DE534BB1FE558408DE50A20A0E170
:10E620000B30A0E10800A0E10910A0E15F0C00EBB5
:10E630000170A0E10060A0E140DBFFEB0040A0E141
:10E64000A6DAFFEB0130A0E10020A0E10710A0E175
:10E650000600A0E1D3D9FFEB304084E20140C5E4DD
:10E6600040309DE5050053E10080A0E10190A0E16C
:10E67000E9FFFF1A58409DE50020A0E3A43B1FE5F9
:10E6800050108DE2030091E8C7D9FFEB0020A0E114
:10E690000130A0E10800A0E10910A0E113DBFFEBCD
:10E6A000000050E37801001A50308DE20C0093E82E
:10E6B0000000A0E3DC1B1FE5BAD9FFEB0020A0E1BE
:10E6C0000130A0E10800A0E10910A0E1F5DAFFEBBC
:10E6D000000050E303FEFF0A40309DE50320A0E167
:10E6E000011073E5300051E3FBFFFF0A64309DE544
:10E6F000013083E214709DE510308DE514208DE526
:10E7000084FEFFEA0610A0E10520A0E30400A0E1DA
:10E7100095F6FFEB0060A0E134009DE50610A0E156
:10E72000A8F8FFEB000050E36DFEFFDA3120A0E314
:10E7300014009DE510309DE50070A0E10120C0E4CB
:10E74000013083E214008DE568FEFFEA10309DE59C
:10E75000013083E210308DE50170A0E314809DE567
:10E7600034A09DE520B09DE5060000EA0A10A0E176
:10E770000030A0E30A20A0E30400A0E17AF6FFEB5A
:10E7800000A0A0E1017087E20610A0E10A00A0E16C
:10E7900078FBFFEB0B0057E1309080E20190C8E47A
:10E7A000F1FFFFBA20309DE5000053E303B0A0C1A4
:10E7B00001B0A0D30070A0E314309DE534A08DE536
:10E7C0000BB083E00120A0E334109DE50400A0E13C
:10E7D0002AF8FFEB0610A0E134008DE579F8FFEB95
:10E7E000000050E301205BE5ED0000DA14109DE528
:10E7F00001304BE2020000EA030051E1F200000A9E
:10E80000012073E5390052E301B083E2F9FFFF0A0A
:10E81000012082E20020C3E50610A0E10400A0E18F
:10E820004AF6FFEB000055E3EE00000A000057E354
:10E83000050057119001000A0710A0E10400A0E1B3
:10E8400014709DE514B08DE540F6FFEB2EFEFFEA57
:10E850000280A0E328B08DE2000C9BE8FCFCFFEAFC
:10E8600008309DE5000053E308FFFF1A08208DE201
:10E87000060092E8FF34C2E30F36C3E3000053E31F
:10E880000230A0E101FFFF1AAC8D1FE5038008E014
:10E89000000058E3E0FDFF0A24309DE5013083E2EB
:10E8A00024308DE51C309DE5013083E20180A0E33A
:10E8B0001C308DE5D8FDFFEA0510A0E10620A0E19F
:10E8C0000400A0E1A1F7FFEB0050A0E134909DE52A
:10E8D0000510A0E10920A0E10400A0E114F7FFEB7E
:10E8E0000080A0E10910A0E10400A0E117F6FFEB11
:10E8F00034808DE5BAFDFFEA0400A0E134109DE507
:10E9000092F7FFEB34008DE5B8FDFFEA0060A0E36D
:10E910000650A0E1F2FDFFEA13F6FFEB0050A0E184
:10E920000080A0E172FEFFEA0130A0E39C308DE59B
:10E9300020308DE586FCFFEA0060A0E30650A0E1F0
:10E9400079FFFFEA08208DE2060092E8000051E31B
:10E95000B0FDFF1AFF34C2E30F36C3E3000053E3F8
:10E9600008809D150230A0E1ABFDFF1AC5FFFFEA4C
:10E9700020309DE5000053E33DFDFF0A60309DE53A
:10E98000000053E357FDFFDA40308DE510309DE580
:10E99000013043E20020A0E30A00A0E10B10A0E157
:10E9A00064308DE5C43E1FE5800B00EB00A0A0E1C4
:10E9B00001B0A0E1010088E2C8D9FFEB0A20A0E184
:10E9C0000B30A0E1790B00EB0020A0E3E83E1FE54F
:10E9D000F5D8FFEB0080A0E10D9541E2B7FCFFEA1E
:10E9E0004C209DE5000052E368309D05433E8312B4
:10E9F0001C209DE50330831236306302032082E041
:10EA00001C208DE524209DE5033082E00270A0E10A
:10EA100024308DE53C609DE558FDFFEA0400A0E14F
:10EA200034109DE53C209DE548F7FFEB34008DE573
:10EA30006EFDFFEA0010A0E30400A0E1441084E5AD
:10EA40009FF5FFEB003050E214308DE50301000A22
:10EA500014309DE510209DE5403084E56C309DE547
:10EA60000E0052E30020A0C30120A0D3000053E316
:10EA70000020A0B3000052E30C01000A30209DE505
:10EA8000983F1FE5033092E710209DE5823183E037
:10EA90000020E0E3000C93E820208DE528708DE253
:10EAA000C00097E80A20A0E10B30A0E10600A0E139
:10EAB0000710A0E1E10B00EB20DAFFEB0080A0E102
:10EAC00086D9FFEB0A20A0E10B30A0E1370B00EB69
:10EAD0000130A0E10020A0E10710A0E10600A0E1C4
:10EAE000B0D8FFEB20309DE514509DE5010053E3C5
:10EAF000303088E20130C5E47D00000A08408DE531
:10EB00000190A0E320409DE5140000EA0A20A0E166
:10EB10000B30A0E10600A0E10710A0E1C70B00EB5D
:10EB200006DAFFEB0080A0E16CD9FFEB0A20A0E140
:10EB30000B30A0E11D0B00EB019089E20130A0E158
:10EB40000020A0E10710A0E10600A0E195D8FFEBAE
:10EB5000303088E2040059E10130C5E46300000A66
:10EB60000020A0E360339FE5100B00EB0020A0E342
:10EB70000030A0E30060A0E10170A0E1C3D9FFEB89
:10EB8000000050E3E0FFFF0A10308DE2880093E8B8
:10EB9000013083E208409DE510308DE514508DE58D
:10EBA0005CFDFFEA0100001A010019E30EFFFF1AE5
:10EBB00001304BE2000000EA012073E5300052E32F
:10EBC00001B083E2FBFFFF0A12FFFFEA10309DE570
:10EBD000013083E210308DE53130A0E314209DE553
:10EBE0000030C2E50BFFFFEA14709DE514B08DE51F
:10EBF00048FDFFEA10309DE5013083E210308DE5DD
:10EC000014208DE53130A0E397FCFFEA0B10A0E162
:10EC100034B08DE509B0A0E10390A0E110309DE58E
:10EC2000000052E3013083E210308DE50B0000DA82
:10EC30000120A0E30400A0E110F7FFEB0610A0E123
:10EC400034008DE55FF7FFEB000050E37F0000DA52
:10EC5000390059E35500000A24309DE5319083E2E4
:10EC60000570A0E10090CAE50850A0E1E9FEFFEAC6
:10EC700040409DE564309DE5013083E214709DE5E0
:10EC800010308DE514508DE522FDFFEA64309DE5DE
:10EC9000013083E214709DE540509DE510308DE514
:10ECA0006AFCFFEA0400A0E1041095E504F5FFEB1F
:10ECB000007050E27600000A102095E5022082E202
:10ECC0000221A0E10C1085E20C0087E24EDDFFEB93
:10ECD0000710A0E10120A0E30400A0E1E7F6FFEBAC
:10ECE0000080A0E145FDFFEA40409DE57DFCFFEA94
:10ECF00008409DE510309DE5013083E20020A0E151
:10ED000010308DE50130A0E127D8FFEB0A20A0E10B
:10ED10000B30A0E10060A0E10170A0E173D9FFEB2E
:10ED2000000050E32600001A0710A0E10A20A0E12D
:10ED30000B30A0E10600A0E154D9FFEB000050E346
:10ED400014709DE50100000A010018E33FFCFF1A62
:10ED500014508DE5EFFCFFEA34B08DE5390053E344
:10ED600009B0A0E10390A0E110309DE5013083E2FD
:10ED700010308DE50D00000A013089E20570A0E138
:10ED80000030CAE50850A0E1A2FEFFEA34B08DE5EC
:10ED900009B0A0E10390A0E110309DE5013083E2CD
:10EDA0000570A0E110308DE50850A0E184FEFFEA77
:10EDB0003920A0E30570A0E10020CAE50850A0E1D9
:10EDC00089FEFFEA14709DE520FCFFEA0390A0E1B4
:10EDD000390053E310309DE5013083E234B08DE516
:10EDE00010308DE501B08AE2F0FFFF0A000057E322
:10EDF00098FFFFCA99FFFFEA60309DE510908DE50E
:10EE000020308DE5B3FCFFEA0510A0E10030A0E35F
:10EE10000A20A0E30400A0E1D3F4FFEB60309DE5FD
:10EE200000005AE30050A0E110908DE520308DE500
:10EE3000A8FCFF1AE7FCFFEA40508DE50DFEFFEA53
:10EE40000280A0E340B08DE2000C9BE880FBFFEA6B
:10EE500082FFFF1A010019E37CFFFF1A7FFFFFEA20
:10EE600068309FE568009FE50020A0E364109FE5FF
:10EE700003308FE000008FE087F9FFEB14709DE511
:10EE800014B08DE5A0FCFFEA3C306312C2FCFF1A0F
:10EE900073FCFFEA40309FE540009FE50720A0E1BA
:10EEA0003C109FE503308FE000008FE07AF9FFEB24
:10EEB0000110A0E39C208DE50020E0E338108DE5F3
:10EEC00060208DE520208DE511FCFFEA0000244044
:10EED000B8310000C8340000AA01000084310000ED
:10EEE00094340000EA02000070402DE90140A0E1E6
:10EEF0000060A0E15E0000EB2C3094E5000053E3DD
:10EF00000050A0E10500000A0600A0E11C1094E5F5
:10EF10000FE0A0E113FF2FE1000050E30050E0B349
:10EF2000BC30D4E1800013E31600001A301094E5E1
:10EF3000000051E30500000A403084E2030051E183
:10EF40000600A01195DDFF1B0030A0E3303084E502
:10EF5000441094E5000051E30300000A0600A0E11C
:10EF60008EDDFFEB0030A0E3443084E50BF0FFEBD7
:10EF70000030A0E3BC30C4E109F0FFEB0500A0E1E4
:10EF80007040BDE81EFF2FE10600A0E1101094E5DF
:10EF900082DDFFEBE4FFFFEA70402DE9004051E223
:10EFA0000800000A000050E30050A0E10200000A3F
:10EFB000383090E5000053E30900000AFC30D4E14A
:10EFC000000053E30200001A0000A0E37040BDE817
:10EFD0001EFF2FE10410A0E10500A0E17040BDE894
:10EFE000C0FFFFEAE9EFFFEBFC30D4E1000053E3A0
:10EFF000F4FFFF0AF6FFFFEA6C309FE570402DE951
:10F00000004050E203308FE00A00000A5C209FE5D8
:10F01000023093E7005093E5000055E30200000A38
:10F02000383095E5000053E30900000AFC30D4E1D4
:10F03000000053E30200001A0000A0E37040BDE8A6
:10F040001EFF2FE10410A0E10500A0E17040BDE823
:10F05000A4FFFFEA0500A0E1CCEFFFEBFC30D4E118
:10F06000000053E3F3FFFF0AF5FFFFEAA89FFE1F2E
:10F0700034000000FC20D1E1080012E3F0412DE94A
:10F080000140A0E10070A0E14700001A043091E5C2
:10F09000022B82E3000053E3BC20C1E1640000DAEC
:10F0A000286094E5000056E36400000A0030A0E305
:10F0B000008097E5015A12E2003087E50238A0E1AE
:10F0C0001C1094E52338A0E15F00001A0130A0E392
:10F0D0000520A0E10700A0E10FE0A0E116FF2FE16D
:10F0E000010070E36400000ABC30D4E1286094E5BC
:10F0F0001C1094E5040013E30500000A303094E589
:10F10000000053E3043094E5030040E03C309415E4
:10F11000030040100020A0E10030A0E30700A0E1C0
:10F120000FE0A0E116FF2FE1010070E34800001A94
:10F13000002097E51D0052E3000052130110A003C8
:10F140000010A013160052E301108103000051E3E8
:10F15000FC30D4E13200000A023BC3E3BC30C4E11E
:10F16000010A13E30030A0E3043084E5103094E595
:10F17000003084E54B00001A301094E5000051E3A4
:10F18000008087E52D00000A403084E2030051E151
:10F190000700A01101DDFF1B0030A0E30300A0E188
:10F1A000303084E5F041BDE81EFF2FE1106091E5AD
:10F1B000000056E32100000A0238A0E12338A0E154
:10F1C000030013E30030A013005091E514309105C3
:10F1D000065045E0000055E3006081E5083081E518
:10F1E000030000CA150000EA000055E3006086E055
:10F1F000120000DA0530A0E10620A0E10700A0E13E
:10F200001C1094E524C094E50FE0A0E11CFF2FE161
:10F21000000050E3005045E0F2FFFFCA0000E0E3C9
:10F22000BC30D4E1403083E3BC30C4E1F041BDE800
:10F230001EFF2FE13C3091E5000053E397FFFFCA2A
:10F240000000A0E3F041BDE81EFF2FE1500094E56F
:10F25000A7FFFFEAFC30D4E1023BC3E3BC30C4E1CA
:10F26000010A13E30030A0E3102094E50C0084E8C9
:10F27000C0FFFF0A500084E5BEFFFFEA003097E5BB
:10F28000000053E397FFFF0A160053E31D005313DA
:10F29000BC30D411403083130500A00100808705E5
:10F2A000BC30C411E6FFFFEA000052E3B1FFFF1AD1
:10F2B000EFFFFFEA70402DE9004050E20150A0E16D
:10F2C0000200000A383094E5000053E30400000A0D
:10F2D000FC00D5E1000050E30500001A7040BDE8D5
:10F2E0001EFF2FE129EFFFEBFC00D5E1000050E30A
:10F2F000F9FFFF0A0510A0E10400A0E17040BDE89D
:10F300005BFFFFEA90309FE570402DE9004050E23E
:10F3100003308FE01800000A80209FE5023093E759
:10F32000005093E5000055E30200000A383095E5EF
:10F33000000053E30900000AFC30D4E1000053E36D
:10F340000300A0010100001A7040BDE81EFF2FE17C
:10F350000410A0E10500A0E17040BDE844FFFFEA11
:10F360000500A0E109EFFFEBFC30D4E1000053E31E
:10F370000300A001F3FFFF0AF4FFFFEA20209FE54E
:10F3800020109FE5023093E701108FE0000093E525
:10F390003EEFFFEB7040BDE81EFF2FE19C9CFE1F7F
:10F3A000340000001400000024FFFFFF0C002DE9D2
:10F3B00004E02DE50CD04DE214308DE210209DE5E7
:10F3C00004308DE5480200EB0CD08DE204E09DE4B2
:10F3D00008D08DE21EFF2FE10E002DE904E02DE59F
:10F3E00008D04DE210308DE22C209FE50010A0E106
:10F3F00004308DE524009FE502208FE0000092E7B5
:10F40000000090E50C209DE5370200EB08D08DE26E
:10F4100004E09DE40CD08DE21EFF2FE1B49BFE1FA3
:10F420003400000070402DE901E0A0E10210A0E1ED
:10F430000020A0E300C0A0E138009FE538409FE530
:10F4400000008FE0045090E7002085E50E00A0E169
:10F450000320A0E10C40A0E18CE8FFEB010070E389
:10F460000200001A003095E5000053E300308415D7
:10F470007040BDE81EFF2FE16C9BFE1F04000000E2
:10F48000040011E5000050E3040040E2003091B7B1
:10F49000030080B01EFF2FE1F0472DE9086091E5E1
:10F4A000030056E10350A0E10140A0E10270A0E199
:10F4B000003091E52800008ABC20D1E1120D12E352
:10F4C0000D00001A0650A0E10520A0E10300A0E114
:10F4D0000710A0E194DBFFEB0000A0E3082094E517
:10F4E000003094E5066042E0055083E0086084E562
:10F4F000005084E5F047BDE81EFF2FE1101091E5B4
:10F50000019043E0143094E501A085E2833083E06C
:10F51000A33F83E009A08AE0C3005AE1C3A0A09101
:10F52000010B12E30080A0E10D00000A0A10A0E127
:10F5300068DCFFEB006050E21800000A0920A0E13F
:10F54000101094E530DBFFEBBC30D4E1123DC3E397
:10F55000803083E3BC30C4E1050000EA0560A0E12F
:10F56000D8FFFFEA0A20A0E1DBF6FFEB006050E2E3
:10F570000700000A093086E009904AE0106084E53F
:10F5800014A084E50560A0E1089084E5003084E5DE
:10F59000CCFFFFEA0800A0E1101094E5FFDBFFEBD1
:10F5A0000C30A0E3003088E5BC30D4E1403083E388
:10F5B0000000E0E3BC30C4E1CDFFFFEAF04F2DE9ED
:10F5C000083092E50CD04DE2000053E30280A0E148
:10F5D00004008DE55800000A007092E50140A0E1AA
:10F5E000000091E5085091E5087087E2330000EAD9
:10F5F000BCC0D4E1120D1CE32100000A10E094E528
:10F60000142094E50E5040E0822082E0A22F82E098
:10F61000061085E0C220A0E1011081E2020051E164
:10F6200002B0A09101B0A0810120A081010B1CE3D8
:10F630002C00000A0210A0E104009DE525DCFFEB90
:10F6400000A050E24200000A0520A0E1101094E55D
:10F65000EDDAFFEBBC20D4E1122DC2E3802082E37F
:10F66000BC20C4E105008AE005504BE0085084E569
:10F6700010A084E50650A0E106A0A0E1000084E50A
:10F6800014B084E50A20A0E10910A0E126DBFFEB1D
:10F69000083098E5082094E5000094E5066043E012
:10F6A000055042E00A0080E0000056E3085084E57F
:10F6B000000084E5086088E51F00000A087087E202
:10F6C000046017E5000056E305A0A0E1089017E5E7
:10F6D000F9FFFF0A060055E1C4FFFF9A0650A0E1BA
:10F6E00006A0A0E1E6FFFFEA0E10A0E104009DE500
:10F6F00079F6FFEB00A050E2D9FFFF1A04509DE518
:10F70000101094E50500A0E1A4DBFFEB0C30A0E3B2
:10F71000003085E50020A0E30000E0E3BC30D4E148
:10F72000403083E3BC30C4E1082088E5042088E54C
:10F730000CD08DE2F04FBDE81EFF2FE10030A0E3BA
:10F740000300A0E1043088E50CD08DE2F04FBDE865
:10F750001EFF2FE10C30A0E304209DE5003082E580
:10F76000EBFFFFEAF04F2DE994C39FE50340A0E1D2
:10F77000BC30D1E10CC08FE07CD04DE2800013E3BF
:10F7800001A0A0E100B0A0E10280A0E108C08DE5E9
:10F790000200000A103091E5000053E3CB00000A9C
:10F7A0000030A0E32C308DE52030A0E33130CDE5F2
:10F7B0003030A0E30170A0E348539FE514408DE58D
:10F7C0003230CDE505508FE00020D8E5000052E34F
:10F7D000250052130840A0E10600000A0460A0E1E1
:10F7E0000120F4E5000052E325005213FAFFFF1A4E
:10F7F000083054E08400001A000052E39000000A30
:10F800000030A0E30020E0E318308DE524308DE5E2
:10F810001C208DE520308DE55B30CDE570308DE529
:10F82000018084E2040000EA0480A0E118309DE534
:10F83000050040E0170083E118008DE50840A0E1D5
:10F840000520A0E30110D4E40500A0E1A40600EB2C
:10F85000000050E30460A0E1F2FFFF1A18309DE5BC
:10F86000100013E32020A0135B20CD15080013E344
:10F870002B20A0130010D8E55B20CD152A0051E302
:10F880003700001A14209DE5001092E5000051E3B6
:10F89000001061B2042082E2023083B324108DA5EF
:10F8A00024108DB514208DE518308DB50110D8E5E4
:10F8B000024088E22E0051E33D00000A48829FE5A5
:10F8C00008808FE00320A0E30800A0E1840600EB9D
:10F8D000000050E34020A0130480A0010640A001D6
:10F8E00018309D15080040101200831118008D1566
:10F8F00018029FE50010D4E50620A0E300008FE089
:10F90000018084123010CDE5750600EB000050E355
:10F910005200000AF8319FE508209DE5033092E788
:10F92000000053E33200000A14308DE200308DE510
:10F93000E0319FE50A20A0E10B00A0E103308FE059
:10F9400018108DE20000A0E10090A0E1010079E331
:10F950003B00000A2C309DE5093083E02C308DE51A
:10F9600098FFFFEA302041E2090052E30860A081DD
:10F97000CFFFFF8A24309DE5000000EA014084E2C9
:10F980000010D4E5033183E0833082E0302041E28F
:10F99000090052E30800A0E10480A0E1F6FFFF9A0D
:10F9A0002E0051E30460A0E124308DE5024080E2A6
:10F9B000C1FFFF1A0110D6E52A0051E33100001AF9
:10F9C00014309DE5002093E5043083E2000052E30B
:10F9D00014308DE5023086E20210D6E5034086E25F
:10F9E0000360A0E10030E0B31C208DE51C308DB534
:10F9F000B1FFFFEA14309DE5073083E20730C3E32F
:10FA0000083083E214308DE5D1FFFFEA0820A0E141
:10FA10000A10A0E10B00A0E10C308DE59DFEFFEB8C
:10FA2000010070E30600000A2C209DE50C309DE5E6
:10FA3000033082E02C308DE50120D6E5000052E352
:10FA40006EFFFF1ABC30DAE1400013E30000E01360
:10FA50002C009D057CD08DE2F04FBDE81EFF2FE10C
:10FA600014308DE200308DE5AC309FE50A20A0E136
:10FA70000B00A0E103308FE018108DE20C0200EBC8
:10FA80000090A0E1B0FFFFEA0030A0E3302041E2A7
:10FA9000090052E30460A0811C308DE5014084829E
:10FAA00085FFFF8A0400A0E10110F4E5033183E043
:10FAB000833082E0302041E2090052E3F8FFFF9AF0
:10FAC0000460A0E11C308DE5024080E27AFFFFEA8D
:10FAD0004010A0E3FFDAFFEB000050E30030A0E1AC
:10FAE0000C30A00300008AE510008AE50000E00366
:10FAF00000308B05D6FFFF0A4030A0E314308AE5C2
:10FB000026FFFFEA3898FE1FAC2B0000B82A000041
:10FB1000802A00002400000054FBFFFF1CFAFFFFB6
:10FB200008C092E501C04CE200005CE310402DE902
:10FB30000230A0E101E0A0E108C082E5070000AAD0
:10FB4000184092E504005CE10040A0B30140A0A38E
:10FB50000A0051E30040A003000054E30600000A3D
:10FB6000002093E5011082E2001083E500E0C2E589
:10FB70000E00A0E11040BDE81EFF2FE1050300EBE1
:10FB80001040BDE81EFF2FE1F0412DE90240A0E149
:10FB9000642091E5020A12E30170A0E10060A0E197
:10FBA0001200001A000053E3035084100150451264
:10FBB000014044120400001A0000A0E3F041BDE837
:10FBC0001EFF2FE1050054E1FAFFFF0A0720A0E124
:10FBD0000600A0E10110F4E5D0FFFFEB010070E3A7
:10FBE000F7FFFF1A0000E0E3F041BDE81EFF2FE140
:10FBF0002351B0E1EFFFFF0A044044E2055184E0E5
:10FC0000010000EA040055E1EAFFFF0A0720A0E135
:10FC10000600A0E10410B4E5DA0300EB010070E394
:10FC2000F7FFFF1A0000E0E3EEFFFFEAF84F2DE9CF
:10FC3000083092E5000053E30280A0E10300A00138
:10FC4000043082051800000A64C091E5020A1CE332
:10FC500001B0A0E11600000A0060A0E1009092E56A
:10FC6000089089E2200419E92A71B0E11600000A1F
:10FC70000040A0E3045045E2010000EA040057E11F
:10FC80001000000A0B20A0E10600A0E10410B5E579
:10FC9000BC0300EB010070E3014084E2F6FFFF1AB1
:10FCA0000030A0E3083088E5043088E5F84FBDE86F
:10FCB0001EFF2FE1D90300EB0030A0E3083088E5F8
:10FCC000043088E5F8FFFFEA083098E503A0CAE3AE
:10FCD0000A3043E0000053E3083088E5089089E2E9
:10FCE000DFFFFF1A0300A0E1ECFFFFEAF04F2DE970
:10FCF00094C39FE57CD04DE20CC08FE000B050E291
:10FD000001A0A0E10280A0E10340A0E108C08DE5D0
:10FD10000200000A38309BE5000053E3D800000AD7
:10FD2000BC30DAE1080013E37300000A10309AE5F2
:10FD3000000053E37000000A0030A0E32C308DE592
:10FD40002030A0E33130CDE53030A0E30170A0E3F6
:10FD500038539FE514408DE53230CDE505508FE0F6
:10FD60000020D8E5000052E3250052130840A0E12E
:10FD70000600000A0460A0E10120F4E5000052E35F
:10FD800025005213FAFFFF1A083054E08B00001AC6
:10FD9000000052E39700000A0030A0E30020E0E3F7
:10FDA00018308DE524308DE51C208DE520308DE563
:10FDB0005B30CDE570308DE5018084E2040000EA1F
:10FDC0000480A0E118309DE5050040E0170083E1C4
:10FDD00018008DE50840A0E10520A0E30110D4E45F
:10FDE0000500A0E13E0500EB000050E30460A0E147
:10FDF000F2FFFF1A18309DE5100013E32020A01336
:10FE00005B20CD15080013E32B20A0130010D8E5CC
:10FE10005B20CD152A0051E33E00001A14209DE519
:10FE2000001092E5000051E3001061B2042082E26C
:10FE3000023083B324108DA524108DB514208DE5D8
:10FE400018308DB50110D8E5024088E22E0051E34C
:10FE50004400000A38829FE508808FE00320A0E379
:10FE60000800A0E11E0500EB000050E34020A013B5
:10FE70000480A0010640A00118309D150800401024
:10FE80001200831118008D1508029FE50010D4E5BB
:10FE90000620A0E300008FE0018084123010CDE541
:10FEA0000F0500EB000050E35900000AE8319FE520
:10FEB00008209DE5033092E7000053E33900000A73
:10FEC00014308DE200308DE5D0319FE50A20A0E1AD
:10FED0000B00A0E103308FE018108DE20000A0E1DC
:10FEE0000090A0E1010079E34200000A2C309DE57A
:10FEF000093083E02C308DE598FFFFEA0A10A0E17D
:10FF00000B00A0E17B0200EB000050E389FFFF0A39
:10FF10000000E0E33B0000EA302041E2090052E348
:10FF20000860A081C8FFFF8A24309DE5000000EA38
:10FF3000014084E20010D4E5033183E0833082E0A5
:10FF4000302041E2090052E30800A0E10480A0E172
:10FF5000F6FFFF9A2E0051E30460A0E124308DE506
:10FF6000024080E2BAFFFF1A0110D6E52A0051E3F1
:10FF70003100001A14309DE5002093E5043083E23F
:10FF8000000052E314308DE5023086E20210D6E51F
:10FF9000034086E20360A0E10030E0B31C208DE561
:10FFA0001C308DB5AAFFFFEA14309DE5073083E2CF
:10FFB0000730C3E3083083E214308DE5CAFFFFEA5F
:10FFC0000820A0E10A10A0E10B00A0E10C308DE5B3
:10FFD000ECFEFFEB010070E30600000A2C209DE51B
:10FFE0000C309DE5033082E02C308DE50120D6E514
:10FFF000000052E367FFFF1ABC30DAE1400013E370
:020000021000EC
:10000000C2FFFF1A2C009DE57CD08DE2F04FBDE8C9
:100010001EFF2FE114308DE200308DE580309FE52A
:100020000A20A0E10B00A0E103308FE018108DE260
:100030009F0000EB0090A0E1A9FFFFEA0030A0E3E1
:10004000302041E2090052E30460A0811C308DE5BC
:10005000014084827EFFFF8A0400A0E10110F4E5E4
:10006000033183E0833082E0302041E2090052E333
:10007000F8FFFF9A0460A0E11C308DE5024080E2A9
:1000800073FFFFEAC1EBFFEB24FFFFEAB492FE1F10
:100090001426000020250000E824000024000000B1
:1000A000ACFCFFFF58FBFFFF04E02DE501C0A0E121
:1000B00000E0A0E10230A0E11C209FE51C109FE5BC
:1000C00002208FE0012092E70E10A0E1000092E5EF
:1000D00004E09DE40C20A0E103FFFFEAEC8EFE1F8C
:1000E00034000000F0472DE90290A0E10360A0E198
:1000F000082091E5103091E5020053E10230A0B1F3
:10010000003089E54320D1E5000052E3013083123D
:1001100000308915003091E5200013E30140A0E193
:100120000050A0E120809DE55A00000A002099E5DA
:10013000022082E2002089E5003091E5060013E309
:100140000310A0E11900001A0C1094E5022041E010
:10015000000052E30310A0D1140000DA0070A0E305
:1001600019A084E2040000EA0CC094E5003099E58F
:1001700003C04CE007005CE10B0000DA0130A0E3B3
:100180000A20A0E10610A0E10500A0E10FE0A0E137
:1001900018FF2FE1010070E3017087E2F1FFFF1A01
:1001A0000000E0E3F047BDE81EFF2FE1001094E5FA
:1001B0004330D4E5003053E20130A013200011E3B6
:1001C0000700000A3010A0E3032084E04310C2E5DA
:1001D000012083E24510D4E5022084E04310C2E50B
:1001E000023083E20610A0E10500A0E1432084E292
:1001F0000FE0A0E118FF2FE1010070E3E7FFFF0A25
:10020000003094E5063003E2043053E20130A013DD
:10021000002099E50C7094E5027047E0A73F93E158
:10022000102094E5083094E51300000A020053E121
:10023000150000DA0070A0E3023043E0037087E0AD
:100240001A9084E20040A0E3010000EA070054E1B4
:100250000D0000AA0130A0E30920A0E10610A0E1F2
:100260000500A0E10FE0A0E118FF2FE1010070E31D
:10027000014084E2F4FFFF1AC8FFFFEA020053E1E5
:10028000ECFFFFCA000057E3ECFFFF1A0000A0E3F9
:10029000F047BDE81EFF2FE1060013E30200000A4D
:1002A000003052E20130A013CDFFFFEA002099E5B3
:1002B000A4FFFFEAF04F2DE90270A0E11820D1E57C
:1002C0001CD04DE20380A0E1000052E3433081E204
:1002D0000140A0E10060A0E140C09DE50C308DE54B
:1002E0003300000A583042E2FF1003E2200051E3DD
:1002F0006500008A200053E303F18F90620000EA5A
:10030000C90000EA600000EA5F0000EA5E0000EA5F
:100310005D0000EA5C0000EA5B0000EA5A0000EAC7
:10032000590000EA580000EA570000EA7C0000EAA1
:100330005C0000EA540000EA530000EA520000EAC0
:10034000510000EA570000EA4F0000EA4E0000EAC0
:100350004D0000EA4C0000EA090000EA610000EAF2
:10036000850000EA480000EA470000EA750000EA5C
:10037000450000EA5B0000EA430000EA420000EAB0
:10038000AF0000EA00309CE5002094E5040083E221
:10039000141094E500008CE5800012E3003093E532
:1003A0000200001A400012E3B010C3110000001A4E
:1003B000001083E50030A0E3103084E5439084E230
:1003C0000730A0E10410A0E10600A0E100808DE567
:1003D00014208DE242FFFFEB010070E32000000AD1
:1003E0000920A0E10710A0E10600A0E1103094E58B
:1003F0000FE0A0E118FF2FE1010070E31800000AF0
:10040000003094E5020013E314E09DE50CC094E590
:100410001700000A0E304CE0000053E3140000DA2D
:100420000050A0E3199084E2040000EA0CC094E5B7
:1004300014E09DE50E304CE0050053E10C0000DABD
:100440000130A0E30920A0E10710A0E10600A0E12F
:100450000FE0A0E118FF2FE1010070E3015085E2F9
:10046000F1FFFF1A0000E0E31CD08DE2F04FBDE881
:100470001EFF2FE10E005CE10C00A0A10E00A0B158
:100480001CD08DE2F04FBDE81EFF2FE10130A0E34C
:100490004220C4E5429084E2103084E50030A0E3BD
:1004A0004330C4E5C5FFFFEA003094E500209CE539
:1004B000800013E3041082E200108CE50100001AB2
:1004C000400013E38A00001A002092E50250A0E1E8
:1004D000000052E35C0000BA40A29FE50AB0A0E32E
:1004E0000AA08FE03E0000EA001094E500309CE591
:1004F000800011E3040083E200008CE50100001A93
:10050000400011E37800001A005093E56F0052E3B9
:100510007A00000A08A29FE50AB0A0E30AA08FE0D3
:100520002D0000EA0120A0E300309CE5001093E5D7
:10053000043083E200308CE5429084E24210C4E54E
:10054000102084E5D4FFFFEA00309CE5042083E21C
:1005500000208CE5009093E50010A0E30900A0E1E5
:10056000042094E55E0300EB000050E309304010E6
:100570000430940504308415C6FFFFEA003094E58A
:10058000203083E3003084E57820A0E394A19FE548
:100590004520C4E50AA08FE000209CE5045092E4C9
:1005A000800013E300208CE50200001A400013E3F2
:1005B0000558A0112558A011010013E32030831322
:1005C00000308415000055E310B0A01310B0A00354
:1005D000003094052030C303003084050020A0E3E0
:1005E0004320C4E5042094E5000052E3082084E59C
:1005F000370000BA001094E5000055E30410C1E391
:10060000001084E51C00001A000052E343908402AD
:100610003100001A08005BE32300000A0C309DE55E
:1006200009B043E010B084E564FFFFEA5830A0E36E
:10063000F4A09FE54530C4E50AA08FE0003094E5C2
:10064000D4FFFFEA003094E5CEFFFFEA2D20A0E3BF
:100650004320C4E5042094E5000052E3082084E52B
:10066000005065E2290000BA0AB0A0E3BCA09FE5F3
:100670000430C3E3003084E50AA08FE0439084E2B5
:100680000500A0E10B10A0E1EE0300EB05C0A0E126
:100690000120DAE70B005CE10050A0E1012069E5F0
:1006A000F6FFFF2A08005BE3DBFFFF1A003094E54A
:1006B000010013E3D8FFFF0A103094E5042094E50D
:1006C000030052E13030A0D3013049D5019049D226
:1006D000D1FFFFEA000055E3E7FFFF1A0020DAE54B
:1006E000429084E24220C4E5C9FFFFEAB050D3E162
:1006F00085FFFFEAF050D2E10520A0E173FFFFEA99
:100700002CA09FE508B0A0E30AA08FE0B2FFFFEAAB
:1007100020A09FE50AB0A0E30AA08FE0D6FFFFEA81
:10072000A41E0000681E0000041E00004C1D0000F6
:100730000C1D00007C1C00006C1C000070402DE9AA
:1007400001E0A0E10210A0E10020A0E300C0A0E1D0
:1007500038009FE538409FE500008FE0045090E7A7
:10076000002085E50E00A0E10320A0E10C40A0E1FF
:1007700043C0FFFA010070E30200001A003095E563
:10078000000053E3003084157040BDE81EFF2FE1E8
:100790005488FE1F04000000F0412DE9006050E283
:1007A0000150A0E10240A0E10200000A383096E5C5
:1007B000000053E33300000AFC00D4E1183094E554
:1007C0000028A0E1080010E3083084E52228A0E119
:1007D0002200000A103094E5000053E31F00000AD5
:1007E000020A12E364209405022AC20364208405ED
:1007F000002094E5141094E5020A8003033042E0DF
:10080000BC00C401FF5005E2030051E10570A0E106
:10081000013083C2240000DA081094E5011041E29F
:10082000081084E5011082E2001084E50050C2E562
:10083000142094E5030052E11400000ABC30D4E116
:100840000A0055E30030A01301300302000053E317
:100850000E00001A0700A0E1F041BDE81EFF2FE1E5
:100860000410A0E10600A0E1220000EB000050E32C
:100870000B00001AFC00D4E10028A0E1103094E540
:100880002228A0E1D5FFFFEAC0E9FFEBC9FFFFEA9C
:100890000410A0E10600A0E185FAFFEB000050E3A0
:1008A000EBFFFF0A0070E0E3E9FFFFEA0410A0E1BC
:1008B0000600A0E17EFAFFEB000050E3F8FFFF1A0C
:1008C0000130A0E3002094E5D2FFFFEA00C0A0E1E0
:1008D00018309FE50120A0E114109FE503308FE060
:1008E000013093E70C10A0E1000093E5A9FFFFEAB7
:1008F000D086FE1F3400000070402DE968319FE56E
:1009000068219FE503308FE0023093E7003093E5E4
:10091000000053E30050A0E10140A0E10200000A02
:10092000382093E5000052E32000000AFC20D4E1C7
:100930000238A0E1080012E32338A0E11E00000AFB
:10094000101094E5000051E32600000A010013E2B4
:100950000700001A020013E314009405000051E39D
:10096000080084E50000A0130900000A7040BDE8FB
:100970001EFF2FE100C0A0E3140094E5000051E346
:10098000000060E2180084E508C084E50000A013C0
:10099000F5FFFF1A800013E3402082130000E013EC
:1009A0000100A001BC20C4117040BDE81EFF2FE172
:1009B0000300A0E175E9FFEBDBFFFFEA100013E3A2
:1009C0002300000A040013E31100001A101094E53C
:1009D000082082E30238A0E1000051E3BC20C4E11A
:1009E0002338A0E1D8FFFF1A0A0D03E2020C50E3FE
:1009F000D5FFFF0A0410A0E10500A0E1BB0100EB58
:100A0000FC20D4E10238A0E1101094E52338A0E1E5
:100A1000CDFFFFEA301094E5000051E30700000A23
:100A2000403084E2030051E10200000A0500A0E129
:100A3000DAD6FFEBFC20D4E10030A0E3303084E5CF
:100A40000030A0E3101094E52420C2E30A0084E8FB
:100A5000DEFFFFEA0930A0E3402082E3003085E5B5
:100A60000000E0E3BC20C4E1BFFFFFEAA886FE1F50
:100A700034000000F0432DE90CD04DE20070A0E1FD
:100A80000180A0E10240A0E120EDFFEB010050E376
:100A90000200001A013048E2FE0053E32C00009AE5
:100AA0000820A0E10700A0E15C3084E204108DE2A0
:100AB000470200EB010070E30060A0E12D00000A96
:100AC000000050E32600000A0410DDE50050A0E31A
:100AD00005908DE2070000EA003094E5012083E2F2
:100AE000002084E50010C3E5015085E2060055E1D1
:100AF0001B00002A0110D9E4083094E5013043E2DC
:100B0000000053E3083084E5F2FFFFAA182094E5C3
:100B1000020053E10030A0B30130A0A30A0051E36A
:100B20000030A003000053E3EAFFFF1A0420A0E115
:100B30000700A0E117FFFFEB010070E3E9FFFF1AD8
:100B40000060A0E10600A0E10CD08DE2F043BDE81A
:100B50001EFF2FE1FF1008E20060A0E10410CDE5C8
:100B6000D9FFFFEA0860A0E10600A0E10CD08DE209
:100B7000F043BDE81EFF2FE1BC30D4E1403083E3F9
:100B8000BC30C4E1EEFFFFEAFC30D2E1020A13E31D
:100B900064C09205023A830302CA8C03BC30C201CE
:100BA00064C08205B2FFFFEA70402DE964309FE522
:100BB00064209FE503308FE0023093E7006093E507
:100BC000000056E30050A0E10140A0E10200000A4D
:100BD000383096E5000053E30B00000AFC30D4E106
:100BE000020A13E364209405023A8303022A820373
:100BF000642084050510A0E10420A0E10600A0E126
:100C0000BC30C4017040BDE899FFFFEA0600A0E1D6
:100C1000DEE8FFEBF0FFFFEAF883FE1F3400000080
:100C2000083092E5000053E39800000AF04F2DE9E8
:100C3000FC30D1E10338A0E1020713E30270A0E128
:100C400000A0A0E10140A0E10CD04DE22388A0E18A
:100C50002400000A102091E5000052E32100000A60
:100C6000029018E2006097E52900000A0090A0E3D6
:100C70000950A0E124B094E51C1094E568849FE538
:100C8000000055E31300000A080055E10530A031CB
:100C90000830A0210920A0E10A00A0E10FE0A0E1B6
:100CA0001BFF2FE1000050E3710000DA083097E5E8
:100CB000003043E0000053E3083087E5009089E00E
:100CC000005045E06100000A000055E324B094E5BF
:100CD0001C1094E5EBFFFF1A009096E5045096E592
:100CE000086086E2E5FFFFEA0410A0E10A00A0E147
:100CF00000FFFFEB000050E3F900001AFC30D4E1E4
:100D00000338A0E12388A0E1029018E2006097E593
:100D1000D5FFFF1A018018E25E00001A0850A0E11A
:100D200008B094E5000094E5000055E34300000A94
:100D3000020413E32338A0E19100000A05005BE1FF
:100D40000B20A0E1B800008A120D13E32300000A73
:100D5000142094E5101094E5822082E0019040E098
:100D6000A22F82E0010085E2C220A0E1090080E01C
:100D7000020050E102B0A09100B0A0810020A0814B
:100D8000010B13E3C300000A0210A0E10A00A0E176
:100D900050D6FFEB003050E2CD00000A0920A0E160
:100DA000101094E504308DE517D5FFEBBC20D4E19D
:100DB000122DC2E3802082E3BC20C4E104309DE513
:100DC000090083E014B084E509904BE00520A0E120
:100DD00005B0A0E1103084E5089084E5000084E5CA
:100DE0000590A0E10050A0E30810A0E104208DE5EB
:100DF0004DD5FFEB083094E504209DE50BB043E0B2
:100E0000003094E5022083E008B084E5002084E50A
:100E1000080097E5098088E0099040E0000059E368
:100E2000089087E50900000AFC30D4E1000055E392
:100E300008B094E5000094E50338A0E1BBFFFF1A79
:100E4000008096E5045096E5086086E2B5FFFFEA6B
:100E50000000A0E30CD08DE2F04FBDE81EFF2FE1B3
:100E60000410A0E10A00A0E111F9FFEB000050E33B
:100E70002A00000AFC30D4E10000E0E3403083E3C4
:100E8000BC30C4E10CD08DE2F04FBDE81EFF2FE175
:100E90000000A0E31EFF2FE10900A0E109B0A0E1DE
:100EA0000980A0E1240000EA000050E32B00000AC2
:100EB0000920A0E1020058E10820A031101094E5BB
:100EC000143094E5085094E5000094E5055083E063
:100ED000010050E10010A0930110A083050052E131
:100EE0000010A0D3000051E35E00001A020053E19D
:100EF000500000CA245094E50B20A0E10A00A0E1B4
:100F00001C1094E50FE0A0E115FF2FE1005050E226
:100F1000D7FFFFDA059059E00100A013CFFFFF0AC9
:100F2000083097E5053043E0000053E3083087E5DB
:100F300005B08BE0058048E0C4FFFF0A000058E3DD
:100F4000D8FFFF1A083086E2048013E5000058E35A
:100F50000360A0E108B013E5083083E2F9FFFF0A5F
:100F60000820A0E10A10A0E30B00A0E1DC0000EBE8
:100F7000000050E35300000A010080E20B9040E0C3
:100F8000CAFFFFEA103094E5000053E11200003A76
:100F9000149094E5050059E10F00008A060175E3FD
:100FA0000500A0310201E0230910A0E1AD0100EB32
:100FB0000820A0E1990003E01C1094E5249094E53A
:100FC0000A00A0E10FE0A0E119FF2FE1009050E23C
:100FD000A7FFFFDA095045E08CFFFFEA05005BE15F
:100FE0000B90A0310590A0210810A0E10920A0E1FC
:100FF000CDD4FFEB083094E5093043E0083084E5B8
:10100000000053E3003094E5093083E0003084E5CC
:10101000EFFFFF1A0410A0E10A00A0E1A4F8FFEB23
:10102000000050E3EAFFFF0A91FFFFEA05B0A0E1EC
:101030000520A0E169FFFFEA0B10A0E10250A0E14A
:1010400004208DE5B8D4FFEB083094E504209DE53D
:10105000023043E0083084E5003094E5022083E06C
:10106000002084E5AAFFFFEA0520A0E10B10A0E123
:10107000ADD4FFEB003094E5053083E00410A0E12F
:101080000A00A0E1003084E589F8FFEB000050E39E
:101090009FFFFF0A76FFFFEA0A00A0E10EF0FFEBD8
:1010A000003050E245FFFF1A0A00A0E1101094E55D
:1010B0003AD5FFEB0C20A0E3FC30D4E100208AE518
:1010C0008030C3E36BFFFFEA012088E20290A0E1D9
:1010D00077FFFFEA0C20A0E3FC30D4E100208AE592
:1010E00064FFFFEA0000E0E359FFFFEA00FCFF7F36
:1010F000F0432DE9BC30D1E13C819FE5020013E3D0
:1011000008808FE00140A0E15CD04DE20700000ABA
:101110000120A0E3433081E2003081E5103081E519
:10112000142081E55CD08DE2F043BDE81EFF2FE185
:10113000FE10D1E1000051E30060A0E1200000BA00
:101140000D20A0E1DB0000EB000050E31B0000BA23
:10115000019BA0E3027BA0E304509DE50F5A05E24A
:10116000023A45E2005073E20350A5E00910A0E105
:101170000600A0E157D5FFEB000050E31700000A7E
:10118000B8309FE5033098E73C3086E5FC30D4E189
:10119000000055E3803083E3149084E5000084E58B
:1011A000100084E5BC30C4E11800001A073083E168
:1011B000BC30C4E15CD08DE2F043BDE81EFF2FE1FE
:1011C000BC30D4E1805013E2019BA0030570A00164
:1011D0000050A0134090A0130570A011E2FFFFEA99
:1011E000FC30D4E1020C13E3CDFFFF1A0110A0E3A1
:1011F0000330C3E3432084E2023083E3BC30C4E124
:10120000002084E5102084E5141084E5C4FFFFEA83
:101210000600A0E1FE10D4E1BA0000EB000050E3AC
:10122000BC30D4110330C313013083130338A01131
:10123000FC30D4014338A011DBFFFFEAAC7EFE1F77
:101240000800000070402DE90140A0E1FE10D1E14E
:10125000000051E30250A0E10360A0E158D04DE24C
:101260000F0000BA0D20A0E1920000EB000050E357
:101270000B0000BA012BA0E3020BA0E304309DE5B4
:101280000F3A03E2021A43E2003071E20130A3E0B8
:10129000003086E5002085E558D08DE27040BDE83D
:1012A0001EFF2FE10030A0E3FC10D4E1800011E22A
:1012B000003086E50500000A4020A0E30300A0E11D
:1012C000002085E558D08DE27040BDE81EFF2FE17B
:1012D000013BA0E3003085E558D08DE27040BDE8C9
:1012E0001EFF2FE1030010E3FF1001E23400000AAB
:1012F000000052E30030A0E101C042E20200001A07
:10130000180000EA01C05CE21600003A0300A0E108
:101310000120D3E4010052E11EFF2F01030013E37B
:101320000300A0E1F6FFFF1A03005CE370402DE923
:101330000E00008A00005CE31E00000A0020A0E10D
:101340000C3080E0010000EA030052E11900000ABD
:101350000200A0E101C0D2E401005CE1F9FFFF1A44
:101360007040BDE81EFF2FE10000A0E31EFF2FE14B
:101370000020A0E1014481E14C609FE54C509FE5D5
:10138000044884E10200A0E1003090E5043023E04D
:1013900006E083E00330CEE1050013E1042082E2A1
:1013A000E5FFFF1A04C04CE203005CE30200A0E189
:1013B000F3FFFF8ADEFFFFEA0000A0E37040BDE814
:1013C0001EFF2FE102C0A0E1D6FFFFEAFFFEFEFEF6
:1013D0008080808070402DE94CC09FE54CE09FE507
:1013E0000CC08FE00EC09CE710D04DE2E0509CE5B1
:1013F00000C051E20C20A00104108D020360A0E1A6
:101400000040A0E10FE0A0E115FF2FE1010070E333
:101410000020A0038A30A003002086050030840548
:1014200010D08DE27040BDE81EFF2FE1CC7BFE1F87
:101430005400000070402DE90240A0E168C09FE523
:1014400068309FE50CC08FE003309CE7005093E5C7
:101450005C309FE503309CE7000050E310D04DE284
:10146000E06093E50120A0110230A0010010A0115E
:101470000020A0010430A0110500A0010500A0116A
:1014800004108D020FE0A0E116FF2FE1010070E3D0
:101490000020A0038A30A0030020840500308505C9
:1014A00010D08DE27040BDE81EFF2FE1687BFE1F6B
:1014B000340000005400000070402DE93C309FE5EE
:1014C0003CC09FE503308FE00C5093E70030A0E371
:1014D0000040A0E10100A0E10210A0E1003085E59C
:1014E000E9BCFFFB010070E30200001A003095E543
:1014F000000053E3003084157040BDE81EFF2FE16B
:10150000E87AFE1F0400000070402DE900E0A0E32F
:1015100034309FE534209FE503308FE0025093E79D
:101520000040A0E10100A0E100E085E52DE2FFEB35
:10153000010070E30200001A003095E5000053E35B
:10154000003084157040BDE81EFF2FE1947AFE1F25
:1015500004000000012051E21EFF2F013600003A76
:10156000010050E12200009A020011E12300000A6C
:101570000E0211E38111A0010830A0030130A01375
:10158000010251E3000051310112A0310332A031B8
:10159000FAFFFF3A020151E3000051318110A031FE
:1015A0008330A031FAFFFF3A0020A0E3010050E1B0
:1015B0000100402003208221A10050E1A100402031
:1015C000A3208221210150E12101402023218221F9
:1015D000A10150E1A1014020A3218221000050E39C
:1015E0002332B0112112A011EFFFFF1A0200A0E177
:1015F0001EFF2FE10100A0030000A0131EFF2FE13A
:10160000010851E32118A0211020A0230020A033BD
:10161000010C51E32114A02108208222100051E383
:101620002112A02104208222040051E3032082829F
:10163000A12082903002A0E11EFF2FE1000050E3C4
:101640000000E013BBD1FFEA000051E3FAFFFF0AFC
:1016500003402DE9BEFFFFEB0640BDE8920003E02A
:10166000031041E01EFF2FE1000051E34300000A98
:1016700001C020E000106142012051E22700000A71
:101680000030B0E100306042010053E12600009AD2
:10169000020011E12800000A0E0211E38111A001ED
:1016A0000820A0030120A013010251E303005131DF
:1016B0000112A0310222A031FAFFFF3A020151E3E8
:1016C000030051318110A0318220A031FAFFFF3A8E
:1016D0000000A0E3010053E101304320020080211B
:1016E000A10053E1A1304320A2008021210153E158
:1016F0002131432022018021A10153E1A131432066
:10170000A2018021000053E32222B0112112A01176
:10171000EFFFFF1A00005CE3000060421EFF2FE1B4
:1017200000003CE1000060421EFF2FE10000A033FA
:10173000CC0FA001010080031EFF2FE1010851E33F
:101740002118A0211020A0230020A033010C51E378
:101750002114A02108208222100051E32112A0218F
:1017600004208222040051E303208282A12082907F
:1017700000005CE33302A0E1000060421EFF2FE1A5
:10178000000050E30201E0C30201A0B369D1FFEA07
:10179000000051E3F9FFFF0A03402DE9B3FFFFEB1F
:1017A0000640BDE8920003E0031041E01EFF2FE178
:1017B00070402DE9FFC0A0E307CC8CE3214A1CE078
:1017C000235A1C100C0034110C0035117500000B4D
:1017D000054084E0036021E08C1AC1E18C3AC3E14A
:1017E000015690E103569211011681E3013683E31D
:1017F0001D00000A90C28EE00050A0E391E2A5E037
:10180000022106E290E3A5E00060A0E39153A6E088
:1018100000003CE301E08E13FF4044E2020C56E37B
:10182000034CC4E20200002A8EE0B0E10550B5E0AE
:101830000660A6E0861582E1A51A81E18505A0E192
:10184000AE0A80E18EE5A0E1FDC054E2070C5C83A6
:101850001100008A02015EE3A0E0B0010000B0E2E6
:10186000041AA1E07040BDE81EFF2FE1026106E20C
:10187000011086E1020080E1031021E0AC4054E059
:101880000C5074C0041A81C17040BDC81EFF2FC126
:10189000011681E300E0A0E3014054E25D0000CACC
:1018A000360074E30000A0D3021101D27040BDD80D
:1018B0001EFF2FD1004064E2204054E21A0000AA2B
:1018C0000C4094E20C0000CA144084E2205064E210
:1018D0001035A0E13004A0E1110580E1022101E210
:1018E0000211C1E3A30F90E03114A2E083E09EE176
:1018F000A30FC0017040BDE81EFF2FE10C4064E261
:10190000205064E21034A0E13005A0E1110480E130
:10191000021101E2A30F90E00010A1E283E09EE13A
:10192000A30FC0017040BDE81EFF2FE1205064E20C
:1019300010E58EE13034A0E1113583E13104A0E1FE
:10194000021101E23104C0E1A30F80E083E09EE1D7
:10195000A30FC0017040BDE81EFF2FE1000034E37B
:101960000800001A026101E28000B0E10110A1E06C
:10197000010611E301404402FAFFFF0A061081E16B
:10198000000035E31EFF2F11026103E28220B0E167
:101990000330A3E0010613E301504502FAFFFF0AFA
:1019A000063083E11EFF2FE10C0034E1235A0CE0E6
:1019B0000C0035110700000A816090E183609211EC
:1019C000E5FFFF1A031021E0021101E20000A0E38D
:1019D0007040BDE81EFF2FE1816090E10200A00190
:1019E0000310A001836092111000000A0C0034E182
:1019F0000100001A016690E10C00001A0C0035E1AC
:101A00000300001A036692E10200A0110310A01166
:101A10000600001A031021E0021101E27F1481E3A5
:101A20000F1681E30000A0E37040BDE81EFF2FE128
:101A30007F1481E33E1781E37040BDE81EFF2FE174
:101A400070402DE9FFC0A0E307CC8CE3214A1CE0E5
:101A5000235A1C100C0034110C0035115E00000BD1
:101A6000054044E003E021E0035692E10116A0E1C5
:101A70004C00000A0336A0E10152A0E3233285E1C5
:101A8000223C83E10224A0E1215285E1205C85E132
:101A90000064A0E102110EE2030055E102005601CC
:101AA000FD40A4E2034C84E20100002AA330B0E12F
:101AB0006220A0E1026056E00350C5E0A330B0E12F
:101AC0006220A0E10106A0E302C7A0E302E056E025
:101AD00003E0D5E0026046200E50A0210C008021DA
:101AE000A330B0E16220A0E102E056E003E0D5E0DF
:101AF000026046200E50A021AC008021A330B0E14E
:101B00006220A0E102E056E003E0D5E0026046205A
:101B10000E50A0212C018021A330B0E16220A0E171
:101B200002E056E003E0D5E0026046200E50A0211E
:101B3000AC01802106E095E10D00000A0552A0E10C
:101B4000265E85E10662A0E18331A0E1A23E83E149
:101B50008221A0E12CC2B0E1DBFFFF1A010611E3F4
:101B60000600001A001081E10000A0E302C1A0E31A
:101B7000D5FFFFEA010611E3001081010000A00378
:101B8000FDC054E2070C5C8343FFFF8A03C055E0AD
:101B900002C05600A0C0B0010000B0E2041AA1E0EB
:101BA0007040BDE81EFF2FE102E10EE221168EE13A
:101BB000AC4094E00C5074C0041A81C17040BDC8A0
:101BC0001EFF2FC1011681E300E0A0E3014054E2B3
:101BD00031FFFFEA06E085E12FFFFFEA235A0CE020
:101BE0000C0034E10C00350190FFFF0A0C0034E1D9
:101BF0000600001A014690E18CFFFF1A0C0035E147
:101C000083FFFF1A0200A0E10310A0E187FFFFEAB3
